:020000040800F2
:1000000000000120F5A60008DFA60008E1A6000810
:10001000E3A60008E5A60008E7A600080000000027
:10002000000000000000000000000000E9A6000839
:10003000EBA6000800000000EDA60008EFA60008EF
:1000400045A7000845A7000845A7000845A70008E0
:1000500045A7000845A7000845A7000845A70008D0
:1000600045A7000845A7000845A7000845A70008C0
:1000700045A7000845A7000845A7000845A70008B0
:1000800045A7000845A7000845A7000845A70008A0
:100090000000000045A7000845A7000845A7000884
:1000A00045A7000845A7000845A700088D330008AC
:1000B00045A7000845A7000845A7000845A7000870
:1000C00045A7000845A7000845A7000845A7000860
:1000D000C92D0008014F000845A7000845A70008E2
:1000E00045A70008618B000845A7000845A7000840
:1000F00045A70008000000000000000045A7000818
:1001000045A7000845A70008F58A000845A700088C
:1001100045A7000845A7000845A7000845A700080F
:1001200045A7000845A7000845A7000845A70008FF
:0801300045A7000845A70008DF
:1001380010B5054C237833B9044B13B10448AFF319
:1001480000800123237010BD28000020000000005B
:10015800F8C5000808B5034B1BB103490348AFF3C2
:10016800008008BD000000002C000020F8C5000831
:1001780010F8012B11F8013B012A28BF9A42F7D049
:10018800D01A7047034613F8012B002AFBD1181A1E
:100198000138704781F0004102E000BF83F000435E
:1001A80030B54FEA41044FEA430594EA050F08BF0A
:1001B80090EA020F1FBF54EA000C55EA020C7FEACE
:1001C800645C7FEA655C00F0E2804FEA5454D4EB4B
:1001D8005555B8BF6D420CDD2C4480EA020281EA15
:1001E800030382EA000083EA010180EA020281EA4D
:1001F8000303362D88BF30BD11F0004F4FEA01319F
:100208004FF4801C4CEA113102D0404261EB4101AD
:1002180013F0004F4FEA03334CEA133302D0524233
:1002280063EB430394EA050F00F0A780A4F10104EF
:10023800D5F1200E0DDB02FA0EFC22FA05F2801829
:1002480041F1000103FA0EF2801843FA05F359410F
:100258000EE0A5F120050EF1200E012A03FA0EFC8E
:1002680028BF4CF0020C43FA05F3C01851EBE371B8
:1002780001F0004507D54FF0000EDCF1000C7EEBD5
:1002880000006EEB0101B1F5801F1BD3B1F5001F13
:100298000CD349085FEA30004FEA3C0C04F1010432
:1002A8004FEA445212F5800F80F09A80BCF1004F5B
:1002B80008BF5FEA500C50F1000041EB045141EADD
:1002C800050130BD5FEA4C0C404141EB0101013CA6
:1002D80028BFB1F5801FE9D291F0000F04BF014695
:1002E8000020B1FA81F308BF2033A3F10B03B3F167
:1002F80020020CDA0C3208DD02F1140CC2F10C02F7
:1003080001FA0CF021FA02F10CE002F11402D8BF54
:10031800C2F1200C01FA02F120FA0CFCDCBF41EA20
:100328000C019040E41AA2BF01EB0451294330BDEF
:100338006FEA04041F3C1CDA0C340EDC04F11404CC
:10034800C4F1200220FA04F001FA02F340EA0300A3
:1003580021FA04F345EA030130BDC4F10C04C4F1E9
:10036800200220FA02F001FA04F340EA03002946C9
:1003780030BD21FA04F0294630BD94F0000F83F413
:10038800801306BF81F480110134013D4EE77FEAF6
:10039800645C18BF7FEA655C29D094EA050F08BF42
:1003A80090EA020F05D054EA000C04BF1946104623
:1003B80030BD91EA030F1EBF0021002030BD5FEA67
:1003C800545C05D14000494128BF41F0004130BD8F
:1003D80014F580043CBF01F5801130BD01F00045E3
:1003E80045F0FE4141F470014FF0000030BD7FEA56
:1003F800645C1ABF194610467FEA655C1CBF0B4651
:10040800024650EA013406BF52EA033591EA030F67
:1004180041F4002130BD00BF90F0000F04BF00215F
:10042800704730B54FF4806404F132044FF0000592
:100438004FF0000150E700BF90F0000F04BF00210B
:10044800704730B54FF4806404F1320410F0004571
:1004580048BF40424FF000013EE700BF42004FEA6C
:10046800E2014FEA31014FEA02701FBF12F07F43E9
:1004780093F07F4F81F06051704732F07F4208BFA0
:10048800704793F07F4F04BF41F40021704730B5A7
:100498004FF4607401F0004521F000411CE700BFF3
:1004A80050EA010208BF704730B54FF000050AE076
:1004B80050EA010208BF704730B511F0004502D577
:1004C800404261EB41014FF4806404F132045FEA79
:1004D800915C3FF4D8AE4FF003025FEADC0C18BF22
:1004E80003325FEADC0C18BF033202EBDC02C2F114
:1004F800200300FA03FC20FA02F001FA03FE40EAA6
:100508000E0021FA02F11444BDE600BF70B54FF0A9
:10051800FF0C4CF4E06C1CEA11541DBF1CEA135587
:1005280094EA0C0F95EA0C0F00F0DEF82C4481EAEF
:10053800030621EA4C5123EA4C5350EA013518BF0F
:1005480052EA033541F4801143F4801338D0A0FBFC
:1005580002CE4FF00005E1FB02E506F00042E0FBA9
:1005680003E54FF00006E1FB03569CF0000F18BFAF
:100578004EF0010EA4F1FF04B6F5007F64F5407457
:1005880004D25FEA4E0E6D4146EB060642EAC621EA
:1005980041EA55514FEAC52040EA5E504FEACE2E57
:1005A800B4F1FD0C88BFBCF5E06F1ED8BEF1004F5A
:1005B80008BF5FEA500E50F1000041EB045170BDD6
:1005C80006F0004646EA010140EA020081EA03011A
:1005D800B4EB5C04C2BFD4EB0C0541EA045170BD16
:1005E80041F480114FF0000E013C00F3AB8014F190
:1005F800360FDEBF002001F0004170BDC4F10004D9
:10060800203C35DA0C341BDC04F11404C4F1200559
:1006180000FA05F320FA04F001FA05F240EA0200B4
:1006280001F0004221F0004110EBD37021FA04F6EA
:1006380042EB06015EEA430E08BF20EAD37070BDA4
:10064800C4F10C04C4F1200500FA04F320FA05F003
:1006580001FA04F240EA020001F0004110EBD37005
:1006680041F100015EEA430E08BF20EAD37070BD75
:10067800C4F1200500FA05F24EEA020E20FA04F34E
:1006880001FA05F243EA020321FA04F001F00041FD
:1006980021FA04F220EA020000EBD3705EEA430E6E
:1006A80008BF20EAD37070BD94F0000F0FD101F09D
:1006B8000046400041EB010111F4801F08BF013CD6
:1006C800F7D041EA060195F0000F18BF704703F014
:1006D8000046520043EB030313F4801F08BF013D9B
:1006E800F7D043EA0603704794EA0C0F0CEA135557
:1006F80018BF95EA0C0F0CD050EA410618BF52EA11
:100708004306D1D181EA030101F000414FF0000016
:1007180070BD50EA410606BF1046194652EA430624
:1007280019D094EA0C0F02D150EA013613D195EA98
:100738000C0F05D152EA03361CBF104619460AD1E0
:1007480081EA030101F0004141F0FE4141F47001EA
:100758004FF0000070BD41F0FE4141F4780170BDDA
:1007680070B54FF0FF0C4CF4E06C1CEA11541DBF3F
:100778001CEA135594EA0C0F95EA0C0F00F0A7F841
:10078800A4EB050481EA030E52EA03354FEA01316E
:1007980000F088804FEA03334FF0805545EA131381
:1007A80043EA12634FEA022245EA111545EA106549
:1007B8004FEA00260EF000419D4208BF964244F1E0
:1007C800FD0404F5407402D25B084FEA3202B61AFF
:1007D80065EB03055B084FEA32024FF480104FF4D3
:1007E800002CB6EB020E75EB030E22BFB61A754647
:1007F80040EA0C005B084FEA3202B6EB020E75EBDA
:10080800030E22BFB61A754640EA5C005B084FEA41
:100818003202B6EB020E75EB030E22BFB61A75460E
:1008280040EA9C005B084FEA3202B6EB020E75EB19
:10083800030E22BFB61A754640EADC0055EA060EDA
:1008480018D04FEA051545EA16754FEA06164FEA1D
:10085800C30343EA52734FEAC2025FEA1C1CC0D1C9
:1008680011F4801F0BD141EA00014FF000004FF056
:10087800004CB6E711F4801F04BF01430020B4F117
:10088800FD0C88BFBCF5E06F3FF6AFAEB5EB030CCF
:1008980004BFB6EB020C5FEA500C50F1000041EBCC
:1008A800045170BD0EF0004E4EEA113114EB5C0499
:1008B800C2BFD4EB0C0541EA045170BD41F480116C
:1008C8004FF0000E013C90E645EA060E8DE60CEA74
:1008D800135594EA0C0F08BF95EA0C0F3FF43BAF91
:1008E80094EA0C0F0AD150EA01347FF434AF95EA48
:1008F8000C0F7FF425AF104619462CE795EA0C0F2C
:1009080006D152EA03353FF4FDAE1046194622E7F8
:1009180050EA410618BF52EA43067FF4C5AE50EAD2
:1009280041047FF40DAF52EA43057FF4EBAE12E7C2
:100938004A0011D212F5001211D20DD56FF4787356
:10094800B3EB62520ED44FEAC12343F0004343EAAB
:10095800505323FA02F070474FF00000704750EAF6
:10096800013002D14FF0FF3070474FF00000704760
:1009780080F0004002E000BF81F0004142001FBF4C
:100988005FEA410392EA030F7FEA226C7FEA236C55
:100998006AD04FEA1262D2EB1363C1BFD21841404A
:1009A80048404140B8BF5B42192B88BF704710F0E0
:1009B800004F40F4000020F07F4018BF404211F083
:1009C800004F41F4000121F07F4118BF494292EAEB
:1009D800030F3FD0A2F1010241FA03FC10EB0C0017
:1009E800C3F1200301FA03F100F0004302D54942A4
:1009F80060EB4000B0F5000F13D3B0F1807F06D351
:100A080040084FEA310102F10102FE2A51D2B1F148
:100A1800004F40EBC25008BF20F0010040EA03003D
:100A28007047490040EB0000013A28BFB0F5000FBD
:100A3800EDD2B0FA80FCACF1080CB2EB0C0200FA73
:100A48000CF0AABF00EBC25052421843BCBFD040C2
:100A58001843704792F0000F81F4000106BF80F43C
:100A680000000132013BB5E74FEA41037FEA226CFF
:100A780018BF7FEA236C21D092EA030F04D092F0CA
:100A8800000F08BF0846704790EA010F1CBF0020FE
:100A9800704712F07F4F04D1400028BF40F000405B
:100AA800704712F100723CBF00F50000704700F07B
:100AB800004343F0FE4040F4000070477FEA2262A2
:100AC80016BF08467FEA23630146420206BF5FEA73
:100AD800412390EA010F40F4800070474FF0000373
:100AE80004E000BF10F0004348BF40425FEA000C3A
:100AF80008BF704743F0964301464FF000001CE0E2
:100B080050EA010208BF70474FF000030AE000BF37
:100B180050EA010208BF704711F0004302D5404275
:100B280061EB41015FEA010C02BF844601460020E7
:100B380043F0B64308BFA3F18053A3F50003BCFA02
:100B48008CF2083AA3EBC25310DB01FA02FC6344AF
:100B580000FA02FCC2F12002BCF1004F20FA02F2B6
:100B680043EB020008BF20F00100704702F12002A9
:100B780001FA02FCC2F1200250EA4C0021FA02F20A
:100B880043EB020008BF20EADC7070474FF0FF0C0F
:100B98001CEAD0521EBF1CEAD15392EA0C0F93EA0A
:100BA8000C0F6FD01A4480EA010C400218BF5FEAAC
:100BB80041211ED04FF0006343EA501043EA51111F
:100BC800A0FB01310CF00040B1F5000F3EBF490019
:100BD80041EAD3715B0040EA010062F17F02FD2A1D
:100BE8001DD8B3F1004F40EBC25008BF20F0010000
:100BF800704790F0000F0CF0004C08BF49024CEA17
:100C0800502040EA51207F3AC2BFD2F1FF0340EAA8
:100C1800C250704740F400004FF00003013A5DDC19
:100C280012F1190FDCBF00F000407047C2F100025A
:100C3800410021FA02F1C2F1200200FA02FC5FEA47
:100C4800310040F1000053EA4C0308BF20EADC7091
:100C5800704792F0000F00F0004C02BF400010F403
:100C6800000F013AF9D040EA0C0093F0000F01F0B0
:100C7800004C02BF490011F4000F013BF9D041EAD2
:100C88000C018FE70CEAD15392EA0C0F18BF93EAD4
:100C98000C0F0AD030F0004C18BF31F0004CD8D1FE
:100CA80080EA010000F00040704790F0000F17BF85
:100CB80090F0004F084691F0000F91F0004F14D0CB
:100CC80092EA0C0F01D142020FD193EA0C0F03D123
:100CD8004B0218BF084608D180EA010000F0004026
:100CE80040F0FE4040F40000704740F0FE4040F401
:100CF800400070474FF0FF0C1CEAD0521EBF1CEAA0
:100D0800D15392EA0C0F93EA0C0F69D0A2EB0302BD
:100D180080EA010C49024FEA402037D04FF0805357
:100D280043EA111143EA10130CF000408B4238BF1C
:100D38005B0042F17D024FF4000C8B4224BF5B1A2A
:100D480040EA0C00B3EB510F24BFA3EB510340EA78
:100D58005C00B3EB910F24BFA3EB910340EA9C0026
:100D6800B3EBD10F24BFA3EBD10340EADC001B0196
:100D780018BF5FEA1C1CE0D1FD2A3FF650AF8B423A
:100D880040EBC25008BF20F0010070470CF0004C47
:100D98004CEA50207F32C2BFD2F1FF0340EAC25072
:100DA800704740F400004FF00003013A37E792F033
:100DB800000F00F0004C02BF400010F4000F013A91
:100DC800F9D040EA0C0093F0000F01F0004C02BF8C
:100DD800490011F4000F013BF9D041EA0C0195E7F5
:100DE8000CEAD15392EA0C0F08D142027FF47DAF8E
:100DF80093EA0C0F7FF470AF084676E793EA0C0F7E
:100E080004D14B023FF44CAF08466EE730F0004C7B
:100E180018BF31F0004CCAD130F000427FF45CAF0B
:100E280031F000437FF43CAF5FE700BF4FF0FF3C79
:100E380006E000BF4FF0010C02E000BF4FF0010CCC
:100E48004DF804CD4FEA40024FEA41037FEA226C95
:100E580018BF7FEA236C11D001B052EA530C18BFB7
:100E680090EA010F58BFB2EB030088BFC81738BF1C
:100E78006FEAE17018BF40F0010070477FEA226C0A
:100E880002D15FEA402C05D17FEA236CE4D15FEA06
:100E9800412CE1D05DF8040B704700BF844608463A
:100EA8006146FFE70FB5FFF7C9FF002848BF10F1FB
:100EB800000F0FBD4DF808EDFFF7F4FF0CBF012040
:100EC80000205DF808FB00BF4DF808EDFFF7EAFFCA
:100ED80034BF012000205DF808FB00BF4DF808ED85
:100EE800FFF7E0FF94BF012000205DF808FB00BF7A
:100EF8004DF808EDFFF7D2FF94BF012000205DF800
:100F080008FB00BF4DF808EDFFF7C8FF34BF01200C
:100F180000205DF808FB00BF4FEA4002B2F1FE4F27
:100F28000FD34FF09E03B3EB12620DD94FEA0023A3
:100F380043F0004310F0004F23FA02F018BF40427C
:100F480070474FF00000704712F1610F01D1420263
:100F580005D110F0004008BF6FF0004070474FF017
:100F68000000704742000ED2B2F1FE4F0BD34FF093
:100F78009E03B3EB126209D44FEA002343F0004307
:100F880023FA02F070474FF00000704712F1610F2A
:100F980001D1420202D14FF0FF3070474FF00000FC
:100FA800704700BF0022427082700122C270B1FAFD
:100FB80081F10222490902710322017042717047CE
:100FC80043788B421FD0012941700AD0022910D0E2
:100FD800C1B90123C37081700223037103234371D4
:100FE8007047037843B1012383700223C370002341
:100FF800F3E70378002BF6D0022383700023C37035
:101008000123EAE7FEE7704782B00B88ADF80030AD
:101018004B88ADF802308B88ADF80430CB88ADF83A
:1010280006300239431C053013F8012F0DF1080C66
:101038000CEB4202834232F8082C21F8022FF3D13C
:1010480002B0704708448078704738B54FF07F3356
:10105800C0F8A03004464FF6FF737F220025A0F8A1
:10106800A43080F8A62080F8A950A0F8AA30AC30A7
:1010780000F04BFD84F8B85038BD70B511461546E0
:1010880004461E4600F0E8FC294604F1140000F06E
:10109800E3FC294604F1280000F0DEFC294604F1AF
:1010A8003C0000F0D9FC294604F1500000F0D4FCC3
:1010B800294604F1640000F0CFFC294604F17800C9
:1010C80000F0CAFC294604F18C0000F0C5FC04F1CC
:1010D800AC0032464FF4FA734FF4FA6100F0FBFCAF
:1010E8002046BDE87040FFF7B0BF704700F0BBBCBA
:1010F800143000F0B8BC283000F0B5BC90F8A4302B
:1011080013B990F9A000704790F9A100704790F8C2
:10111800A43013B990F9A200704790F9A300704762
:1011280010B5044607F03EFF38B104F1140000F092
:101138009EFC012838BF0120C0B210BD10B504467E
:1011480007F030FF38B104F1500000F090FC01289E
:1011580038BF0120C0B210BD4FF47A71AC3000F036
:10116800DBBC0021AC3000F0D7BC08B5AC3000F0D7
:10117800E4FCB0F57A7FA8BF4FF47A7020EAE070FB
:1011880008BD10B5044600F048FC04F1140000F056
:1011980044FC04F1280000F040FC04F13C0000F09D
:1011A8003CFC04F1500000F038FC04F1640000F04D
:1011B80040FC04F17800BDE8104000F03ABC7F28FC
:1011C80007D0002807DA10F1800F06D04042C0B2DD
:1011D800704700207047012070477F20704710B18A
:1011E800404240B270477F2070477F280FD010F1EF
:1011F800310F0EDA10F1780F0DDB7830FE2340B294
:10120800584323304623B0FBF3F0C0B27047FF20A9
:101218007047FE207047002070477F2805D031B105
:10122800002806DA4042C0B27047FF207047FE200F
:101238007047002070477F2811D010F1310F10DA65
:1012480010F1780F10DB783040F2A96340B25843B0
:1012580023304623B0FBF3F0AC3080B27047002057
:10126800704740F255707047AC20704763289FBFA5
:1012780040F2A9635843323064239DBFB0FBF3F0BA
:10128800AC3080B240F2557070474FF4F063A0F56F
:101298008060584340F2FF7390FBF3F000F57870DC
:1012A80080B27047FFF7F1BF4FF49663A0F58060F6
:1012B800584340F2FF7390FBF3F000F2DC5080B229
:1012C8007047A0F58060D0EB001048BF033040F3B2
:1012D8008F007047032812DD0C2812DD0F2812DD5D
:1012E800122812DD162812DD192812DD1C2812DD3D
:1012F8001F2812DD2128CCBFFF20062070470020C0
:10130800704701207047022070470820704703206B
:101318007047072070470420704705207047000079
:1013280005289ABF014B185CFF2070477DC600084E
:101338007F281ABF4042C0B2002070477F2811D0D2
:1013480010F1320F10DA884210DD401A6423C1F11F
:10135800FF21584301F57F01CE31313090FBF1F088
:10136800C0B27047FF207047642070470020704764
:10137800014B4840185C704784C6000852B110B44D
:10138800054C0A4411F8013B58408A42205CF9D1C7
:1013980010BC7047704700BF84C60008002805DBF2
:1013A800212805DC044B33F81000704700207047F3
:1013B8004FF4FA60704700BFAEC70008392808D854
:1013C80022280ED9094B2338C0B2C34003F00100CC
:1013D80070475F2807D0613819288CBF002001208A
:1013E8007047002070470120704700BF01EC7F0064
:1013F800F8B50246451E461D00245F2715F8010F63
:10140800FF2804BF0134E4B2FFF7D8FF00B92F70FA
:10141800AE42F3D1062C04D119B10B6813608B8846
:10142800938000239371F8BD2DE9F843DFF83490D9
:10143800471E441D012500264FF0280817F8011FF4
:1014480008480BF07CF8034610B1A0EB0903DBB2A7
:10145800A3FB05329E19A742A5FB0853EED13046DF
:10146800BDE8F88384C7000810B54179A1F13000C0
:10147800C3B2092B07D80523B0FBF3F303EB8303AF
:10148800C01AC0B210BD044C20460BF058F8002812
:10149800F1D0001BC0B2EEE784C7000870B504465F
:1014A800FEF770FE82B20023551E98B2A84214FAC5
:1014B80083F104DA265C302E03F10103F5D0121A09
:1014C80001322046BDE870400BF008B82DE9F04F16
:1014D8000D4699B0164600211A461F4680460BF065
:1014E80017F800212A2201A800910BF011F8DFF863
:1014F800CC90DFF8CCA0DFF8CCB005EB4606AE42C6
:1015080011D16846FEF73EFE30B100F160030DEBE5
:101518000300002300F8613C694640460BF052F88E
:1015280019B0BDE8F08F35F9020B47F6FF73984202
:10153800E7D0002812DC59460CA80BF043F868469F
:10154800FEF720FE04460CA8FEF71CFE0444A74242
:10155800D5D30CA968460AF0E3FFD0E7B0F57A7F47
:101568000BDA0CA980B20AF0F1FB0CA8FFF796FF82
:1015780051460CA80AF0D4FFE1E764230CA93230E5
:10158800B0FBF3F080B20AF0E1FB0CA8FFF786FF8E
:101598000CA8FEF7F7FD00F15F036B4400F1600152
:1015A8000DEB010013F8302C00F8302C2E2203F834
:1015B800302C002300F82F3C4946DAE73AC60008E9
:1015C80035C6000830C60008F0B589B06D4600245D
:1015D8002F468E1CE1B28A4204D83946FFF776FFBF
:1015E80009B0F0BD36F8241025F8021B0134F1E7E4
:1015F80042F210736421B0FBF3F203FB1200B0FB5C
:10160800F1F301FB130000EB023000EB831080B212
:10161800704770B50E460021054614460AF078FF5B
:1016280000239AB2944200D870BDF25C002AFBD025
:10163800EA540133F5E70000052911D8DFE801F085
:101648000306080A0C0E0749FFF7E3BF0649FBE744
:101658000649F9E70649F7E70649F5E70649F3E7D2
:101668000649F1E73EC6000843C6000848C6000818
:101678004DC6000852C6000857C600085CC60008D8
:10168800052911D8DFE801F00306080A0C0E0749FE
:10169800FFF7BFBF0649FBE70649F9E70649F7E741
:1016A8000649F5E70649F3E70649F1E75EC600088B
:1016B80063C6000868C600086DC6000872C6000840
:1016C80076C600085CC6000870B50E4614460021B0
:1016D800013205460AF01CFF00239AB2944200D852
:1016E80070BDF25C002AFBD0EA540133F5E7914261
:1016F80006D19DF900008342CCBF0020012070472D
:1017080003290DD0032A09D0022909D0022A05D0BD
:10171800012905D0531E584258417047012070478F
:10172800002070477D23438043F2390309B2C36028
:10173800002301808180C38003727047C268044916
:10174800044B01FB023323F00043C360980F70473A
:10175800FD430300C39E260010B501290446807985
:101768000ED8042801D80130A071012AE0790BD8DD
:10177800042801D80130E071032925D14B2319E051
:101788000028F2D00138EFE708B10138E0710329E9
:101798000AD1032A18D19DF90820934208DC3ADAC5
:1017A80023885B421BB205E002290DD1022AF1E72A
:1017B800B4F9003062881A4412B27C2A30DD7D22E6
:1017C8006280002222722FE09142D7D825D30129C6
:1017D80010D1012A0ED1A279E3799A4208D302D90D
:1017E8006FF07C03E6E72046FFF7A8FF0028F7D054
:1017F8007D23DFE7B4F90400B4F900302288B4F996
:101808000210002804DB7C29D4DD524213B2D1E750
:101818007C31CFDBF9E70023CCE76FF04A03C9E757
:1018280012F17C0F02DB6280A38010BD4FF6837239
:1018380062800122C6E7000002680449044B01FBEC
:10184800023323F000430360180C7047FD43030084
:10185800C39E2600F0B5002597B001608580044638
:101868005622294668460AF053FE0126E27DAA421E
:1018780009D80023802104F1B800A37517B0BDE88A
:10188800F0400AF045BE2046FFF7D6FFE7797B1BFC
:10189800002190FBF3F202FB1300C0B2EC460A46AB
:1018A800CBB29F4223D800230022277B1146D0B217
:1018B800874227D80029D9D1A279033A012A04EB13
:1018C800050105D925B191F9172012BB012BCDD9F6
:1018D8000B76A26852F82310583305F10E026B44B8
:1018E800013544F8221003F8586CEDB2BEE71CF835
:1018F80001EBBEF1000F03D18242D5D00132D2B242
:101908000131CDE72069805C0132984208BF01218E
:10191800CDE7501E8342DBDB01329342D8DCA5E7DA
:101928002DE9F047154696B0013D01600271044665
:101938004371EDB25622002168460AF0E9FD0027FE
:10194800022D84BF4FF0010900253E464FF0010AE1
:1019580094F807809CBF4FF00309B8FBF9F8E27DC3
:10196800B24209D80023802104F1B800A37516B04B
:10197800BDE8F0470AF0CCBD2046FFF75DFFA8EBB5
:101988000603002190FBF3F202FB1300C0B2EC4601
:101998000A46CBB2434506D21CF801EBBEF1000F54
:1019A8002AD1824226D1434528BF434603FB095129
:1019B800002094F80CE001F0FF018446C2B296457D
:1019C8001CD8BCF1000FCAD116B1FFB9012BC6D97A
:1019D800A2191F461176A26852F8211006F10E02CC
:1019E800013644F8221003F158026A44F6B202F8AC
:1019F80058ACB4E70132D2B20131CAE72269125CAD
:101A080001308A4208BF4FF0010CD7E77A1E934293
:101A1800DEDB7A1C9342DBDCA1E7D0E901236421F9
:101A2800D31AC36082604B43418AB3FBF1F303745A
:101A38007047D0E90123D31AC0E9022370474368ED
:101A48002BB1C26864214A43B2FBF3F2D3B20374E8
:101A58000023C360436070470023C0E9023341821A
:101A68004360037470474368013343607047007CE8
:101A7800704743680B44436070470023C0E9013353
:101A8800C36003747047F0B5047C0360012C11D95E
:101A980044688568C668141B4FF47A774D1B7C43ED
:101AA80005FB16442B4494FBF3F33344C360C0E9AD
:101AB8000121F0BD1CB9C46001230374F7E7436832
:101AC8004FF47A74D31A634384680C1B93FBF4F3C2
:101AD800C3600223F1E72DE9F041044610461D4694
:101AE80016468846FEF7FAFF074606EB0800FEF79B
:101AF800F5FF01463846FFF7FDF865602060284687
:101B0800FEF7F0FFA060BDE8F08110B5044640681C
:101B1800FEF7E8FFA06010BD38B5856804460846A2
:101B2800FEF7E0FF2946FEF727FF2168FFF72EF8AA
:101B38002946FEF723FFA06038BD08B54FF07C5159
:101B48008068FEF71BFFFFF7E7F908BD704770478D
:101B5800704700207047704700207047002070478A
:101B6800704700207047002070474FF0B04382B0A4
:101B7800DA6C0243DA64DB6C03400193019B02B028
:101B880070474FF0B04382B09A6D02439A659B6DDF
:101B980003400193019B02B070474FF0B04382B0FD
:101BA8001A6E02431A661B6E03400193019B02B032
:101BB800704750E8003F23F0800340E80032002AD5
:101BC800F7D17047044B1888044B1B8880B29BB22E
:101BD800C01A18BF0120704734290020322900207C
:101BE800704700000288044B5140C9B233F81130E5
:101BF80083EA12230380704728E000089AB110B4E2
:101C0800B0F800C0084C0A4411F8013B83EA0C0301
:101C1800DBB2914234F8133083EA1C2CA0F800C0E0
:101C2800F2D110BC7047704728E0000837B54FF66E
:101C3800FF730446ADF806304518AC4203D1BDF831
:101C4800060003B030BD14F8011B0DF10600FFF7C4
:101C5800C9FFF2E708B5FFF7B5FF003818BF012044
:101C680008BD0020704700000278024B51405B5CC1
:101C7800037070479CCC0008FF230370704700BFB7
:101C8800704770B50B7803704B7843700B78FD2B59
:101C980005460C4638D18B788370CB78C3700B79A6
:101CA80003714B7943718B7983718B68C3718B682E
:101CB800C3F30F2303728B7A43720A26627804F106
:101CC8000C01A8190AF086FC6378B4F80C21334497
:101CD800981CEA545A1CB4F80C1192B2090AA95477
:101CE800A278D20780B20ED504F58872054404F5AF
:101CF8008E7452F8041B45F8041BA242F9D11278DD
:101D08002A700F3398B270BD00238B700B798370E3
:101D18004B79C3708B7903718B6843710626CDE7C5
:101D280008B52422034800210AF0F2FB024B0022E6
:101D38001A7008BD28060020F80200202DE9F0419D
:101D48001378037092F8018080F80180FD2B044617
:101D58000F46154654D193788370D378C37013799E
:101D6800037153794371937983716B7A127A1B04E7
:101D780003EB0223EA79134423F07F430A26A2687F
:101D880063F31702A260A919424604F10C000AF095
:101D980021FC7A7B904507D208F10C00A2EB0802DF
:101DA800002120440AF0B4FB63781E44AB195A782A
:101DB800AB5D03EB0223A4F80C31A378DB070ED547
:101DC800023615FA86F304F5887203F10C0153F80C
:101DD800040B42F8040B8B42F9D11B781370BB7AC1
:101DE80084F82131FB7A84F822313B7B84F8233153
:101DF8007B7B84F824313B7884F82031BDE8F0817E
:101E08000023438093780371D378437113798371E6
:101E180053790626B3E7000070B50D4C0D4E054604
:101E2800062204F10A0106F58970FFF74DFC237CB0
:101E3800C3F3031386F81A31637CC3F3030386F8EC
:101E48001B31637ADB0744BF02232B7370BD00BFCD
:101E58001D1F0020A400002070B50446BDF81450D2
:101E6800E2702420237122461B0A207063715820D7
:101E78002B0AA1706070A57102F8073F049B5919DD
:101E88008B420CD16A1D92B2E11C0020FFF776FA52
:101E980005F10806A05505F1090080B270BD13F8D8
:101EA800010B02F8010FEBE70A4A0B4B12680B49CA
:101EB800A3FB02323220920C00FB02F2084B486866
:101EC80002F5FA72A3FB023292094B681B1A9A4276
:101ED800FBD870471C00002083DE1B43001000E085
:101EE800D34D621008B5FFF7DFFF024B4FF4805265
:101EF8009A6108BD00040048024B4FF480529A6270
:101F0800FFF7D2BF0004004802780A4B90F801C0DE
:101F18008178D243D2B29A5C82EA0C0290F803C06C
:101F28009A5C4A40995C027981EA0C01595C4A4002
:101F3800985C70479CCC0008F8B53C29BDF81C504B
:101F4800044635D0A1F12106714271414900D007FC
:101F580048BF41F00801E37092074FEA13234FF09E
:101F6800240248BF41F01001227023716F222B0A0E
:101F7800A61C6270A170A37165713046FFF7C4FF9B
:101F88002246069B02F8070F59198B4212D1A91D48
:101F980089B23046FFF74AFE05F1080705F1090343
:101FA8009BB2E055000AE05405F10A0080B2F8BD82
:101FB8000121CCE713F8010B02F8010FE5E7000057
:101FC800074B084A5B6A02F5006353E8003F43F099
:101FD800200302F5006040E800310029F3D1704782
:101FE80000380140003001402DE9F04F0C4651887F
:101FF800B1F58C7F85B0054611D300211170D91C2D
:10200800C9B2012995BF01210023518053809CBF8B
:102018002370117000232B7005B0BDE8F08F107885
:102028000E2800F28B8001A656F820F00720000841
:102038007120000899200008B320000845210008F5
:1020480045210008452100084521000845210008D0
:1020580045210008452100084521000845210008C0
:1020680045210008C5200008481C50806354217889
:10207800FD299BB206D10C330A21D380918002231B
:102088001370C7E708330621D38091800E23F7E742
:10209800481C50806354D80742BFD1880D31D18085
:1020A800012B8CBF00230323EAE7002B01F1010079
:1020B8005080635414BF00230E23E1E7481C50806E
:1020C80063545388D1888B4232D3002353801370D2
:1020D80002232B7069802378FD2B35D163792B720D
:1020E800A3796B72637A227A1B0403EB0223E279E9
:1020F80013446B60637803F10C026A80A278D107FD
:1021080001D519336B8000266968DFF8F0806E818D
:102118004FF4BC720C20B31801335B0800FB03F7C3
:1021280058F80770B94218D25A1EB242F3D816E0CE
:1021380092889A423FF66EAF01236CE70023137032
:1021480053809380D38066E7E3782B7223796B7290
:1021580063796B6063780833D4E71E46E5D80C27AB
:10216800774358F80730994227D123782046FD2B2A
:1021780010F801BF0CBF4FF00A094FF0060909EB30
:102188000B03591E89B247440193FFF74FFD97F897
:1021980004A0ADF80E0051460DF10E00FFF722FD28
:1021A800019BE218E35C527803EB0223BDF80E2092
:1021B8009BB29A4203D005232DE703232BE7BB7973
:1021C800DA0706D5FA79934582BF04EB09018A5CE0
:1021D800AA729B0709D50C2303FB068362781B7A36
:1021E8009A4282BF4C44E35CEB720C2303FB0683E8
:1021F80085F80CA05B796B730EE700BF9CCD0008D7
:10220800F0B50546FD2305F80C3B85B004468DF86E
:10221800043090F8243103F10C020244012B42D817
:102228000026637066808DF805308B7A23718DF8EF
:1022380008308B7AADF8066001338B7263798DF8BC
:102248000930A3798DF80A30A368C3F317031A126B
:102258008DF80B3009211B140DF105008DF80D3098
:102268008DF80C20FFF7E2FC6778ADF802003A46DB
:1022780029460DF10200FFF7C1FC94F82311FFF77E
:10228800B1FC94F82421BDF80230A4F80C3197422F
:1022980010D207F10C00D21B3146204405B0BDE82E
:1022A800F0400AF035B912F8010D0028B8D1013B09
:1022B800DBB2B3E705B0F0BD044A00231380044A3B
:1022C8001380044A1380044A13807047322900207F
:1022D80034290020362D0020382D0020044AD2F859
:1022E800903023F40043C2F89030FFF7DDBD00BF03
:1022F8000004005808B5FFF7D7FD044AD2F890301B
:1023080043F40043C2F8903008BD00BF00040058F1
:1023180007B503688DF807101B6901220DF1070145
:10232800984703B05DF804FB70B5044608460D46AF
:10233800FDF728FF236882B2294620461B69BDE8BD
:1023480070401847B0F1904F02D10120FFF70DBC43
:10235800084B984205D003F58063984203D10420C6
:10236800F4E70220F2E7044B984201D18020EDE720
:10237800704700BF00040048001C00480C4B9842FE
:1023880003D14FF40060FFF708BCB0F1804F05D0CF
:10239800084B984205D14FF40030F4E70120FFF7CD
:1023A800F0BB054B984202D14FF48020EBE7704711
:1023B800002C014000440140004801402DE9F04351
:1023C80087B00E46054614460021142201A89DF840
:1023D80038809DF83C901F460AF09AF800960B2C1E
:1023E80007D8DFE804F007070A12141414161616A3
:1023F8001A1CFEE70323019301E002230493032F31
:1024080011D8DFE807F0111321110123F6E70123A2
:10241800F1E7012301930393F1E70223EBE702239A
:1024280001930123F7E7FEE702230293B8F1100FA7
:102438000CD8DFE808F02D2D0C11131517191B1DEA
:102448001F21232527292B000123EEE7FEE701237F
:102458000593022301931EE00223F9E70323F7E71C
:102468000423F5E70523F3E70623F1E70723EFE75E
:102478000823EDE70923EBE70A23E9E70B23E7E75E
:102488000C23E5E70D23E3E70E23E1E70F23DFE75E
:10249800B8F1000FDDD1B9F1000F02D02846FFF7DF
:1024A80051FF053C042C05D8DFE804F0030B0403B6
:1024B8000B00AE626946284608F0DCFF07B0BDE8AD
:1024C800F083AE61F6E713B54FF0010C0024CDE9B7
:1024D800004CFFF773FF02B010BD000030B587B0A5
:1024E800002315460446ADF80630FFF747FF042DD4
:1024F80004D8DFE805F02E3204363F00FEE71E4B15
:102508001E4A1B68B3FBF2F39BB20022CDE90221FD
:10251800013B01A92046ADF804300492059209F068
:10252800D5F9236823F080032360A36823F4A0333C
:1025380023F00703A360636823F070036360636894
:1025480023F470036360A36823F08003A36007B0DB
:1025580030BD094B0A4A1B68D4E7074B094A1B6878
:10256800D0E7054B064A1B68B3FBF2F303EB830382
:102578005B00C9E70123C8E71C00002080A81201FE
:1025880040420F0000127A0010B50446FFF7A6FF7C
:10259800236843F00103236010BD00224FF0FF3190
:1025A800FFF7F2BF1A4B10B51A4C5B68236008F0AE
:1025B800C7F84FF0904008F01FFF174808F01CFFBD
:1025C800164808F019FF164809F00EFB154809F0DF
:1025D8000BFB09F0ADF84FF0E022002313615361C3
:1025E800936172B64FF0FF319A0002F1604202F532
:1025F80061420133082BC2F88010C2F88011F3D170
:1026080062B6034B1B6883F3088823689847FEE784
:102618000000FF1FF40200200004004800080048E2
:1026280000380140004400400749084A881AEFF37F
:102638000883521A1A44013A013B984288BF002283
:10264800AA2109F065BF00BF0000012000040000B6
:10265800044B5A69586910F0020018BFC2F3800091
:10266800704700BF000400584FF0B042D2F89430D1
:1026780043F40043C2F894304FF47A7300BF013B2F
:102688009BB2002BFAD14FF0B043D3F8942022F438
:102698000042C3F89420D3F894205204FBD40C4B86
:1026A800D3F8902022F40042C3F890204FF47A72B5
:1026B80000BF013A92B2002AFAD1D3F8902042F42E
:1026C8000042C3F890204FF400629A61704700BF3F
:1026D8000004005810B50323052240214FF0904014
:1026E800FFF7F1FEBDE810400323052280214FF0DB
:1026F8009040FFF7E8BE08B5FFF7AAFF003818BFFB
:10270800012008BD08B5FFF7F6FF00B908BD00BFF6
:10271800F9E74FF0904380229A6240229A6170470D
:102728004FF0904340229A6280229A6170470000DD
:10273800024B4FF480225A60704700BF00E100E06E
:1027480010B5134C0323204606220421FFF7BBFED5
:102758001048032302224FF40051FFF7B4FE03236D
:102768001A464FF400414FF09040FFF7ACFE204668
:10277800032305224FF48071FFF7A5FEBDE8104042
:102788000323052201214FF09040FFF79CBE00BFB4
:1027980000040048000800484FF090431869C0F34F
:1027A800C030704708B5FFF7F7FF00B908BD00BF94
:1027B800F9E74FF0904301229A624FF48072C3F810
:1027C80018247047044B4FF480729A624FF090437C
:1027D80001229A61704700BF000400481648416909
:1027E800F02321F0F00193FAA3F3B3FA83F3022262
:1027F80003F00F0302FA03F30B4343610F4BD3F8C3
:10280800842022F40052C3F88420D3F8802022F4D4
:102818000052C3F880205A6822F400525A601A689D
:1028280042F400521A60064BD02283F829234FF451
:1028380000725A60704700BF00000140000800584D
:1028480000E100E0054B4FF40052DA60D3F8802035
:1028580042F40052C3F88020704700BF00080058B7
:10286800064B1A6822F001021A605A6822F40032F4
:102878005A601A6842F001021A607047004400402A
:10288800064B1A6822F001021A605A6842F40032B4
:102898005A601A6842F001021A607047004400400A
:1028A8000023032202214FF09040FFF70CBE4FF0A7
:1028B8009043186980F00200C0F3400070470000A0
:1028C80010B5074C0023204605221021FFF7FBFD19
:1028D80020460023BDE8104005220821FFF7F3BD7C
:1028E8000004004805494B691A04DB4302F48012CE
:1028F80003F0100313438B61704700BF00040048C6
:1029080005494B691A04DB4302F4002203F008036B
:1029180013438B61704700BF000400480C4BD3F889
:10292800FC2022F08072C3F8FC20D3F8FC2042F08F
:102938008072C3F8FC20A3F55D431A6822F00102F7
:102948001A601A6842F001021A6000225A60704741
:1029580000ED00E00649074B074A1B68B3FBF2F39A
:1029680010B54C6843434A68121B9A42FBD310BD0A
:10297800001000E01C00002040420F001FB5022399
:10298800CDE9013101A801236946039308F042F813
:1029980000280CBF0420052005B05DF804FB0146A3
:1029A80008B5012007F0F0FF00280CBF042005201F
:1029B80008BD08B5FFF7E2FF031F5842584108BD9C
:1029C80008B5FFF7ECFF031F5842584108BD000047
:1029D8002DE9F047294B2A4D01280E46144629496E
:1029E800294A0FBF79277827AA461D4606BF884679
:1029F8009A46904607F07CFF39462846FFF7D9FFEC
:102A080028B9002407F086FF2046BDE8F087002E8D
:102A180008BF4FF4FC64073424F0070405F11007DD
:102A2800B1463444AAEB050AA1450BD14FF0113247
:102A38004FF0FF332846FFF7C3FF041E18BF0124D9
:102A4800A400DFE76EB90AEB0703D3E90023B3F16B
:102A5800FF3F08BFB2F1FF3F06D1083709F1080967
:102A6800E2E7D9E90023F2E7B84505D93846FFF788
:102A7800A7FF0028F1D1C4E70324C3E700C0030877
:102A880000C80308FFCF0308FFC7030810B507F005
:102A98002FFF09487821FFF78CFF044638B1074813
:102AA8007921FFF786FF041E18BF0124A40007F050
:102AB80031FF204610BD00BF00C0030800C803084E
:102AC80030B5084D002340F2EF749AB2914201D814
:102AD800042030BDA34203D05A5DC2540133F4E749
:102AE8000320F6E710C0030838B504460D4672B651
:102AF8000A4601460020FFF76BFF62B6042806D19C
:102B080072B601202A462146FFF762FF62B638BD39
:102B180038B5124B1C68D3F80058B4F1113F09D1ED
:102B2800B5F1113F17D0002211460120BDE8384009
:102B3800FFF74EBFB5F1113F03D1002211461046F1
:102B4800F4E7FFF7A3FF042804D12C4001340CBF9D
:102B58000220012038BD0420FCE700BF00C00308A4
:102B6800044B9A689107FCD518739A68D207FCD56C
:102B7800187B70470000015870B50C46451E8E182A
:102B8800B44200D170BD15F8010FFFF7E9FF04F852
:102B9800010BF5E7084611461A46FFF7EDBF00009E
:102BA80070B5064E04464518A54200D170BD307870
:102BB800FFF7D6FF04F8010BF6E700BF140000206A
:102BC80008461146FFF7ECBF38B504464518AC4235
:102BD80000D138BD14F8010BFFF7C2FFF7E708462C
:102BE8001146FFF7F1BF000010B58CB02822002174
:102BF80002A809F08DFC4FF0B0431C4C5A6E42F00D
:102C080001025A665B6E03F001030193019BFFF713
:102C18002BFD082208924FF48272002303924FF48E
:102C28000072CDE90533CDE90933029307920723F2
:102C38004FF4E06202A920460B93049208F00CFEC0
:102C4800636823F010036360636823F0080363601C
:102C5800236843F040032360A3689B07FCD5237BCC
:102C6800034BFF221A700CB010BD00BF00000158C2
:102C780014000020034B18739A68D207FCD5187B00
:102C8800704700BF0030014038B5441E8D18A94276
:102C980000D138BD14F8010FFFF7ECFF01F8010B64
:102CA800F5E7084611461A46FFF7EEBF38B5064D58
:102CB80004460144A14200D138BD2878FFF7DAFF65
:102CC80004F8010BF6E700BF15000020084611467E
:102CD800FFF7ECBF10B5014404468C4200D110BD8B
:102CE80014F8010BFFF7C6FFF7E708461146FFF790
:102CF800F1BF000070B58CB02E4C2822002102A82C
:102D080009F006FC4FF48050FEF747FF0146032305
:102D1800204606224FF48056FFF7D5FB0125A66111
:102D28000624CDE9004503230A2220214FF09040D4
:102D3800FFF744FBCDE9004503230A2231464FF053
:102D48009040FFF73BFB03231A46CDE900454FF4BB
:102D580000614FF09040FFF731FB0822164C0892B3
:102D68004FF48272002303924FF40072CDE90533C9
:102D7800CDE909330293079207234FF4E06202A9D1
:102D880020460B93049208F067FD636823F0100354
:102D98006360636823F008036360236843F04003BB
:102DA8002360A3689B07FCD5237B044BFF221A7082
:102DB8000CB070BD00040048003001401500002030
:102DC8001B4B10B4DC69A00611D51A6891060ED504
:102DD800184819495A6A038809880133C3F30A0352
:102DE80089B299421FBF1549D2B2CA54038010480C
:102DF8001F232206036215D503681B0612D5104B44
:102E0800104A1988138889B29BB299420CD013884A
:102E18000133C3F30903138013880B4A9BB2D35CB5
:102E2800DBB2836210BC704710BCFEF7C2BE00BFA5
:102E380000380140342900203229002032210020A6
:102E4800382D0020362D0020362900200E490F4A43
:102E58000B8812880133C3F3090392B29A4211D046
:102E68000B4AD0540B4A0B8002F5006353E8003F2D
:102E780043F0800302F5006040E800310029F3D1F7
:102E88000120704700207047382D0020362D002083
:102E9800362900200030014038B504464518AC42B8
:102EA80000D138BD14F8010BFFF7D0FFF7E708464B
:102EB8001146FFF7F1BF0000054B064A1B88128830
:102EC8009B1A98B21B0444BF00F5006080B270479B
:102ED8003429002032290020FFF7EEBF0848094AAC
:102EE8000188138889B29BB29942F9D013880133BB
:102EF800C3F30A0313801388034A9BB2D05C70475C
:102F0800342900203229002032210020FFF7E6BFB3
:102F180070B588B00C460646154600212022684642
:102F280009F0F6FA231E18BF01231B03CDE9023569
:102F380069460C23034801960494059308F078FE2B
:102F480008B070BD0038014010B5064C236823F066
:102F580001032360FFF7DCFF236843F001032360CC
:102F680010BD00BF00380140002208461146FFF797
:102F7800EBBF000073B53B4C236823F001032360CB
:102F8800082501264FF48040FEF707FE4021CDE9D1
:102F98000056354803230A22FFF710FA03231A467E
:102FA800CDE9005630488021FFF708FA0022114683
:102FB8004FF46140FFF7ACFF636823F4904363600C
:102FC800A36823F02A03A360284BB02283F82423A4
:102FD80010225A602046FEF7ECFD254A02F50063F0
:102FE80053E8003F23F0400302F5006040E8003159
:102FF8000029F3D1402323621E4B19801E4B1980F0
:1030080002F5006353E8003F23F0200302F5006057
:1030180040E800310029F3D1184B1980184B19806A
:10302800104B5A6822F400625A609A6822F008022B
:103038009A605A6822F480425A609A6822F0220202
:103048009A609A6842F480529A601A6842F00102C3
:103058001A60DA699102FCD5DA695202F9D502B030
:1030680070BD00BF003801400004004800E100E0E6
:1030780000300140362D0020382D00203229002054
:103088003429002008B5FFF775FFBDE80840FEF7B2
:1030980097BFFFF7F7BF0000024B1A68024B1A6090
:1030A800704700BF3C2D002034030020054A064B22
:1030B8001968136899421DBF01330120136000206D
:1030C800704700BF340300203C2D0020034A044B06
:1030D80011681B780B441360704700BF3C2D00201B
:1030E800200000200148FFF758BA00BF0044014003
:1030F800014B586A80B270470044014008B5FFF799
:10310800F1FFBDE80840FFF7C7BF70B504460D469C
:10311800164607F0EDFB083D04EBC606B44204D1A1
:10312800042407F0F7FB204670BD55F8082FD4E9B2
:1031380000016B68994208BF904201D10834EDE75D
:103148002046FFF73DFC0028F8D10446E9E70000D7
:103158001FB503788BB10A4B1B68B3F5FA6F0CD314
:103168000023002203700023CDE90023CDE90223C8
:10317800406802226946FFF7C8FF05B05DF804FB06
:103188003C2D0020000000000123F0B50380444BD3
:10319800444AD3E9005104464348914208BF854256
:1031A80085B04FF0000202D1227005B0F0BD3AA1FF
:1031B800D1E900013D4F6260C3E900013C484FF08E
:1031C800AA33D0E90021B1F1FF3F08BFB2F1FF3FB8
:1031D800D0E9026505D0994208BF9A4201D00A4356
:1031E80009D1B5F1FF3F08BFB6F1FF3F0DD09D42B1
:1031F80008BF9E4209D01030B842E2D172B67A2197
:103208002B48FFF7D6FB62B629486060D0E9003248
:10321800CDE90032B2F1FF3F08BFB3F1FF3FD0E97B
:10322800025109D1B1F1FF3F08BFB5F1FF3F22D1EB
:103238004FF0AA331A4623E04FF0AA36B24208BF2D
:10324800B3420BD1B1F1FF3F08BFB5F1FF3F0FD03B
:10325800B14208BFB5420ED10023EBE753EA02079B
:1032680009D1B14208BFB54205D14FF48071218020
:103278001D46114604E0002323701A461D461946D0
:10328800CDE90032CDE9025102226946FFF73DFF40
:103298008BE700BFAFF3008012345678FEDCBA909B
:1032A80000000020FEDCBA901234567800D80308DB
:1032B80000D003080A490B8803B9FEE772B64FF03D
:1032C800804309885A6A114464325963DA636FF09B
:1032D80002021A616FF008021A6162B6704700BFF5
:1032E8004400002000B5032289B04FF0FF314FF0B1
:1032F8008040FFF749F920220021684609F008F9C3
:1033080064236A4601214FF08040039308F018FBBC
:10331800C8236A464FF480714FF08040039308F049
:103328000FFB054BA02283F81B234FF000621A60A5
:1033380009B05DF804FB00BF00E100E04FF08043F6
:10334800DA6842F00202DA60DA6842F00802DA600B
:103358007047000010B501EB8101084B01EB8101BA
:1033680089001980064B044600221A70FFF7BAFF3D
:103378002046BDE81040FFF7E1BF00BF4400002031
:10338800310300204FF080431A6991070AD56FF086
:1033980002021A615A6B6432DA63084A596B12885E
:1033A8000A445A634FF080431A69120705D56FF033
:1033B80008021A61024B01221A707047440000206B
:1033C80031030020F8B51B4C1B4F90220021201D13
:1033D80009F09EF806260F23A38032462C2339468F
:1033E800A01926806680FEF7EFF84FF001124FF41F
:1033F8008033C4E90D2300252C233246394604F1D5
:103408003E00A587FEF7E0F80C4BE3660C4984F80C
:103418007250012304F17C00A4F87030C4E91D55F2
:1034280009F0D0F87F2384F89130052384F892308E
:10343800F8BD00BF6002002058CC0008010007005A
:103448006DC8000870B5094E05460C46415C30460B
:1034580009F075F8034628B1831B0133DBB2282B2A
:1034680028BF0023F35C2B5570BD00BF70CC00084B
:1034780070B50C461146064609F0A4F844B100257B
:10348800052130460135FFF7DDFFEBB29C42F7D846
:1034980070BD0000F7B5054605F11106214C224A1A
:1034A800014636016846FFF7E3FFB01C6946204431
:1034B80009F088F8264404EB0512002302277772E6
:1034C800A2F81A31142202FB05400421012280F8D7
:1034D80050104FF4807540F20111A0F84A70C26490
:1034E800A0F8522080F85520A0F85650A0F858109F
:1034F80040F2032084F83430E784A562A08584F87C
:103508002E2084F8303084F83330C4F83A30C4F8C8
:103518003E30C4F84230A4F84610A4F8481003B06E
:10352800F0BD00BFA400002018C80008F7B5054684
:10353800AF4CB04A05F11106014637016846FFF75E
:1035480097FFB81C274469462044FDF751FF7B7A52
:10355800A94A052B88BF022304EB061088BF7B729B
:103568001188437A41FA03F3DF070FD40223437229
:1035780061B14807C1F3800308D441FA03F7FF0794
:10358800D8B240F1D18104EB0613587204EB05114F
:103598002B0191F81A01052802D9002081F81A0197
:1035A800E718508897F81A1140FA01F1C90711D4A1
:1035B800012187F81A1168B18707C0F3400109D4BF
:1035C80040FA01FC1CF0010FCFB200F0B281E11803
:1035D80081F81A71E11891F81B01032802D900201B
:1035E80081F81B0104EB0616717A012903D9042915
:1035F80001D000219180E618908896F81B1140FAB6
:1036080001F111F001010ED186F81B1158B110F02B
:10361800010108D140FA01F7FF07CEB240F18E81CF
:10362800234483F81B61142303FB054191F84A00E6
:10363800052802D9022081F84A0003FB054393F8C4
:103648004B10042902D9002183F84B10142303FBE3
:103658000543918E93F84B0041FA00F0C00712D44D
:10366800012083F84B0071B18807C1F340030AD4E5
:1036780041FA03F6F707D8B240F16581142303FB3A
:10368800054383F84B00142303FB054393F84C10C0
:10369800032902D9012183F84C10142000FB0540AE
:1036A800D18E90F84C3041FA03F313F0010310D196
:1036B80080F84C3069B111F001030AD141FA03F6E0
:1036C800F607D8B240F14481142303FB054383F87D
:1036D8004C00142303FB054393F84E10012902D92B
:1036E800002183F84E10142000FB0540118F90F83C
:1036F8004E3041FA03F313F0010310D180F84E3035
:1037080069B111F001030AD141FA03F6F707D8B2FB
:1037180040F12381142303FB054383F84E0014234F
:1037280003FB054393F84F10022902D9002183F8BF
:103738004F10142000FB0540518F90F84F3041FA8C
:1037480003F313F0010310D180F84F3069B111F081
:1037580001030AD141FA03F6F607D8B240F1028113
:10376800142303FB054383F84F00142303FB05418F
:1037780091F84D00022802D9002081F84D0003FB82
:10378800054393F85010052902D9042183F85010F5
:10379800142303FB054191F85200012802D90120A6
:1037A80081F8520003FB054393F85510012902D90B
:1037B800012183F85510142303FB054393F8531094
:1037C800022902D9002183F85310142000FB054078
:1037D800918F90F8533041FA03F313F0010318D195
:1037E80080F85330A9B111F0010312D106E000BFEF
:1037F800A400002018C800086002002041FA03F65F
:10380800F707D8B240F1B380142303FB054383F8CC
:103818005300142303FB054191F856000C2802D9E4
:10382800002081F8560003FB054393F84C1001294A
:1038380006D193F84F10022904BF002183F84F10D6
:10384800142303FB0543012183F8571040F20111AB
:10385800A3F8581094F82630052B02D9022384F8CF
:10386800263094F82730042B02D9002384F8273017
:10387800B2F86C0094F8273040FA03F313F0010F04
:10388800804B0ED1012184F8271050B18607C0F370
:10389800400106D440FA01F7FF07CEB26CD583F891
:1038A800276094F82810022902D9002184F82810EA
:1038B80094F82910022902D9012184F82910B2F8B4
:1038C8006E1094F8292041FA02F212F001020CD18C
:1038D80084F8292049B111F0010206D141FA02F613
:1038E800F607D0B24CD583F8290094F82A200C2A80
:1038F80002D9002284F82A2093F832200C2A02D90F
:10390800002283F8322093F82B20042A02D90022BF
:1039180083F82B2000225C49104611F9014F14F15D
:10392800780F31DA087031E00133102B7FF425AEBF
:103938002CE6013110297FF443AE4BE60131102902
:103948007FF468AE6FE60133102B7FF491AE9AE6F0
:103958000133102B7FF4B2AEBBE60133102B7FF49A
:10396800D3AEDCE60133102B7FF4F4AEFDE6013371
:10397800102B7FF443AF4CE7013110298AD190E72F
:103988000132102AAAD1B0E7782CCBDC0132D2B2AE
:103998000C2AC2D13D490022012011F8014F013201
:1039A800022CD2B288BF0870042AF6D193F83420CA
:1039B800012A02D9002283F83420354AB2F870105F
:1039C80093F8342041FA02F212F001020CD183F884
:1039D800342049B111F0010206D141FA02F4E4079A
:1039E800D0B211D583F8340093F82C20052A02D9D7
:1039F800032283F82C2093F82D20032A08D80AD113
:103A0800002283F8342006E00132102AE5D1EBE7E2
:103A1800022283F82D2093F82E20022A02D90122AF
:103A280083F82E2093F83020022A02D9002283F846
:103A3800302093F833200C2A02D9002283F833204F
:103A4800142101FB0531FF2203EB05154FF6FF702A
:103A580081F8512081F8542083F82F2083F83120F1
:103A68004FF0FF32C5F81C21A5F820011A629A848C
:103A7800A1F85A20A1F85C2083F83500DA861A8765
:103A880003B0F0BDA4000020DD000020E900002004
:103A98006002002030B5052804D8DFE800F01E04D5
:103AA80023191E23FEE720251F2400220F21104B77
:103AB80098700338012894BF002001201A711977E3
:103AC8001A74A3F84850A3F84A409873987630BD02
:103AD80009256F2400220721E9E714253224002252
:103AE8000A21E4E73525132401221921DFE700BF65
:103AF800480000202DE9F74300F11106804F814C62
:103B0800360106F10209B94405464846FDF78CFC22
:103B18000421804601903E440DEB0100FEF786F833
:103B280040F20113A4F85230A4F85430737AE083B9
:103B38002E0107EB0515C4F80880C4F8148095F821
:103B48001A0163704FF0000884F85180FFF7A2FF54
:103B580097F826206C4B13F9223023732376637869
:103B6800052B06D8DFE803F0035356585A5C84F84F
:103B78000D8004236376654B617B1B8884F82810CD
:103B880003F00102980748BF42F00202A2855D07D0
:103B980042BFA28D42F00402A285180742BFA28D3F
:103BA80042F01002A285DA0642BFA28D42F020023E
:103BB800A2859B0642BFA38D43F00803A38500237B
:103BC80084F82A3021B94846FDF74EFC84F82A00CB
:103BD8003E4496F81B2184F829206AB1E18B02EB58
:103BE800021303EB03230B44E383A3684FF0113163
:103BF80001FB0233A360636194F82850E38B63628E
:103C0800052D0FD8DFE805F00F595B184F51012338
:103C18006373AEE70223FBE70423F9E70523F7E71D
:103C28000323F5E7FEE7A378032B03D8DFE803F0C7
:103C3800034B4903FEE71825354E84F8205016E952
:103C48000F0086E80F00042384F838301023A38778
:103C5800022384F83030284640F2E243A4F84C307E
:103C6800FCF740FF4FF07F51FCF790FFFDF77AF922
:103C7800092D4FEA550398BF0523B4F8482084F866
:103C880050304FF47A73B3FBF2F3A4F8403097F84E
:103C98002C30C0B2A4F84E00052B24D8DFE803F07E
:103CA800152C202326290225C6E7A378022B08D045
:103CB800052B06D0012B06D0FEE71925BCE7062503
:103CC800BAE70C25B8E71225B6E74FF41653636434
:103CD8000023A4F8563084F8583003B0BDE8F083C8
:103CE8004FF41643F3E74FF46143F0E74FF4E13341
:103CF800EDE74FF46133EAE74FF49643E7E700BF97
:103D0800A40000204800002058CC000860020020D1
:103D18007800002002484FF4DE72FF2108F0F8BB5B
:103D2800A400002002484FF4DE71FEF7DDBE00BF9C
:103D3800A400002002484FF4DE71FEF7C1BE00BFA8
:103D4800A400002008B5FFF7F5FF034B1878BDE87D
:103D58000840FFF7EBBB00BF4800002038B5FFF76D
:103D6800D9FFFEF7D5FE04280CD0FFF7D3FFFEF7E6
:103D7800CFFE042803D1FFF7DDFF042806D0FFF7A4
:103D8800C9FF03E0FFF7D6FF0428EED126492748EC
:103D9800264C102208F0E0FB38B1254910222046B5
:103DA80008F0DAFB08B1FFF7B5FFA38AB3F5215F86
:103DB80028D008D30025E8B20135FFF76BFB0A2DA0
:103DC800F9D10023E3774FF42153A3820125226917
:103DD8001549164842F642039A424FF010021CBF9A
:103DE8002361012508F0B8FB70B10F490F48102274
:103DF800FDF70FFC0F4910480822FDF70AFCFFF7F2
:103E080091FF03E00025E2E7002DF8D10023E377D6
:103E18000A4C2370FFF7D6FA2078FFF787FB207843
:103E2800BDE83840FFF766BE1FC80008A4000020A0
:103E380030C8000841C80008560200204800002089
:103E480030B5C01A1628A8BF16206FF00805A8427A
:103E58009DF80C40B8BF2846A042C8BF20B2C0B2E7
:103E680008701844107030BD07B5084611461A4648
:103E7800162300930023FFF7E3FF03B05DF804FB6C
:103E880007B5084611461A46162300930023FFF784
:103E9800D7FF03B05DF804FB0129F7B5054600D943
:103EA800FEE70B4E06EB01131C460F016278F15D2D
:103EB80003619B7808F0CCF8E3790193A379009328
:103EC80022796379E178284608F0E9F803B0F0BD73
:103ED80048E20008836810B5044603B9FEE70021EC
:103EE80008F078F84FF47A70FEF734FD2046012187
:103EF80008F087F8A36820461978FFF7CDFF10BDB2
:103F080038B5836804466BB1024652F8183BDD6940
:103F180000F11903A847217E20460222BDE8384057
:103F280008F01FB938BD000070B58160897A86B085
:103F3800044601B1012108F064F8204608F0F3F9BD
:103F4800204608F0CBF9217BFF2903D0FA2220462E
:103F580008F0D0F9A3685B7A013B042B04D8DFE8AA
:103F680003F0043E3E414100FEE7E922E1212046FC
:103F780008F0FEF90121204608F08DF99621204627
:103F880008F0CAF93821204608F0DCF9204608F084
:103F9800E1F9A368204693F90810FFF7B1FFA36879
:103FA8009D7A15B319782046FFF776FF002211464F
:103FB800204608F040F80023009340F203222046F0
:103FC8004FF6FF7108F09AF820464FF6FF7108F097
:103FD800BCF8204606B0BDE8704008F06CB9DB229A
:103FE800D721C4E76F226B21C1E70F4B0F49DE8B46
:103FF8000F4B63614CF250330093204619230B2278
:1040080008F0C6F90123CDE903335B23CDE9015359
:104018001023194620460095042208F0F7F9314686
:10402800204608F017FAC1E748000020A0860100E2
:1040380028E2000873B504460D4616460DF107013F
:104048000DF1060208F0E6F89DF8061033462A46F8
:10405800204607F090FF02B070BD38B504461D46F3
:1040680013460A46002107F05FFF20464FF6FF710E
:1040780008F06BF8A9012046BDE8384008F07EB882
:1040880010B5044608F017F920464FF6FF71BDE851
:10409800104008F05AB8836873B50D46144623B922
:1040A80081220A70237002B070BD9E7A0DF106015C
:1040B800B6B108F099F894F90030002B04DABDF88D
:1040C80006201344ADF80630BDF90630002B0BDB93
:1040D8004FF6FF73ADF80630BDF806302B70E2E7F7
:1040E80008F0C9F92670EFE77F33F5DA4FF68173E8
:1040F800F0E7000038B58168036891F90810DD69B8
:10410800044600F1190300F11802A847A3689A7A37
:1041180042B11A78012A00D9FEE7044B03EB0213D7
:10412800236138BD024B6361FBE700BF48E200082A
:1041380028E20008836810B5044683B103691BB9F7
:1041480043690BB9FFF7D6FFA3689B7A1BB12369B4
:10415800B3F90C0010BD6369B3F91C00FAE71846FF
:10416800F8E7836810B5044643B103691BB943698E
:104178000BB9FFF7BFFF94F9190010BD1846FCE70B
:104188002DE9F0478C46BCF1200F11461D46BDF8BD
:1041980020E09DF824209DF82830044600D9FEE749
:1041A800052D857100D9FEE736482E0100EB05176D
:1041B800805900B9FEE7BE6897F80C80A0602661B8
:1041C8003879E071002684F80C8084F8D950A682EA
:1041D8004FF001094EFA06F7FF0742BFB4F814A0E2
:1041E80009FA06F747EA0A0706F1010648BFA78257
:1041F800062EEFD1A68A06B9FEE7A0EB0800C0B2EA
:10420800604528BF6046052DE07530D0012D35D8B2
:1042180002F1FF35EDB220D0022D19D85D1E032D15
:1042280010D80C2801D90C25E575E57D854200D903
:10423800E0752046FDF774FB002384F8D830A37599
:10424800BDE8F087122884BF1223E3750023ECE74A
:10425800042B88BF00230022EBE7022D04D80C288A
:1042680003D90C23E37500E000220023E1E7531E85
:10427800022BF9D80828F8D90823F3E72046FDF7D8
:10428800E9FAD9E7F8CB000890F8D8305BB190F894
:10429800D930074A180102EB03139B6819781358A1
:1042A80053F821007047837D0E3350F82300704780
:1042B800F8CB0008024690F8D80030B528B3B2F819
:1042C800DC30B2F8DA1001339BB29942A2F8DC3044
:1042D8001BD80023A2F8DC30948A92F8D930062142
:1042E8000133DBB2062B28BF002344FA03F5ED07A0
:1042F80007D5074C1901615801B9FEE782F8D93092
:1043080030BD013911F0FF01EAD10020F8E700BF04
:10431800F8CB0008837DC27D0133DBB29A4298BF97
:104328000023837590F8F63090F8F7200133DBB25C
:104338009A4298BF002380F8F630704713B5194B9E
:104348000288DB8B9A42044627D1837813F0D00F7A
:1043580025D18379812B22D84FF6FF730D22014690
:104368000DF10600ADF80630FDF748FCB4F80D2055
:10437800BDF806309A420ED14C2204F10D01FDF72A
:104388003DFCB4F85900BDF80630C01A18BF01202A
:10439800800002B010BD0320FBE70120F9E70220EE
:1043A800F7E700BF480000200A7ACB7902F007023D
:1043B80043EA022303804B7A0A7A03F03F035B0146
:1043C80043EAD20343808B7A4A7A9B0043EA9213EA
:1043D800CA7A02F0010243EA822383800B7BCA7AFD
:1043E80003F00F03DB0143EA5203C3800B7BC3F3E3
:1043F8000112012A11D813F0300F14BF0123002332
:104408009B0203830B7B7F2B0AD813F0C00F14BFCA
:10441800012300239B024383704740F2FF73F0E7B8
:1044280040F2FF73F7E70A7ACB7902F0070243EA12
:10443800022303804B7A0A7A03F03F035B0143EAC5
:10444800D20343808B7A4A7A9B0043EA9213CA7A52
:1044580002F0010243EA822383800B7BCA7A03F0CD
:104468000F03DB0143EA5203C3800A7CCB7B02F0D3
:10447800070243EA022303814B7C0A7C03F03F03D3
:104488005B0143EAD20343818B7C4A7C9B0043EA6D
:104498009213CA7C02F0010243EA822383810B7DD6
:1044A800CA7C03F00F03DB0143EA5203C3814B7D4F
:1044B800DB0003828B7DDB004382CB7DDB008382C4
:1044C8000B7EDB00C3820B7BC3F30112012A2BD8BE
:1044D80013F0300F14BF012300239B0203830B7BCF
:1044E8007F2B24D813F0C00F14BF012300239B0295
:1044F80043830B7DC3F30112012A1BD813F0300F3D
:1045080014BF012300239B0283830B7D7F2B14D8C8
:1045180013F0C00F14BF012300239B02C3834FF481
:10452800806303844384704740F2FF73D6E740F208
:10453800FF73DDE740F2FF73E6E740F2FF73EDE754
:1045480037B5214BDB8B03804A78837862F3C3034A
:1045580083704A79C37862F30003C3708A79437918
:1045680062F386134371044691F902000D46FCF785
:1045780026FEE37860F34703E370EA78237962F371
:10458800060323712A79DBB202F0010203F07F03EC
:1045980043EAC21323712A796379C2F3450223F0EF
:1045A8003F031343637159224FF6FF7321460DF100
:1045B8000600ADF80630FDF721FBBDF80630A4F87B
:1045C800593003B030BD00BF480000202DE9F34149
:1045D8009DF820601546522E88464FF05B024FF03A
:1045E800000104461F4628BF522607F091FF2D4BB5
:1045F800DB8B23802A78A37862F30203A37069789F
:10460800C90001F00801DBB203F0070341EA081111
:104618001943A1706A79E37862F30003E370AA7919
:10462800637962F38613637195F90200FCF7C7FD9D
:10463800E37860F34703E370EA78237962F30603CB
:1046480023712A79DBB202F0010203F07F0343EA07
:10465800C21323712A796379C2F3450223F03F0319
:1046680013436371A379224666F3470302F8063FB2
:104678003E443B46B34210D14FF6FF7359222146C0
:104688000DF10600ADF80630FDF7B8FABDF80630B2
:10469800A4F8593002B0BDE8F08113F8011B02F804
:1046A800011FE7E74800002007B5009313460A46B4
:1046B8000121FFF78BFF03B05DF804FB30B5374BE2
:1046C800027893F8261061F30302027093F827101A
:1046D80061F30712027093F82810427861F303021D
:1046E800427093F8291061F30712427093F82A1068
:1046F800827861F30302827093F83210827961F351
:104708000302827193F82B10827861F3071282708A
:1047180093F83410C27961F30302C27193F82C1034
:10472800C27861F30302C27093F82D1061F3071287
:10473800C27093F82E10027961F303020271427974
:1047480093F8301061F30302427193F833108279C1
:1047580061F30712827103F1390100F10A0200F1D5
:10476800160411F9015F02F8015FA242F9D193F82A
:104778004610C27D61F30102C27593F8471061F3D8
:104788008302C27593F8481061F30512C27593F855
:10479800493063F38712C27530BD00BFA400002002
:1047A8000278314BC2F3030230B583F82620027831
:1047B800C2F3031283F827204278C2F3030283F876
:1047C80028204278C2F3031283F829208278C2F3A2
:1047D800030283F82A208279C2F3030283F8322085
:1047E8008278C2F3031283F82B20C279C2F3030242
:1047F80083F83420C278C2F3030283F82C20C278ED
:10480800C2F3031283F82D200279C2F3030283F85E
:104818002E204279C2F3030283F830208279C2F352
:10482800031283F8332003F1390100F10A0200F181
:10483800160412F9015F01F8015FA242F9D1C27DA5
:10484800C2F3010283F84620C27DC2F3810283F8D5
:104858004720C27DC2F3011283F84820C27DC2F30B
:10486800811283F8492030BDA400002070B552267B
:1048780098B0324604460D4603A8002107F048FECA
:10488800212342F642008DF80C30FCF7B1FEADF85A
:104898000E004FF42150FCF7ABFE1C49ADF8100098
:1048A80014220DF11200FCF7B4FE1948FFF759FC69
:1048B800184B8DF8260093F851308DF827300AA848
:1048C800FFF7FCFE4FF68073ADF84630124A134BE3
:1048D800CDE91223124B149347F6FF73ADF8543009
:1048E800104BB3F86C208DF85620B3F86E20B3F84F
:1048F80070308DF857208DF85830009603AB2A4653
:1049080002212046FFF762FE18B070BD47C80008B4
:10491800C81E00204800002001000A001900640099
:104928009E00FF7F6002002038B5104D044600F15C
:104938001B01062205F58970FCF7C6FE94F82130A4
:10494800C3F3030385F8193194F82130C3F3031333
:1049580085F81A3194F82230C3F3030385F81B3124
:1049680004F12500BDE83840FFF71ABFA400002075
:104978000A4A126882600A4A00238380837183810D
:104988000384136803615368064A436113688361AB
:104998005368C3614EF66023036070473C2D0020C6
:1049A8005CC8000865C8000838B5114D114C0220D4
:1049B800FFF770F82846FFF763FB2046FFF760FB18
:1049C80028466FF07F01FFF79BFA6FF07F012046C2
:1049D800FFF796FA2846FFF77DFA2046FFF77AFA9E
:1049E8002846FFF74DFB2046FFF74AFB38BD00BFBE
:1049F800C81E0020E41E002008B590F820300246AA
:104A08008BB9FDF754FF10B982F8210008BD92F860
:104A1800213001335BB2312B82F82130F6DD0123DE
:104A280082F82030F2E7FDF742FF18B1322382F80E
:104A38002130EBE792F82130013B5BB2002B82F882
:104A48002130D8BF82F82000E0E700000A4B90F838
:104A580020201B6872B182689B1AB3F57A6F01D95E
:104A680001234371037923B9437913B101230371F6
:104A7800037370478360F5E73C2D00200346007BF5
:104A8800821E012A4FF0000202D893F8201009B9BB
:104A98001A737047104670470A4A38B513880133AD
:104AA8009BB2502B04460D4601D8138038BD002315
:104AB80005491380FDF738FC29462046FDF734FCEC
:104AC800F4E700BF380300206EC800082DE9F84F4E
:104AD800154604460F466B496B4EFDF725FC2946E3
:104AE8002046FDF721FC694B0022012F1A800FD1C7
:104AF8001023B362082746F2A810B761FDF72AFF12
:104B0800B762FDF727FF29462046FFF7C5FFF2E702
:104B1800BB1E08220C2B00F2A880DFE803F031410D
:104B2800521C07A6A6A6626262626200564E4FF049
:104B380008081027C6F8188046F2A810B762FDF7D3
:104B480009FFC6F82880B761FDF704FF294620460B
:104B5800FFF7A2FFEDE74C4E4FF008081027C6F804
:104B6800188046F2A810B761FDF7F4FEC6F8288051
:104B7800B762FDF7EFFE29462046FFF78DFFEDE708
:104B8800B262414E102746F2A810B761FDF7E2FE67
:104B9800B762FDF7DFFE29462046FFF77DFFF2E703
:104BA8001023B361384E082746F2A810B761FDF705
:104BB800D1FEB762FDF7CEFE29462046FFF76CFF0F
:104BC800F2E7B261304E102746F2A810B761FDF740
:104BD800C1FEB762FDF7BEFE29462046FFF75CFF1F
:104BE800F2E7A7F1090BDFF8A0805FFA8BFB00263C
:104BF8004FF0080A5E453CBF1023C8F818304FF044
:104C0800040946F2A810C8F818A0FDF7A3FEC8F8D2
:104C180028A0FDF79FFE09F1FF3929462046FFF736
:104C28003BFF19F0FF09ECD11023C8F828304FF0EA
:104C3800040946F2A810C8F818A0FDF78BFEC8F8BA
:104C480028A0FDF787FE09F1FF3929462046FFF71E
:104C580023FF19F0FF09ECD10136A7F10803F6B2DA
:104C6800DBB2B34238BF0026C4E71023B261B36198
:104C78004CF25030FDF76EFE29462046FFF70CFF38
:104C8800F6E700BF6EC8000800040048380300209B
:104C980010B514461A4618B90348FFF7CBF910BDEA
:104CA80002482146F9E700BFC81E0020E41E002084
:104CB80070B514461D460C48FDF72BFD2B462246C1
:104CC8000E46FFF7CAF97D20FDF744FEFDF771FD9A
:104CD80006482B4622463146FFF7BFF9BDE870402B
:104CE8007D20FDF737BE00BFC81E0020E41E00204F
:104CF8002DE9F041184C05465B270E463A4600213F
:104D0800204607F005FCAB692360EB696360134B31
:104D180013491B789A1E53425341627A63F3000287
:104D280062724222A27228220023E27204F10E006B
:104D3800142223736373FCF76CFC59212046FCF79B
:104D480075FF084BA4F859003A46214630461B7FA8
:104D5800BDE8F041FFF7ACBF541D00202B03002035
:104D680047C800084800002008B530B9054801F1D7
:104D7800A202A031FFF78FF908BD01F1A302024892
:104D8800A131F7E7C81E0020E41E00200A4608B536
:104D980001460148FFF79AFE0C0000200023FF227D
:104DA800037043708370C27003717047C178034603
:104DB80029B9827801710132827001207047007828
:104DC80001281ED0022805D0C8B99A781871013276
:104DD8009A70F2E798785A784240D20704D40130A2
:104DE800002298701A71E8E7FF2902D10020187193
:104DF80070471A790132D2B291421A71EFD300206A
:104E08007047FF29F2D01A790132D2B291421A7151
:104E1800F5D29A7801329A7000221A717047000010
:104E280010B5437802789A421BD0052B8ABF052318
:104E380003700370027888BF43700A4B0A4813F95D
:104E480022100A4C83682173217613B11972FFF777
:104E580057F80748836823B194F918101972FFF7B7
:104E68004FF810BD58CC0008C81E0020480000208C
:104E7800E41E002010B50AB9437010BD541E0B2C57
:104E8800FBD80332D2B231F8122040F27E618A4256
:104E980003D95AB222EAE2721AE0B2F5C17F02D20D
:104EA8009A1E52B2F6E740F2A9518A4204D95AB280
:104EB800052A1CDCDA1EF4E740F256218A4218D98A
:104EC80040F2D4418A4208D95AB2042AF2DD0222B9
:104ED8009A42C8BF5AB24270CFE7B2F54B7F04D2AC
:104EE8005AB2032AE6DD0122F2E75A1ED9E7032265
:104EF800EEE70022ECE700000E48C3691A0617D552
:104F080003681B0614D50C4B0C4A1988138889B200
:104F18009BB299420AD013880133DBB213801388FD
:104F2800074A9BB2D35CDBB283627047FCF741BE91
:104F3800704700BF00440040302100202E2100208F
:104F48002E2000200E490F4A0B8812880133DBB24D
:104F580092B29A4212D00C4AD0540B804FF04022A1
:104F680002F5806353E8003F43F0800302F5806058
:104F780040E800310029F3D1012070470020704734
:104F8800302100202E2100202E20002038B5044694
:104F98004518AC4200D138BD14F8010BFFF7D2FF19
:104FA800F7E708461146FFF7F1BF000070B588B073
:104FB8000C460646154600212022684607F0A8FA46
:104FC800231E18BF01231B03CDE9023569460C23B4
:104FD800034801960494059306F02AFE08B070BDB4
:104FE8000044004010B5064C236823F001032360F9
:104FF800FFF7DCFF236843F00103236010BD00BF07
:105008000044004008B541B14FF4005204484FF441
:105018008061FFF7E7FFFDF723FC012008BD00BF13
:10502800A086010008B531B1002211460348FFF7F8
:10503800D9FFFDF715FC012008BD00BF9A5B0600EB
:1050480008B541B14FF4005204484FF48061FFF7AE
:10505800C9FFFDF715FC012008BD00BFA0860100AF
:1050680013B52F4C236823F0010323604FF400305D
:10507800FCF787FD08230120CDE900300A2203232D
:1050880004214FF09040FDF799F900221146254878
:10509800FFF78CFF636823F490436360A36823F0F1
:1050A8002A03A360204BC02283F8252320225A60BC
:1050B8002046FCF77EFD4FF0402101F5806353E860
:1050C800003F23F0400301F5806040E80032002AE9
:1050D800F3D140232362154B1A80154B1A8063685D
:1050E80023F400636360A36823F00803A360636884
:1050F80023F480436360A36823F02203A360A368BA
:1051080043F48053A360236843F001032360044BF6
:10511800DA699102FCD5DA695202F9D502B010BDFC
:1051280000440040A086010000E100E02E2100209C
:105138003021002030B5214C85B00E2200210546D3
:10514800684607F0E5F9B4F8A030ADF8003020461D
:10515800FBF7E6FF8DF802002046FBF7D8FFB4F80E
:10516800A4308DF803001648ADF80430FEF7F9FFB7
:1051780094F8A6308DF8073094F8A9308DF80830E7
:10518800B4F8AA30ADF80A300E4B8DF806009A78BC
:105198008DF80C2093F8522093F853305AB1002B15
:1051A8000CBF01230323694628468DF80D3004F00F
:1051B800EEFD05B030BD0133DBB2F4E70C1E002074
:1051C800C81E0020480000200148FEF773B800BF41
:1051D8000A1E0020F8B5154D0E4607465B232946E2
:1051E800304614462A46FFF753FDD7E904132868CA
:1051F8006A689A4208BF884209D0002430460C49A0
:10520800FFF7B2FD002C0CBF01200320F8BD592187
:105218002846FCF70BFDB5F859308342EDD114B19F
:10522800FFF7D2FFEAE70124E8E700BF1D1F0020CF
:105238000C1E002013B5012104460844FCF7F6FCB7
:10524800A178ADF806000DF10600FCF7CBFCE1787B
:10525800FCF7C8FC2179FCF7C5FC6179FCF7C2FCB6
:10526800A179FCF7BFFC04F108010322FCF7C6FC96
:10527800627804F10C01FCF7C1FC94F82311FCF7E7
:10528800B1FCBDF80630A4F80C3102B010BD000026
:105298000038024B18BF012018707047F802002030
:1052A8002DE9F041002A4AD1042B00F2A1809EB2D8
:1052B800002B42D04D4C4FF0800EFF250F8894F8FC
:1052C8001EC0C35D23EA0C03C355A37F01325B08EC
:1052D8001FFA82FCA3773BB90B8801330B8084F853
:1052E8001EE00B88C554A37FB1F8008010F8087041
:1052F80027EA030300F80830A37F5B08A3773BB9CC
:105308000B8801330B8084F81EE00B88C554A37FFB
:10531800B1F8008010F8087027EA030300F8083095
:10532800A37F5B08A37733B90B8801330B8084F81C
:105338001EE00B88C5546645C0D8BDE8F081FF2A39
:10534800FBD1032B00F249819FB2002BF5D0274CEB
:1053580000258026B1F800C094F81EE010F80C3043
:1053680023EA0E0300F80C30A37F01355B081FFA0F
:1053780085FCA37733B90B8801330B80A6770B889C
:10538800C254A37FB1F8008010F808E02EEA0303A6
:1053980000F80830A37F5B08A37733B90B88013383
:1053A8000B80A6770B88C254A37F5B08A37733B919
:1053B8000B8801330B80A6770B88C254A37FB1F802
:1053C800008010F808E02EEA030300F80830A37FF5
:1053D8005B08A3772BB90B8801330B80A6770B8862
:1053E800C2546745B6D8BDE8F08100BF2806002042
:1053F8000D889A4C425DA67F22EA06024255A27F9A
:10540800520803F5C063A2773AB90A8801320A80C4
:105418008022A2770A88FF2585540D88A67F425DE1
:1054280022EA06024255A27F5208A2773AB90A88B0
:1054380001320A808022A2770A88FF258554A27F3C
:105448005208A2773AB90A8801320A808022A277E4
:105458000A88FF258554A27F5208A2773AB90A889C
:1054680001320A808022A2770A88FF2585540D8898
:10547800A67F425D22EA06024255A27F5208A27721
:105488003AB90A8801320A808022A2770A88FF2561
:1054980085541E0605D40D88A67F425D22EA0602C1
:1054A8004255A27F5208A2773AB90A8801320A8087
:1054B8008022A2770A88FF2585545D0605D40D88C9
:1054C800A67F425D22EA06024255A27F5208A277D1
:1054D8003AB90A8801320A808022A2770A88FF2511
:1054E80085549A0605D40D88A67F425D22EA0602F5
:1054F8004255A27F5208A2773AB90A8801320A8037
:105508008022A2770A88FF258554DF0605D40D88F6
:10551800A67F425D22EA06024255A27F5208A27780
:105528003AB90A8801320A808022A2770A88FF25C0
:1055380085541E0705D40D88A67F425D22EA06021F
:105548004255A27F5208A2773AB90A8801320A80E6
:105558008022A2770A88FF2585545D0705D40D8827
:10556800A67F425D22EA06024255A27F5208A27730
:105578003AB90A8801320A808022A2770A88FF2570
:1055880085549A0705D40D88A67F425D22EA060253
:105598004255A27F5208A2773AB90A8801320A8096
:1055A8008022A2770A88FF258554DB0705D40A885C
:1055B800A57F835C23EA05038354A37F5B08A37755
:1055C800002B7FF4BAAE0B88802201330B80A277C0
:1055D8000B88FF22C254BDE8F0810E881F4C855D00
:1055E800A77F25EA07058555A57F6D0803F5E063C4
:1055F800A57735B90D8801350D808025A5770D88EB
:1056080042550D88A67F425D22EA06024255A27FD6
:105618005208A2773AB90A8801320A808022A27712
:105628000A88FF258554A27F5208A2773AB90A88CA
:1056380001320A808022A2770A88FF258554A27F3A
:105648005208A277002A7FF418AF0A8801320A802C
:105658008022A2770A88FF2585540EE728060020B5
:105668002DE9F0479C4C802500270F80A577FF2562
:1056780005709846002B00F02C8103F1FF3912FACF
:1056880089F9561EBA463B460BE0554540F0C080A6
:105698000137BFB20A88424580F0B3804E4500F01A
:1056A800078116F8015F002BEFD16B1EDBB2FD2BD3
:1056B80000F2AA803F2B40F2E18005F14103DBB202
:1056C8003F2B00F2AC80A37F01355B08EDB2A377D6
:1056D800002B00F0E4805B08A37743B90B88013303
:1056E8000B808023A3770B88FF22C254A37FAA06CE
:1056F80008D4B1F800C010F80C2022EA030300F81F
:105708000C30A37F5B08A37743B90B8801330B8068
:105718008023A3770B88FF22C254A37FEA0608D40C
:10572800B1F800C010F80C2022EA030300F80C308E
:10573800A37F5B08A37743B90B8801330B808023D1
:10574800A3770B88FF22C254A37F2A0708D4B1F895
:1057580000C010F80C2022EA030300F80C30A37FE5
:105768005B08A37743B90B8801330B808023A377A9
:105778000B88FF22C254A37F6A0708D4B1F800C07F
:1057880010F80C2022EA030300F80C30A37F5B0812
:10579800A37743B90B8801330B808023A3770B8849
:1057A800FF22C254A37FAA0708D4B1F800C010F89A
:1057B8000C2022EA030300F80C30A37F5B08A377D0
:1057C80043B90B8801330B808023A3770B88FF2212
:1057D800C254A37FEA0705D40D88425D22EA030379
:1057E8004355A37F5B08A377BBB90A8801320A80B7
:1057F8008022A2770A88FF2585540A884245FFF44B
:105808004DAF0020BDE8F0870127AA463B4641E797
:10581800FBB25246FFF744FD47E700233AE70A8800
:1058280094F81EC0835C23EA0C038354A37F3F359E
:105838005B08EDB2A37743B90B8801330B80802353
:10584800A3770B88FF22C254A37F5B08A37743B9D1
:105858000B8801330B808023A3770B88FF22C25467
:10586800A37F6A063FF537AFB1F800C010F80C20E7
:1058780022EA030300F80C30A37F2CE7A37F7F35CF
:105888005B08EDB2A377002BEED10B8801330B80B8
:105898008023A3770B88FF22C254A37FE4E70B88F9
:1058A80001330B808023A3770B88FF22C254E3E7E0
:1058B8005BB9A37F802B1EBF013292B20A8090454C
:1058C80094BF00200120BDE8F087FBB25246FFF7E5
:1058D800E7FC0A88EDE700BF280600202DE9F04F15
:1058E80047F26F730022827003800B78A3F1FE03E6
:1058F800B3FA83F35B0983708A780D4612F00101CD
:105908001CBF43F080038370D5F8202122F07F422A
:1059180022F0FF0285B0044612B143F008038370F9
:10592800AA68C2F31702FF2A1ED9B2F5803F18D31E
:1059380063F07F03A37041F002014FF0020B0923CB
:105948004FF00A0C0822E1700B20CDF804C01E4667
:1059580017464FF0070E4FF006094FF0050A0421CD
:1059680017E043F00203A370180600F1D68008235D
:105978004FF0090C07220A204FF0000BCDF804C0A5
:105988001E4617464FF0060E4FF005094FF0040A61
:10599800032195F8018004F8018004EB01082979B6
:1059A80004F80A10697904F80910A97904F80E10A6
:1059B800A178090709D595F82111A15495F8221164
:1059C800A1550346674662460646A968A154A278CF
:1059D800900707D5BA1C1F46AB68C3F30F23A3551E
:1059E80096B23346BBF1000F05D05A1C1F46AB7A5E
:1059F800A35596B23346A278D10606D55A1C1F463F
:105A080095F82331A35596B23346454A127803F1E7
:105A1800010914FA89FA05F10C0B42B16B785A4660
:105A28000DF10E015046FFF71BFE00285AD16A7887
:105A3800504659461FFA82FA06F0CCFD2278394BB7
:105A48006178D243D2B2072F9A5C82EA0102995C4C
:105A5800A27882EA0102995CE27882EA0102995C02
:105A6800227982EA0102995C627982EA0102995CF0
:105A7800A27982EA0102995CE27982EA0102995CE0
:105A88001BD0227A5140082F595C16D0627A5140B7
:105A9800092F595C11D0A27A51400A2F595C0CD0B9
:105AA800E27A51400B2F595C07D0227B51400C2FD2
:105AB800595C1EBF627B5140595CA1551AFA89F3A3
:105AC8009BB2B5F80C21E2545A1CB5F80C1192B2ED
:105AD800090AA154AA78981CD20780B20BD405B041
:105AE800BDE8F08FA378BDF80EA043F04003A37083
:105AF80088F800A0A2E7D5F81071D5F81811D5F8E4
:105B08001461275022180F335660916095F81C11C4
:105B1800117398B205B0BDE8F08F4FF0000B0EE797
:105B2800F80200209CCC00082DE9F04F944D0C465B
:105B380083B0014607462846164606F04BFD914AB3
:105B4800002380202380138482F82200002E00F096
:105B5800CD8095F800C04FF0400B4FEADC1C82F86E
:105B680022B09E464FF0FF0892F8229015F803A045
:105B78004FEA4C0C1AEA090F4FEA590118BF4CF0CA
:105B8800010C82F82210002900F0B380BCF1020F4A
:105B980000F04484BCF1030F00F0DF83BCF1010F77
:105BA80040F0BA809E4240F2A18015F8039019EAAD
:105BB800010F14BF4FF0010C4FF0000C5FEA510ABF
:105BC80040F0B68301339BB29E42138482F82200D0
:105BD80040F28C80E95600294FEA4C0C01DA4CF06F
:105BE800010C82F822B0402100919E427ED9009992
:105BF80015F803904FEA4C0C19EA010F00995FFA67
:105C08008CFC18BF4CF0010C5FEA510A40F0268466
:105C180001339BB29E42138482F8220066D94FEA70
:105C28004C0115F903C015F80390BCF1000FC9B277
:105C380001DA41F001014FEA410C19F0400F5FFA17
:105C48008CFC18BF202100F09F854CF0010C002926
:105C580040F09B8501339BB29E42138482F8220058
:105C680044D915F903904FEA4C0CB9F1000F5FFACB
:105C78008CF115F803C001DA41F0010149001CF06C
:105C8800400FC9B218BF4FF0200A00F0B98541F0A3
:105C9800010182F822A0BAF1000F03D10133138465
:105CA80082F822007D2921D84131238803F1010C93
:105CB800A4F800C0F954138C9E4217D992F8221008
:105CC80015F803C011EA0C0F4FEA510114BF4FF049
:105CD800010C4FF0000C82F8221021B901339BB25D
:105CE800138482F822009E423FF63EAF03B0BDE81F
:105CF800F08F01339BB2BCF1020F138482F82200AB
:105D080000F0AD81BCF1030F00F03482BCF1010F4B
:105D18004FF080013FF446AF9E42E7D915F803C023
:105D280011EA0C0F1ED05FEA51092DD101339BB245
:105D38009E42138482F82200D8D9E9560029C0F27D
:105D4800E8804FF080094FEA590182F8221019B90A
:105D58000133138482F822002388591C218007F814
:105D68000380A8E7490882F8221019B9013313847F
:105D780082F822002388591C218007F803E09AE75B
:105D8800FC0400202806002019EA0C0FDBD0890843
:105D980040F0C08001339BB29E42138482F82200F7
:105DA800A4D9E9560029C0F2668280215FEA510C25
:105DB80040F0418201339BB29E42138482F8220054
:105DC80094D9E95C4FEAD11C49064FEA4C0C40F1E2
:105DD800BD8420214CF0010C82F8221029B901332E
:105DE8009BB2138482F8220080219E427FF67EAF08
:105DF80015F803904FEA4C0C11EA090F5FFA8CFC76
:105E080018BF4CF0010C490840F06E8301339BB277
:105E18009E42138482F822007FF668AFE9564FEA63
:105E28004C0C00295FFA8CFC80F2318480215FEAF7
:105E380051094CF0010C40F0658301339BB29E423E
:105E4800138482F822007FF651AF4FEA4C0115F90E
:105E580003C0BCF1000FC9B280F225844FF080095D
:105E68005FEA590941F0010140F0598301339BB2BF
:105E78009E42138482F822007FF638AF15F903C0DA
:105E88004900BCF1000FC9B280F226844FF08009A6
:105E98005FEA590941F0010140F04D8301339BB29B
:105EA8009E42138482F822007FF620AF15F903C0C2
:105EB8004900BCF1000FC9B2C0F211844FF040098B
:105EC80015F803C0490019EA0C0FC9B200F0528353
:105ED8004FEA590941F0010182F82290B9F1000F07
:105EE80040F0048401339BB2138482F822001FFA25
:105EF80081FC00293FF4E0AE00232188013301F141
:105F08000109A4F8009007F801E099B26145F4D3BB
:105F1800D1E6402115F803C011EA0C0F3FF446AF53
:105F2800490840F0A98101339BB29E42138482F84C
:105F380022007FF6DBAE15F803904FEAD91C19F062
:105F4800400F4FEA4C0C00F0F58320214CF0010C77
:105F5800002940F0F08301339BB29E42138482F8FB
:105F680022007FF6C3AE4FEA4C0C5FFA8CF115F9AC
:105F780003C015F80390BCF1000F01DA41F00101EC
:105F8800490019F0400FC9B218BF4FF0200C00F0BB
:105F98002C8441F00101BCF1000F40F0288401334A
:105FA8009BB29E42138482F822007FF69FAE15F9B9
:105FB80003C04900BCF1000FC9B201DA41F0010188
:105FC80082F822B04FF0400A9E427FF68FAE15F855
:105FD80003C049001AEA0C0FC9B218BF41F0010109
:105FE8005FEA5A0C40F0D58201339BB29E4213847B
:105FF80082F822007FF67AAE15F903C04900BCF199
:10600800000FC9B2C0F275834FF0400C15F8039029
:1060180049001CEA090FC9B200F0DA824FEA5C0CA9
:1060280041F0010182F822C0BCF1000F40F0688302
:1060380001339BB2138482F822001FFA81FC0029E5
:106048003FF43AAE00232188013301F10109A4F895
:10605800009007F8018099B28C45F4D82BE69E424F
:106068007FF644AEE95C4FF04009C909B2F820C098
:106078004B0015F80C1019EA010F4FEA590A01D024
:1060880043F00103BAF1000F40F0B1820CF1010CAA
:106098001FFA8CFC6645A2F820C082F822007FF621
:1060A80025AE15F90C905900B9F1000FC9B280F26C
:1060B800DC82402341F00101002B40F0A5820CF165
:1060C800010C1FFA8CFC6645A2F820C082F8220059
:1060D8007FF60CAE15F90C304FEA4109002B5FFA38
:1060E80089F980F2CB82402149F00109002940F06A
:1060F8009A820CF1010C1FFA8CFC6645A2F820C0AC
:1061080082F822007FF6F2AD15F90C104FEA490328
:106118000029DBB280F2BE824FF0400943F0010350
:10612800B9F1000F40F08E820CF1010C1FFA8CFCC3
:106138006645A2F820C082F822007FF6D7AD15F98F
:106148000C105B000029DBB280F2C382402143F0CF
:10615800010382F8221029B90CF1010CA2F820C021
:1061680082F822002188013301F1010CA4F800C053
:106178007B54A0E59E427FF6B9AD15F803C04FF0F9
:1061880040094FEADC111CEA090F4FEA41014FEAC6
:10619800590A01D041F00101BAF1000F40F03683ED
:1061A80001339BB29E42138482F822007FF69EAD93
:1061B80015F9039015F803C04900B9F1000FC9B2E9
:1061C80001DA41F0010149001CF0400FC9B218BFC3
:1061D8004FF0200A00F0F18241F00101BAF1000FFE
:1061E80040F0ED8201339BB29E42138482F8220074
:1061F8007FF67CAD15F9039015F803C04900B9F195
:10620800000FC9B201DA41F0010149001CF0400F4A
:10621800C9B218BF4FF0200A00F0DA8241F001013C
:1062280082F822A0BAF1000F03D10133138482F857
:106238002200413939E515F8039019EA0C0F14BF0B
:106248004FF0010C4FF0000C5FEA910A40F03782E2
:1062580001339BB29E42138482F822007FF646AD3A
:10626800E95600294FEA4C0C01DA4CF0010C82F88F
:1062780022B04021B9E5402115F8039019EA010F31
:1062880014BF4FF0010C4FF0000C5FEA510A40F0C8
:106298000D8201339BB29E42138482F822007FF65E
:1062A80025ADE95615F8039000294FEA4C0C01DAA0
:1062B8004CF0010C4FEA4C0C19F0400F5FFA8CFCC3
:1062C80018BF4FF0200A00F048824CF0010CBAF1D8
:1062D800000F40F0448201339BB29E42138482F83F
:1062E80022007FF603AD15F903904FEA4C01B9F18E
:1062F800000F15F803C0C9B201DA41F001014900E5
:106308001CF0400FC9B218BF4FF0200A00F0658298
:1063180041F0010182F822A0BAF1000F7FF454AED7
:1063280001339BB2138482F822004FF0800A4BE6B7
:10633800890819EA0A0F00914FEA4C0C01D04CF079
:10634800010C82F8221000297FF44FAC01339BB274
:10635800138482F82200802146E415F803C01CEA61
:10636800010F14BF012100215FEA99097FF40BAFE7
:1063780001339BB29E42138482F822007FF6B6ACAA
:1063880015F9039015F803C0B9F1000F4FEA410160
:1063980001DA41F001011CF0400F4FEA410118BF3A
:1063A8004FF0200900F0BB8141F00101B9F1000F65
:1063B80040F0B78101339BB29E42138482F82200D9
:1063C8007FF694AC15F9039015F803C04900B9F1AC
:1063D800000FC9B201DA41F0010149001CF0400F79
:1063E800C9B218BF4FF0200900F0C38141F0010184
:1063F800B9F1000F40F0BF8101339BB29E42138474
:1064080082F822007FF672ACEB564900002BC9B225
:1064180001DA41F0010182F822B00AE792F82290ED
:1064280019EA0A0F14BF012100215FEA59097FF414
:106438001DAE01331FFA83FC6645A2F820C082F81E
:1064480022007FF653AC15F90C90B9F1000F4FEA12
:10645800410380F202814FF0400A11E64FEA4C0CEA
:10646800890819EA0A0F5FFA8CFC019101D04CF0F7
:10647800010C002940F0D38101339BB29E42138462
:1064880082F822007FF632AC4FEA4C0115F903C0BE
:1064980015F80390BCF1000FC9B201DA41F001010F
:1064A800490019F0400F5FFA81FA18BF4FF0200C2D
:1064B80000F076814AF0010ABCF1000F40F07281C9
:1064C80001339BB29E42138482F822007FF60EAC01
:1064D800EB564FEA4A01002BC9B201DA41F001013B
:1064E80082F822B0FFF7DEBB15F803904FEA4C0C98
:1064F80011EA090F5FFA8CFC7FF499AC5FEA510945
:106508003FF49BAC4FEA4C0115F803C019EA0C0F95
:10651800C9B27FF4A5AC5FEA59093FF4A7AC15F8F6
:1065280003C0490019EA0C0FC9B27FF4B1AC5FEAA5
:1065380059093FF4B3AC15F803C0490019EA0C0F28
:10654800C9B201D041F001015FEA59097FF4B8AC42
:1065580001339BB29E42138482F822007FF6C6ABB9
:1065680015F903C04900BCF1000FC9B2C0F2BA80E6
:106578004FF080094FEA590982F82290B9F1000FCB
:106588003FF4B0AC1FFA81FC00297FF4B5ACFFF7EB
:1065980095BB15F8039049001CEA090FC9B201D050
:1065A80041F001015FEA5C0C7FF430AD01339BB22E
:1065B8009E42138482F822007FF698AB15F903C037
:1065C8004900BCF1000FC9B2C0F296804FF0800CB0
:1065D8004FEA5C0C82F822C0BCF1000F3FF428ADF2
:1065E8001FFA81FC00297FF42DADFFF767BB15F872
:1065F8000C9059001AEA090FC9B24FEA5A037FF4FE
:1066080059AD002B3FF45BAD15F80CA04FEA4109DA
:1066180013EA0A0F5FFA89F94FEA53017FF464AD70
:1066280000293FF466AD15F80CA04FEA490311EABA
:106638000A0FDBB24FEA51097FF470ADB9F1000FD0
:106648003FF472AD15F80CA05B0019EA0A0FDBB233
:106658004FEA59013FF47DAD79E515F80C305B063A
:106668004FEA81014FD5202324E59B005FFA83F987
:1066780015F80C30590648D5202135E58900CBB2EC
:1066880015F80C10490642D54FF0200946E54FF0A1
:10669800400937E715F80C104FEA89034906DBB2C1
:1066A80038D5202153E54FF0400938E719EA0A0F99
:1066B8004FEA91014FEA4C0C3FF44AAC46E419EA20
:1066C8000A0F4FEAD1014FEA4C0C3FF485ABFFF7B4
:1066D80081BB82F822B045E54FF040092BE74FF027
:1066E80080092FE741F0010182F822B01FFA81FCEE
:1066F80002E44FF0800C53E741F0010182F822B028
:106708001FFA81FC9EE420237EE720218BE74FF0CF
:10671800200997E74FF0200182F8221022E54FF078
:106728002009490019EA0C0FC9B24FEA590A3FF487
:1067380055AD51E520214FEA4C0C19EA010F5FFADB
:106748008CFC4FEA510A3FF4C2ADBEE54FF0200180
:1067580082F822102021FFF748BB4FF0200A4FEAA9
:106768004C0119EA0A0FC9B24FEA5A0C3FF413ACAC
:106778000FE44FF02009490019EA0C0FC9B24FEA9B
:10678800590A3FF44DAD49E520214FEA4C0C11EA76
:10679800090F5FFA8CFA4FEA510C3FF48DAE89E687
:1067A8004FF0200C4FEA4A0119EA0C0FC9B24FEA20
:1067B8005C0A3FF46EAAFFF76ABA4FF0200A490054
:1067C8001AEA0C0FC9B24FEA5A093FF411AE0DE6A6
:1067D8004FF0200382F822302BE54FF0200C82F88E
:1067E80022C04FF0200AFFF7EFBB4FF0200C490002
:1067F80019EA0C0FC9B24FEA5C0A3FF48BAD87E582
:106808004FF0200382F82230FFF74CBA49001AEA09
:106818000C0F4FEA9909C9B23FF4C8ADC4E58A46DE
:1068280000994FEA4C0C19EA0A0F4FEAD1015FFAB6
:106838008CFC3FF40CAAFFF708BA00BF2DE9F04F13
:106848005788B7F58F7F8BB0144606460BD90022C0
:10685800227000226F2B628000F065810023337064
:106868000BB0BDE8F08F12780E2A0D4624D80E2AF8
:1068780000F2118101A151F822F000BF5B68000805
:10688800AB6A00089F6A00089F6A0008AB6A0008A4
:10689800AB6A0008AB6A0008AB6A0008AB6A00087C
:1068A800AB6A0008F96A00089F6A00089F6A000836
:1068B8009F6A00081D6B0008692A40F2EA806A2A6C
:1068C80040F0E9809C4FFA8A02F1FF3C1FFA8CFCE9
:1068D800002A00F078820CF1030CDFF860E2BC4477
:1068E800FF22B91C11F8010B424061451EF8022035
:1068F800F8D1934200F0D08100222270C4F802201F
:10690800E280FA8A022AA9D939796F2900F02E8300
:10691800032AA3D079796F2900F03883042A9DD0FF
:10692800B9796F2900F03583052A97D0F9796F294D
:1069380000F03E83062A91D0397A6F2900F045820B
:10694800072A8BD0797A6F2900F03583082A85D0F9
:10695800B97A6F2900F03283092A3FF47FAFF97AB8
:106968006F2900F02E830A2A3FF478AF397B6F290C
:1069780000F02A830B2A3FF471AF797B6F2900F06E
:1069880026830C2A3FF46AAFB97B6F2900F0228373
:106998000D2A3FF463AFF97B6F2900F01E830E2A9E
:1069A8003FF45CAF397C6F2900F01D830F2A3FF458
:1069B80055AF797C6F2900F01383102A3FF44EAF4E
:1069C800B97C6F2900F01283112A3FF447AFF97C94
:1069D8006F2900F00E83122A3FF440AF397D6F29EA
:1069E80008BF4FF012087FF439AF02F101091FFA0E
:1069F80089F93A44A7F816905FFA89F993705049D3
:106A08004A4602A805F0E6FD6F234FF0010CBB7063
:106A18004FF0000E6423A7F800E0A7F816C0237013
:106A280008EB0C0399451FFA89F27FF617AF901E01
:106A380002A9A0EB08005A1E0B440A4413FA80F07E
:106A48004FF06A084FF007094FF0660A05E0002B7F
:106A580040F0BE8190423FF401AFFB8A12F8011F5B
:106A680007EB030B01338BF80210FB822378092B09
:106A7800EDD9A3F1640BBBF1050FEBD8653B042BF3
:106A880000F2BA82DFE813F01F01170112010E01AC
:106A98001B01632A05D800232370C4F80230E38061
:106AA800DDE6254FFA8AB91801328B70FA8222780E
:106AB800092A00F2A480002A3FF4D0AE013A082A3D
:106AC8003FF6CCAE01A151F822F000BF956D000849
:106AD8006568000865680008F76C0008F76C00082E
:106AE8007F6D00084B6D0008B96D0008696D0008DE
:106AF8007A1C6280104EEB55A088727F61888318DB
:106B08009942FFF6ADAE33785F0600F1E4810E23BB
:106B18002370A5E67A1C6280EB55E288638893426D
:106B280010D201239BE604490A800122CA8264220A
:106B38008B702270002392E6280600209CCC000867
:106B48002A060020002363802370022303704280FA
:106B58002B78FD2B00F08780EB7803722B7943723A
:106B68006B7943606A780832728000224FF4BC70F7
:106B7800DFF8CCC27281F6210446013499424FEA0B
:106B880054042ED849D38B4240F08A802B78FD2BB1
:106B98007FD04FF0060B2846DFF8A48210F801AF2B
:106BA8000BEB0A0909F1FF3189B2FBF73FF804EB57
:106BB800440708EB8707ADF808003979019102A866
:106BC800FBF710F805EB090215F80930527801991E
:106BD80003EB0223BDF808209BB29A421FD005237D
:106BE8003DE6601E1418824204F1010780F06C81B2
:106BF80027F0010101EB57015CF82110BDE7A2F174
:106C0800640105293FF62AAE653A042A00F2FD819F
:106C1800DFE802F0817D797593002246E2E7BB79CF
:106C2800DA0706D5FA79924582BF521912F80B2075
:106C3800B2729B070BD56300234408EB83036A7881
:106C48001B7A9A4282BF5B1913F80B30F3724FEA32
:106C58004409A14408EB8908317398F80530737327
:106C68000BB0BDE8F08F6B790372AB7943726B7A26
:106C7800297AEA791B0403EB0123134443606A78F9
:106C880002F10C014180A978C9077FF56EAF19326E
:106C98006AE74FF00A0B7EE70A2201232270DEE53D
:106CA8000323DCE5F97684F80090D3E64FF0680317
:106CB800B9762370CEE6797084F800C0CAE63977D1
:106CC80084F80080C6E6397001F00103618887F80E
:106CD80001E0033B01F1010BA4F802B06B5497F9F2
:106CE8000030002BACBF634653462370B2E662887F
:106CF800511C6180AB54237801332370AEE5072221
:106D0800FB76227016E76822BB76227012E7012212
:106D18007B7022700EE762883B70002103F001034C
:106D2800033B7970511C6180AB5497F90030002BFC
:106D3800C0F232810123237090E56A223B772270EA
:106D4800F8E66288511C6180AB543B787A7813432B
:106D580013F0020340F0D7806288511C6180AB5465
:106D68006288511C6180AB543B78D8064CBF6923BC
:106D78006A23237072E56288511C6180AB543B78AA
:106D88001D074CBF67230723237067E562883A8392
:106D9800511C6180AB543A787B7712F0010200F005
:106DA800D08006220833A280E3800423237055E5AF
:106DB8006288511C6180AB547B7813F00203CFD0FA
:106DC800092323704AE5FF2293E54FF006080CE6F5
:106DD800013B082B3FF63EAE0FF2040B5BF823F0A5
:106DE800216E00085D6A00085D6A00080D6E0008E3
:106DF8000D6E00089B6E0008696E0008B56E0008ED
:106E08004D6E0008638803F1010BA4F802B0E95441
:106E18002378013323701DE663883B8303F1010B5C
:106E2800A4F802B0E9543B78797713F001036DD0E8
:106E380008310623E180A380042323700AE600BFFB
:106E48009CCD0008638803F1010BA4F802B0E95453
:106E58003B78DB067FF534AF4FF069032370F9E523
:106E6800638803F1010BA4F802B0E9543B78797800
:106E78000B4313F0020343D1618801F1010BA4F81D
:106E880002B06B54618801F1010BA4F802B06B5495
:106E9800DEE7638803F1010BA4F802B0E9543B78FC
:106EA80019077FF500AF67232370D3E5638803F1E3
:106EB800010BA4F802B0E9547B7813F00203E1D087
:106EC8004FF009032370C5E5574902EB4200144609
:106ED80051F8201057E602A92844FEF725FE737FD3
:106EE800BDF808106288CB1A9BB21A446280727F80
:106EF8001A447277E2881344E380338BE95406E638
:106F080008232370A6E508232370A7E40C31E18049
:106F180079784FF00A0B11F00101A4F804B028D0D9
:106F2800618801F1010BA4F802B005F801C061887D
:106F380001F1010BA4F802B06B54E3880D33E38030
:106F48007AE779780C33E38011F001014FF00A03F6
:106F5800A38024D06388012158186080E95463888D
:106F680059186180EA54E3880D331DE74FF0020891
:106F78003BE5638803F1010BA4F802B0E954638888
:106F880003F1010BA4F802B0E95455E74FF00308E8
:106F98002BE54FF0040828E5662323705EE4638838
:106FA8005A1C6280E95463885A1C6280E954FCE6E2
:106FB8004FF0050819E54FF0070816E54FF00808E7
:106FC80013E54FF0090810E54FF00A080DE54FF0FA
:106FD8000B080AE54FF00C0807E54FF00D0804E52B
:106FE8004FF00F0801E54FF00E08FEE44FF01008CF
:106FF800FBE44FF01108F8E477290ED084F800E09C
:10700800C4F802E0A4F806E024E5772B09D00023B1
:107018002370C4F80230E38020E44FF06503237046
:1070280018E56523237019E49CCD00082DE9F84381
:107038001F46184B164693F8302004463AB393F887
:107048002B301FB11BB31F1F18BF0127A1F1020866
:1070580004F5E36901F11E0538F8020FFAF724F97F
:1070680029F8020FB8F80000FAF72BF9A845A9F893
:107078002000F1D1084B84F85A771B68C4F85C37B4
:1070880086F00106012384F8606784F81937BDE8A3
:10709800F88300BFA40000203C2D002010B500F2AA
:1070A8007C7400F5B0712046FAF7EBFD01462046E6
:1070B800BDE81040FBF7F0BEB0F8E834B0F8EA24B9
:1070C8009B1A98B21B0444BF00F5007080B20038C8
:1070D80018BF01207047D0F8F826B0F8E81401323C
:1070E800C0F8F826D0F800270132C0F80027B0F819
:1070F800EA24914203461FBF8118013291F8EE0439
:10710800B3F8EC141ABF0A40A3F8EA240020704729
:107118000F4B93F82D305A1E012A02D80D48FFF75D
:10712800DABF032B10D10C4AB2F81E36B2F81C167F
:1071380099420BD0D118013391F82206B2F82016E3
:107148000B40A2F81E367047FBF7C8BE00207047F8
:10715800A400002060060020080F0020064A002333
:107168001380064AA0F8EA341380054AA0F8E834E8
:107178001380044A138070473229002034290020E4
:10718800362D0020382D002008B50848FFF7E6FF07
:10719800074A0023C2F81C36064A1380064A1380A1
:1071A800064A1380064A138008BD00BF6006002007
:1071B800080F00203229002034290020362D002015
:1071C800382D0020B0F8EA24B0F8E8349B1A10B53E
:1071D8009CB21B0448BF04F50074014648BFA4B222
:1071E800FBF76AFE0319D1F8F006184480B210BD07
:1071F800F8B5D0F8F43690F81877CB1AB3F57A7F4B
:1072080004460E4626D2632B01D800207DE0012FCC
:107218000AD0022F19D0002FF7D1FFF7D3FFB0F50E
:10722800806FF2D9012305E0FFF7CCFFB0F5806F3E
:1072380003D9022384F818370CE02046FFF7C2FF71
:10724800B0F5C07FE1D20023F4E7FFF7BBFFB0F54C
:10725800806FE7D33448C4F8F466F9F786FF334DF6
:10726800334A2B681168C3F1000C411A614501DBF0
:1072780099424BDD10600A232B601368B3F5FA7F3F
:10728800BCBF4FF4FA7313601268D4F8F836522171
:107298004A4328496425B1F8481092FBF1F26B4340
:1072A800B3FBF2F35F2B35D8552B35D83B2B03D9DD
:1072B8004B2B34BF5B25322594F81837022B2DD081
:1072C800012B2DD013B9002F18BF33254FF47A7333
:1072D800D4F80027314604F20470FAF7D4FB94F886
:1072E8001837FBB9642D0BD1D4F8F436A3F29A23DE
:1072F800C4F8F436D4F8F83603225B00B3FBF2F393
:10730800C4F8F83684F8FC560120F8BD002BB4DD2B
:10731800013BB1E70025CFE71E25CDE70025D5E7DE
:107328003225D3E70023EBE70C1E002008000020DD
:10733800FC0200204800002070B5D0F8F43690F820
:107348001827CB1AB3F57A7F04460E4614D2032ABF
:1073580008D8DFE802F002092730FFF733FFB0F55D
:10736800487F26D8002029E0FFF72CFFB0F5AF6F43
:1073780011D9022384F81837304B94F81857B3F80A
:107388004800C4F8F466D4F8F836032D4ED8DFE880
:1073980005F03716494B2046FFF714FFA328E1D81C
:1073A8000323E7E7632BDDD9FFF70CFFB0F5AF6FD9
:1073B800E2D20123DEE7002084F8180770BD2125FA
:1073C8004FF47A73D4F80027314604F20470FAF7C0
:1073D8005AFB94F818377BBB642D0BD1D4F8F436DC
:1073E800A3F54873C4F8F436D4F8F83605229B00A0
:1073F800B3FBF2F3C4F8F83684F8FC560120DDE755
:1074080064210F4AB2FBF0F24B43B3FBF2F35F2B5C
:10741800D6D8552B0CD83B2B0CD94B2B34BF5B251E
:107428003225CDE70025CBE75D25C9E76425C7E709
:107438001E25C5E70D46C3E70023DBE7480000200B
:1074480050400100F8B5234F04463846F9F756FE78
:10745800F9F7CBFE064697F9A600F9F7C6FE0546EA
:107468003846F9F754FE94F8FC3684F87231FF2355
:1074780084F87431332384F86531442384F8663101
:10748800D4F8683184F870616D2262F31703C4F888
:107498006831C0F10A000023C4F86C3184F88132E5
:1074A80000B24FF43943A4F8823280F3070009236D
:1074B80084F8730184F8715104F5B07084F884324B
:1074C80004F5AA71FAF79CFE2046BDE8F840FFF7DC
:1074D800E5BD00BF0C1E00202DE9F04F044685B025
:1074E800B4F82E270092B4F830270192B4F8322766
:1074F800B0F828670292B4F838270378B0F822E782
:10750800B0F824C7B0F81CA7B0F81E97B0F82087C9
:10751800B0F82677B0F82A570392B0F82C07B4F8D9
:107528001A27A4F87A610026B4F83617B4F834B7E5
:10753800A4F86C21A4F874E1A4F876C184F87C312D
:10754800A4F86EA1A4F87091A4F87281A4F87871D7
:1075580084F87D61A4F87E51009AA4F88221019AEA
:10756800A4F88421029AA4F88621039AA4F88C210D
:10757800FF2284F86521442284F86621D4F8682122
:10758800A4F88A1184F8813246214FF4F84361F354
:107598001702A4F882322623A4F88001A4F888B13F
:1075A80004F5B07084F88E6184F88F6184F8906176
:1075B80084F89161C4F8682184F8843204F5AA71CA
:1075C800FAF71EFE204605B0BDE8F04FFFF766BD8E
:1075D800F0B591B0044600F23A736D4600F25A765F
:1075E800186859682A4603C20833B3421546F7D1CA
:1075F80020220DEB0200002104F08AFF94F8602796
:1076080094F85A370AB943F00203A4F870310023FA
:107618002678D4F85C2784F87331102384F8743101
:10762800C4F86C2184F872616B4604F2751510AFCA
:107638001A4603CABA4228606960134605F108056C
:10764800F6D1332384F86531442384F86631D4F8BD
:10765800683184F881624FF4D27262F31703C4F878
:1076680068314FF4A053A4F88232492304F5B0706E
:1076780084F8843204F5AA71FAF7C2FD204611B0E5
:10768800BDE8F040FFF70ABD764B2DE9F04F1A68C8
:10769800D0F86437D31A122BA5B0044640F2DF8025
:1076A800DFF8C4B1C0F864279BF800106F4ADFF810
:1076B800C0A192F85330881E4142414192F85200CD
:1076C800002800F0B580002B00F0BE809AF9A000D9
:1076D800F9F7A3FD9BF800109AF9A2908A1E51426F
:1076E800074651419AF9A100F9F797FD9AF9A38045
:1076F80006469AF8A4305F48012B9AF8A5300CBFCB
:1077080003250125012B9AF8AA300CBF45F008057E
:1077180045F00405012B9AF8AB3008BF45F0100579
:10772800012B0CBF45F0200545F04005FCF7ACFDEA
:10773800F9F7D4F95049F9F729FA04F0ABFE4F49A3
:10774800F9F724FA02904A48F9F7EAFC0190484808
:10775800F9F7F4FC9BF8001003908B1E022908BF70
:107768009AF8A9B09AF9A60018BF4FF0000B594231
:107778005941F9F752FD80228246002104A804F0FD
:10778800C7FE019B8DF81430039B8DF815307F23BD
:107798008DF81A308DF81E30029BCDF81F30FF226D
:1077A8000023ADF810508DF81D20257884F86D3130
:1077B80084F86F316FF02F02172384F86C2184F856
:1077C800703104A984F86E51802204F271108DF88A
:1077D80016708DF817908DF818B08DF819A08DF8DF
:1077E8001B608DF81C8004F0F5FE332384F86531A6
:1077F800442384F86631D4F8683184F8815240F221
:10780800811262F31703C4F868314FF41343A4F8E4
:107818008232852304F5B07084F8843204F5AA71A5
:10782800FAF7EEFC204625B0BDE8F04FFFF736BC6E
:1078380053B19AF9A100F9F7F0FC4FF07F099AF9D2
:10784800A3800646FF2754E79AF9A000F9F7E5FC5C
:107858004FF07F089AF9A2900746FF2649E725B01E
:10786800BDE8F08F3C2D00202B03002048000020AD
:107878000C1E00203C03002000007A3A00007A44E5
:107888002DE9F0434D4B0446A9B04D481D68FCF75F
:1078980068FCD4F8683740F6C312EB1A934204D850
:1078A80094F96C37834200F08580464EC4F86857D7
:1078B800B17884F86C07052998BF434B8DF81100FF
:1078C8009CBF33F81190414B8DF80F1098BF33F8D7
:1078D80011504FF006084FF07F0388BF00254FF086
:1078E80000078DF810304246B6F84A30ADF804303B
:1078F8000DF1120088BFA946ADF80630ADF80C703E
:107908008DF80E80F9F7BCFE7178424606A8F9F7A3
:1079180093FE2B48ADF80A50ADF80890FCF70AFC26
:1079280040428DF81E002648FCF704FC40428DF8C2
:107938001F00642239460FA801AE04F0E9FD0FCEFE
:1079480008AD0FC596E807006FF02E0385E807001D
:1079580084F86C31257884F86D711C2384F87031B3
:10796800802208A984F86E5184F86F7104F27110AE
:1079780004F030FE332384F86531442384F86631FB
:10798800D4F8683184F8815240F2811262F3170307
:10799800C4F868314FF41343A4F88232852304F500
:1079A800B07084F8843204F5AA71FAF729FC2046ED
:1079B800FFF774FB29B0BDE8F08300BF3C2D002021
:1079C800C81E002048000020D8CB0008E4CB0008DF
:1079D80010B5B0F870370446A3F1F60C90F87407A8
:1079E800A4F86C31DCF1000343EB0C035B0084F872
:1079F8006E316FF06E0384F870316FF02A0384F8EB
:107A08007131122384F87231002384F873313323DF
:107A180084F86531442384F86631D4F8683184F8F1
:107A28006F014D2060F31703C4F868318F2394F871
:107A3800721794F8732784F883320A2384F8741130
:107A480084F8811204F5B07084F8752184F88222D4
:107A580084F8843204F5AA71FAF7D2FB2046BDE80F
:107A68001040FFF71BBB10B54FF07E53C0F86C31C8
:107A78000023C0F87031C0F87431C0F87831C0F80C
:107A88007C31C0F88031C0F8843180F88C3108210D
:107A9800332380F8881180F865310221442380F867
:107AA800891180F866310121D0F8683180F88B118E
:107AB8004C2161F31703C0F8683149F601030278D5
:107AC800A0F882322123044680F88A2180F8812296
:107AD80080F8843200F5AA7100F5B070FAF790FBCF
:107AE8002046BDE81040FFF7D9BA0000F0B54E783F
:107AF800202E0D468BB0044601F10C013AD83246CF
:107B080001A804F067FD01ABC6F121020021981914
:107B180004F0FEFC9DF82230332B45D19DF823302C
:107B2800442B41D1BDF82030F62B02D0B3F5FA7FB3
:107B38003AD1B4F87027A4F870379A421CBF0022D3
:107B480084F87427012284F86D276A7984F87227EB
:107B5800AA7984F87327B3F5FA7F27D114490798CF
:107B6800F9F7A8F910B39DF82430012B11D184F846
:107B7800743719E00B4601AA05F12C0718685968F3
:107B8800164603C60833BB423246F7D11B7833701A
:107B9800C0E7022B0AD194F874273AB184F87437F5
:107BA800044B1B68C4F878370BB0F0BD0023DEE740
:107BB80088AC96493C2D00204FF47F430380002376
:107BC800C0E90133C0E9033343610376704700001D
:107BD80038B50023C0E90733C0E955334362C0F81C
:107BE8005C310446FAF79CF8254B9878022845D072
:107BF800431F58425841FDF74BFB40F2FF13A4F8CE
:107C0800EC34204B1B68002503F57A73C4F8F4366E
:107C180004F20470C4E9A255C4F89052A4F8EA54D6
:107C2800A4F8E854C4F8F05684F8FC5684F81857B9
:107C3800C4F8F856C4F80057F9F71FFF84F8195725
:107C4800294604F21A70402204F062FC7D2384F86D
:107C58005A57C4F85C5784F86057C4F86457C4F896
:107C68006857A4F86C37A4F8725784F87457C4F8A6
:107C780078572046BDE83840FFF79EBF0120BAE795
:107C8800480000203C2D002030B40E4A92F82E40C7
:107C9800012C14D10C4A0178126881B1016940F6AF
:107CA800C415511AA94202D930BCFFF785BF4168F3
:107CB80029B94169511AFA2984BF4261047630BC56
:107CC800704700BFA40000203C2D00204378032B00
:107CD80006D1C068B0F5834F34BF0020012070473B
:107CE800002070477FB50B46324991F82D1000F1FE
:107CF80028060229044600F11C02314668461BD1B9
:107D0800FEF79CFD9DF80030022B50D104F5B075AC
:107D1800324669462846FAF711F8D4F8683123F054
:107D28007F436E2B2FD1244B9A78052A3DD8DFE864
:107D380002F0303438063038FAF756F9E2E75A6C70
:107D4800B2F5613F94BF002201222046FFF7BEFF33
:107D5800C8B9C2B194F86E31012B14D894F87231B5
:107D6800042B10D11549102204F27B1004F0F4FB07
:107D780048B9782384F8883184F8823184F87C31D2
:107D88002846FDF757FA204604B0BDE87040FFF7D3
:107D980085B95A6CB2F5E13FD4E75A6CB2F5614F38
:107DA800D0E75A6CB2F5164FCCE70122CDE704B004
:107DB80070BD00BFA40000204800002070C8000863
:107DC800F0B54E78082E85B005460C4601F10C0733
:107DD80017D83246394601A804F0FCFB01ABC6F1BE
:107DE80009020021981904F093FB9DF80930032B30
:107DF80005D162792A70064A12682A616B7005B04B
:107E0800F0BDC86879683A7A01AB03C31A70ECE729
:107E18003C2D002030B5037895B004461BB34A7951
:107E28009A4220D14D784D2D01F10C011DD82A46DA
:107E3800684604F0CFFBC5F14E0200210DEB0500AA
:107E480004F066FB049B6360190EC3F3072242F239
:107E5800107000FB0122C3F30743642101FB0323D5
:107E6800E360059BA36015B030BD4E22684604F060
:107E7800B1FBE7E78A68C2F317024C2A16D0942AA6
:107E88000AD0AAB90B4A92F82E20012A10D18B7970
:107E9800012B0DD1FFF794BF064A92F82E20012A34
:107EA80006D18B79012B03D1FFF7B4BFFFF71EBEB4
:107EB800704700BFA4000020B0F8EA34B0F8E82406
:107EC800F0B5D21A93B2120444BF03F500739BB203
:107ED800DD2B85B0044606D800F5257600F5227519
:107EE800F9F770FE08B905B0F0BDFAF7F7FFD4F856
:107EF800F02601320346C4F8F02631462A46684681
:107F0800FAF772F89DF80030022BE9D104F5707584
:107F1800324669462846F9F711FF184B93F82D3079
:107F280004F27C76022B294630460FD1FDF7D6FCA9
:107F380000239AB290420CD8002329462046C4F860
:107F4800F03605B0BDE8F040FFF794BFF9F799FEA9
:107F5800EEE7B4F8E814B4F8EC744A1C3A40B4F804
:107F6800EA7497421EBF0919F75C81F8EE7403F1B1
:107F7800010318BFA4F8E824DBE700BFA400002031
:107F88002DE9F041494BDFF828811E6898F8003048
:107F9800484F022B1EBF0023A0F8EA34A0F8E834AB
:107FA80097F82D30013B012B04467CD8FFF784FF5E
:107FB80097F82E50002D5AD098F80030022B4AD14D
:107FC800012D3DD0022D41D000252046FFF75CFE53
:107FD80094F8193743B1002384F8193797F83030EB
:107FE800012B4ED0022B4FD015B12046FFF72AFAAD
:107FF80094F86D372BB1002384F86D372046FFF7CE
:10800800E7FC94F87437022B11D1D4F87837F61AB4
:10801800B6F57A7F0BD9B4F87037F62B3DD0B3F5A7
:10802800FA7F3CD00023A4F8703784F87437237E95
:10803800CBB3002323762046BDE8F041FFF713BDFC
:1080480031462046FFF7D4F80546BEE731462046BC
:10805800FFF772F9F8E7D4F8F436F31AB3F57A7F34
:1080680008D2002504F20470F9F707FDADE7C4F85B
:10807800F466F7E73223C4F8F46684F8FC36012581
:10808800F0E7FFF729FAAFE7FFF7A2FA2046FFF774
:10809800FBFA2046FFF7F4FBA6E7FAF783FA064B4C
:1080A80001225A71BEE7BDE8F08100BF3C2D0020D7
:1080B8002B030020A40000200003002070B54C888A
:1080C800B4F5427F03464FF000000AD80D780B2D17
:1080D80077D8DFE805F0060F1C2C2F32383B5457B1
:1080E8005B6DA2F124046242488062410A7083F801
:1080F80009033EE04D2A01D0582A06D11A700222FF
:108108000A70002083F8090370BD0022F8E702F026
:10811800FD003C2801D0212AF7D15A701A784D2A3F
:108128000CBF082203220A7000229A70E9E79A70AD
:108138000422DBE79A800522D8E7988800EB022220
:108148009A800622DCE7DA800722CFE7D88800EB9E
:10815800022292B2002ADA800CBF0B220A220A708D
:1081680000224A80012283F80923DB88B3F5407F87
:1081780001D80020C8E7002008704880C4E7DA80EA
:108188000922B3E79A800A220A70EBE7B4F5407F28
:108198003CBFE41822724A88013292B24A80D888D9
:1081A80090429CBF0B220A70012283F80923E0E762
:1081B80083F8082302220870488083F809230120E5
:1081C800A2E708704880D4E7CB88B3F5407F70B544
:1081D80031D8242303700B7843704B7883700B7865
:1081E8004D2B14D1CB88C3708B88037105230022D3
:1081F800CD88D4189542A6B210FA84F415D891F80F
:1082080008232270CA880132981880B270BD8B7812
:10821800C3708B8803718B881B0A4371CB88837169
:10822800CB881B0AC3710823E1E78C180132247A32
:10823800845592B2DCE70020E8E700002DE9F74F0B
:1082480016464A88B2F5427F04460D462ED80B786A
:108258000A2B0FD9A3F16402032A03D9002028703E
:1082680068802DE0653B8F4F022B33D8DFE803F0A1
:1082780063A4A70000210A2BF0D801A050F823F02E
:10828800B5820008CF820008658200086582000870
:1082980013830008218300082D8300083383000816
:1082A8006582000865820008A1830008A6F12407FA
:1082B8007E424FF000007E4168802E7084F80903EA
:1082C80003B0BDE8F08F6F2E0CBF642300232B7022
:1082D8000020F3E716F0040F14BF4D2358233E7017
:1082E80023703A78D1070ED412F0020F14BF21235D
:1082F8003E236370C2F3C003D20648BF43F00203B3
:10830800A3700423E3E73C23F3E7A68005232B703F
:1083180084F809130020D3E7A38803EB0623A3807E
:108328000623D4E7E6800723F1E7E38803EB062377
:10833800E3806523CBE70DF106007E70F9F79CFC1E
:108348003978F9F791FCA7882179F9F78DFC390A72
:10835800F9F78AFCE788A179F9F786FC390AF9F771
:1083680083FC9DF80630B34206D000232B706B8047
:10837800032384F80933CDE7002F0CBF66230A23B3
:108388002B70012384F8093300236B80E288B2F54F
:10839800407FBFD92B70BDE7B2F5407F3CBF1219B3
:1083A80016726B8801339BB26B80E2889A4201D8BF
:1083B80066232B700123DCE77E806723F9E7B7F893
:1083C800028097F8009008EB06284FF6FF730DF12E
:1083D80006001FFA88F84946ADF80630A7F802806B
:1083E800F9F700FC2679B4F804A03146F9F7FAFB4E
:1083F8004FEA1A21F9F7F6FB94F806B0B4F806A08C
:108408005946F9F7EFFB4FEA1A21F9F7EBFB7978B0
:1084180004F10807F9F7E6FB52463946F9F7EEFB8F
:10842800BDF8063043453AD119F0040015D086EA64
:108438000B01E21D002398B2824584F8081307D87F
:108448000223012000222A706A8084F8093337E762
:1084580012F8010F01334140EDE7A178F8F788FFE2
:10846800217984F80803F8F783FFA18884F80803C2
:10847800090AF8F77DFFA17984F80803F8F778FF6F
:10848800E18884F80803090AF8F772FFE28884F89B
:1084980008033946F8F772FF84F80803D0E7032386
:1084A8000020CFE7D81C0020CB88B3F5407F2DE90A
:1084B800F04104460D464AD84B783C2B40D0A3F1F6
:1084C8002100434243415B002A784D2AAA7808BF1D
:1084D80043F00403D10748BF43F0080392074FF065
:1084E8002402227048BF43F010036F226270A37009
:1084F800AB88E370AB881B0A2371EB886371EB8848
:10850800A71C1B0AA3713846F9F7FEFC0822E07184
:10851800E988A2F108039BB2561C8B42B6B204EB61
:1085280002080FD3063189B23846F9F77FFB88F87D
:108538000000000AA055E8880A3080B2BDE8F08142
:108548000123C1E72B441B7AA3543246E0E70020FD
:10855800F4E730B4BDF80C40B4F5407F03D8039479
:1085680030BCF9F7E9BC002030BC704710B50446B0
:108578002420207058206070237100201B0AA170ED
:10858800E2706371A071E0710522E11CF8F7F6FE54
:108598002072092010BD00002DE9F04F0025DFF8FA
:1085A800E4A00D80D71891468FB080460C462B4624
:1085B8002A464FF0FF0BB94502D10FB0BDE8F08F46
:1085C80019F8010B3B28114609D001323831D2B2D3
:1085D8006944202A01F8300C08BF0022EBE7383242
:1085E8006A444FF0000102F8301C0026F2B25AF833
:1085F8003610019302A80092F7F7BAFDDDE90023CF
:10860800A0B9FF2B1FBF2388591C218008F803B08D
:1086180023880AEBC606591C218008F80320337901
:10862800142B01D8189AD554FF231BE00136372E96
:10863800DCD1FE2B06D023885A1C22806FF0010261
:1086480008F80320002602A8F7F79CFD721CF6B272
:10865800B04223880AD85A1C22804FF03B0208F8FF
:108668000320FE230135EDB20022A4E7591C218026
:1086780006F138010DEB010616F8301C08F8031056
:108688001646E0E76CE2000840F2FF3270B40023BF
:10869800A0F820267D2280F8542A0360C0F80E3303
:1086A800A0F81E36A0F81C36A0F8423AA0F8443AC2
:1086B80080F8463AC0F8483AC0F84C3AC0F8503A00
:1086C800C0F8583A00F66724024600F66D250A26D7
:1086D80014F8011F09B1B6FBF1F1AC4282F8701A27
:1086E80082F8713AC2F8743A02F10802F0D170BC0B
:1086F8001522FF2100F52A6003F00ABFF8B5134AD6
:10870800044692F83000F8B192F82B2003B1DAB1A0
:108718008E1E04F5226701F11E0536F8020FF8F7E0
:10872800C3FDAE4227F8020FF7D1012384F8423A7D
:1087380094F8453A83F0010384F8433A94F8463AAA
:1087480083F0010384F8443AF8BD00BFA400002078
:1087580070B5061D04460A4601463046FFF76EFD11
:1087680000B304F6B52531462846FFF72DFD01462E
:108778002846FAF791FB63793C2B13D121890A48E3
:1087880004F65A2304F66622A4EB8404A4F5F754ED
:108798001C3C33F8025F8D4204BF056844F823503F
:1087A8009342F6D170BD00BF3C2D002070B5124B2E
:1087B80093F82D300C4611465A1E012A0AD80F4E3E
:1087C8006518AC4200D170BD14F8011B3046FFF7A4
:1087D80089FAF6E7032B09D1094E6518AC42F2D0A5
:1087E80014F8011B3046FFF7B3FFF7E72046BDE852
:1087F8007040FAF751BB00BFA400002060060020BB
:10880800080F0020B0F81C36B0F81E269B1A98B244
:108818001B0444BF00F5806080B2003818BF0120F7
:108828007047000008B50C4B93F82D305A1E012AEA
:1088380004D8BDE808400948FEF73EBC032B04D124
:10884800BDE808400648FFF7DDBFF9F7BBF9003877
:1088580018BF012008BD00BFA4000020600600204A
:10886800080F002010B500F6B5240B4620463C2121
:108878000222FFF77BFE01462046BDE81040FAF7CA
:108888000BBB00000F4B1A68D0F8483AD31A122BCA
:1088980013B515D9C0F8482A00F6B524202300F6E8
:1088A800222001930090C82303223C212046F9F797
:1088B800D3FA0146204602B0BDE81040FAF7ECBAF8
:1088C80002B010BD3C2D00207FB5224B1A68D0F8AD
:1088D8004C3AD31AC72B044639D91F4DC0F84C2A35
:1088E8004FF480732846ADF80830F8F707FC0646C1
:1088F8001A48FBF71FFC01463046F8F71FFD8DF8B4
:108908000A002846F8F7FAFBF8F712FD95F8A9309F
:108918008DF80B0028468DF80C30F8F701FC8DF81F
:108928000D002846F8F7F3FB072304F6B524019356
:1089380002AB8DF80E0000933C2141F20D03032297
:108948002046F9F789FA01462046FAF7A5FA04B055
:1089580070BD00BF3C2D00200C1E0020C81E00204A
:1089680030B51F4B044687B01E481D68FBF7F9FB5E
:10897800D4F8503A40F6C312EB1A934203D894F94C
:10898800543A83422AD0C4F8505A002384F8540A2F
:108998008DF80830F8F702FD134DADF80900697835
:1089A800ADF80B0004220DF10D00F8F745FEA9788B
:1089B80006220DF11100F8F763FE0F2304F6B52423
:1089C800019302AB00933C2141F20E03032220469F
:1089D800F9F742FA01462046FAF75EFA07B030BDC9
:1089E8003C2D0020C81E002048000020F8B5324D5C
:1089F800324E0024F9F792FF0227FAF77FFBF9F7C6
:108A08005FFFF9F74DFFFAF73DFB2D492D4801F0BF
:108A180083F9FCF725FBC5E90444AC602F73FAF72A
:108A2800E3F8294B1C70F9F755FE284BD02283F840
:108A380032233046F9F78EFF21462846244D03F0AD
:108A4800C9FA4FF47A70F9F785FF2F73C5E9044422
:108A5800AC60FAF74FF91F4B1C70F9F771FEF9F784
:108A6800BDFE1D4B4FF4005230461C4EDA60042701
:108A7800F9F770FFB76241F28830F9F76BFFB76119
:108A88004CF25030F9F766FF2846F9F78BFE21467D
:108A9800284603F09FFA4FF47A70F9F75BFFFBF76B
:108AA8005DF90F48FAF770FB0E4B0F48B3F8481002
:108AB800BDE8F840FAF74EBCC81E0020E093040059
:108AC800CA000020DC1C00201400002000E100E0A7
:108AD800E41E00201500002000080058000400488B
:108AE800241D0020480000200A1E002073B51648E7
:108AF800164C4FF6FF7103F0BDFB208023889B07BF
:108B080012D5134E35798DB10F4808236A460021D6
:108B180003F031FAD6E90402DDE900139A4208BFEE
:108B2800884201D00023238002B070BD02236A4628
:108B38000548294603F01FFA064BDA8BBDF80030CA
:108B48009A4218BF2580EFE7C81E00205006002073
:108B58000003002048000020184B4FF4005273B562
:108B6800DA601748174C4FF6FF7103F083FB20803B
:108B780023889B0712D5144E35798DB110480823E8
:108B88006A46002103F0F7F9D6E90402DDE900138B
:108B98009A4208BF884201D00023238002B070BDEA
:108BA80002236A460648294603F0E5F9074BDA8BA3
:108BB800BDF800309A4218BF2580EFE7000800583A
:108BC800E41E00204E06002000030020480000207C
:108BD800034A00231370034A1370034A1370704743
:108BE800590600201C1F002030030020024A0023E1
:108BF8001370024A13707047590600201C1F00208A
:108C080008B5437E203B042B0FD8DFE803F0050EA0
:108C1800030B0F00FBF788FE064A01231370064A70
:108C2800137002E0054B01221A7008BDFBF78AF8A1
:108C3800F2E700BF590600201C1F00203003002067
:108C4800034B1B78012B01D1FBF710BE704700BF07
:108C5800590600202DE9F043074699B03D48FCF736
:108C6800A5F80646002860D03B4B1C78002C5CD148
:108C78003A4B1B78022B54D1DFF8E4900DF10C0825
:108C880025464846ECB2FFF7CDFD40B14846FEF711
:108C98003FFA0135522D08F8010BF2D12C46314824
:108CA8002146F8F7E6FE3048F8F7DDFEDFF8A48045
:108CB8002E4D98F802308DF800304FF0010995F8E4
:108CC800A4308DF80530284685F8A5708DF8067013
:108CD8008DF80190F8F712FA8DF802002846F8F797
:108CE8001FFA8DF803002846F8F728FA204F8DF868
:108CF80004000EB3184B1B78CBB91E48234603AAB1
:108D08006946FBF7D1FC194801233B70F8F724FAB0
:108D18001648F8F72AFA012388F8033019B0BDE895
:108D2800F0830F48FEF730FAC0E70024BEE7114889
:108D38006946FFF785FFE6E73B7803B9FEE70D488C
:108D48006946FBF7FDFB284687F80090F8F709FA13
:108D58002846DEE7001F00201C1F00202B030020F0
:108D680018000020701E0020481E00200C1E002045
:108D7800F9020020AF1D002070B5CB78284DC3F351
:108D8800000385F8AA304B79C3F3801385F8AB301C
:108D98000646C87840080C46F8F721FA85F8A60078
:108DA80023792048C3F3000385F8A7302379C3F358
:108DB800450385F8A8306379227903F03F035B0007
:108DC80043EAD21385F8A93021461EB9BDE87040A0
:108DD800FBF7EABAFBF727FBA37803F0F003202B95
:108DE80004D12046BDE87040FFF70ABFFFF7FEFE3A
:108DF8000D4B1B78022B12D1A2790C4804F11901F2
:108E08005208FFF7D3FCA17905F178004908F8F773
:108E180030FE05F15000BDE87040F8F724BE70BD83
:108E28000C1E00202C1D00202B0300201800002001
:108E380070B5054658B9194B19491C781948037972
:108E48004BB1012C28D0BDE87040F8F7E5BF164BB0
:108E580016491C78F2E7012C154B164E13D98A785F
:108E6800C2F3C0025A7002221A70E31E58425841D7
:108E7800FFF782FF3046F8F73BF9032C05D130465F
:108E8800F8F739F901E001221A7086F8A450094868
:108E9800BDE87040F8F72AB970BD00BF560600203B
:108EA800781F00200003002057060020D31F002051
:108EB800001F00200C1E00200A4B1A7910B504462A
:108EC8002AB10146BDE810401846FBF711BFFFF76D
:108ED800C1FE054B05491B7F20465B22BDE81040BB
:108EE800FBF7E6BE0003002048000020AF1D00206D
:108EF800244B1A7970B505460E4632B10A46BDE8CC
:108F0800704001461846FCF765B91F4A1F495B23A4
:108F1800FBF7BEFE45BB1D48FBF710FA044628B315
:108F28001B491C48F9F700FA05F130011948C9B284
:108F3800F9F7EEF918491748F9F7F6F9204602F05B
:108F480023FF01461348F9F7EFF912480A21F9F708
:108F5800DFF9012C06D0042C11D001240F49284632
:108F6800FBF702FF204670BD0748D5E72EB10C4835
:108F7800FAF7A0F90CB10224F0E70324EEE7002E7B
:108F8800F9D0F4E700030020D31F0020781F002049
:108F980081C800080C00002088C800080C1E0020AA
:108FA8000A1E0020024B1878831E58425841704709
:108FB8002B03002070B500239CB2A24200D870BDDC
:108FC800058886886C1C34404688A6421EBF2D182A
:108FD800CE5CAE7103F1010318BF0480ECE7B0F872
:108FE8001E36B0F81C262DE9F04FD21A93B21104A0
:108FF80044BF03F580639BB2E62BADF5057D0446BF
:1090080009D800F21C66012704F2123804F20E3562
:10901800F8F7D8FD18B90DF5057DBDE8F08FF9F71B
:109028005DFF294602464046FFF748F80028EFD082
:1090380094F813333E2B1CD0012394F81323212AD0
:1090480009D1B4F8162341F20D018A4278D041F2D1
:109058000E018A4277D0002BD6D004F6B5254146BA
:109068002846FFF721FA294602463046FFF7A2FFB5
:10907800CAE7B4F81633B3F5005F35D194F8983AD7
:10908800002BD9D104A804F2273E04F69F2C994658
:109098001D4603601CF8012FFF2A0DD0D10802F0ED
:1090A80007021EF8011041FA02F2D20742BF07FA7E
:1090B80003F215434FF001090133152BEAD1B9F139
:1090C800000F00D0056004F6B5250423CDE90003A0
:1090D80002223E2142F6FF732846F8F72DFF294663
:1090E80002463046FFF766FFB4F816A3BAF1740FCC
:1090F800A2D10DF1100B04F52A634FF0000900937B
:1091080004F21A32B4F81833ADF80E900DF10E01CE
:109118005846FFF741FABDF80E3084F8989A04F6DD
:10912800B525CDE900B3022253463E212846FFF774
:1091380010FA294602463046FFF73CFF4B467CE7CB
:1091480084F8457A60E784F8467A5DE72DE9F047C8
:10915800354B1B78022B04460CD00023A0F81E3692
:10916800A0F81C3690F86D3A13B10A22B2FBF3F35B
:1091780084F8983A2D4B93F82D30032B51D1204683
:10918800FFF72DFF94F8422A3AB1002384F8423AB7
:109198002046BDE8F047FFF775BB94F8433A33B172
:1091A80084F8432A2046BDE8F047FFF78DBB94F8C2
:1091B800448AB8F1000F06D084F8443A2046BDE846
:1091C800F047FFF7CDBB1A4B1F68D4F8583AFB1A83
:1091D800632B26D9C4F8587A254604F65C2604F190
:1091E800300940F6AB5A95F8702AAAB195F8713A49
:1091F8000133DBB29A420BD885F8718AD5F8743AF4
:10920800FB1A534508D931882046FFF72BFB03E0AA
:1092180085F8713A002BF1D008354D4506F1020664
:10922800E1D1BDE8F08700BF2B030020A400002097
:109238003C2D00202DE9FF477F4E804C3378012BD1
:1092480000F2D5800BB9F9F7EFF9FFF7CFFB616CA6
:109258007B48F9F789FE7B4B00221A809A707A4B7B
:1092680008229A6207254CF25030013DF9F748FB75
:10927800F9F770FB15F0FF05F5D1744803F029F8EC
:10928800013880B24FF6FD77B84203D97049012002
:10929800FBF77CFD6F4803F01CF8013880B2B84238
:1092A80002D96D490220F3E76C4B1D806C4B1D8081
:1092B80094F8523013B994F8543043B1634869496B
:1092C800FAF732FE7D20F9F745FBF9F731FA94F801
:1092D800533013B994F8553043B15E486249FAF7F0
:1092E80023FE7D20F9F736FBF9F7ACFA5F48604FAB
:1092F800FBF73EFB94F82A30029394F82930019347
:10930800A38D009394F82830626A94F820103846A8
:10931800FAF736FF94F83A30029394F8393001930B
:10932800A38F0093626B94F8301094F8383007F1EB
:10933800E0000025FAF724FF4E4BBD754FF0FF08FB
:1093480087F8F650384683F8008083F80180FAF7EA
:109358009BFF01463D4802F062FE07F1E000FAF784
:1093680093FF01463B4802F05AFE434B43481D70A9
:10937800434B1D70434B1D80434B1D70434B1D7069
:10938800434B1D70434B1D70434B1D70434B1D7069
:10939800FFF71EFC424BB4F84A201D70414B94F86D
:1093A80040101D70404B1D70B4F84830F7F765FE4B
:1093B800B4F848103D48F8F7B5F93D48FBF7EEFC1E
:1093C8003C4B3D4893F8291000F0B3FC3B48FEF7AE
:1093D800FFFB3B48FFF758F91C48FAF7C2FE394B28
:1093E8001D80394B1D80F9F757FE86F80080F9F784
:1093F8005DFE002800F08780224A13880BB1013BEC
:1094080013801F4B0F4A1978138802290DD183B195
:10941800013B9BB213809278002A57D0002B5ED173
:10942800F9F760FAF9F76CFA59E0002BF0D1C72385
:10943800F0E740F2F313EDE7511D0020480000204B
:10944800100000205206002000040048C81E00201A
:109458008AC80008E41E002094C800084E060020B0
:10946800500600204C000020580000200003002077
:109478003C030020521D0020580600200C1E00202E
:109488002B0300202E0300202C030020280300209B
:10949800290300202A030020570600205606002032
:1094A80033030020320300204C060020081F002050
:1094B800001F0020A4000020DC1C00206006002003
:1094C800080F0020181F00201A1F002002299848A2
:1094D80040F0A0800BB9F9F705FA08238362954D8F
:1094E8002B88002B00F09C80013B9BB292482B807C
:1094F800FBF782FA9148FAF734FE2B881BB990499A
:109508009048F8F711FF904F3B78002B00F08B80C4
:10951800022B00F0CA8094F8523013B994F85430F2
:109528001BB38A4D2B889BB2FBB13B78032B40F0D1
:10953800C7802B88D90702D500232B803B702B8846
:109548009BB293B12B88824A9B0548BF2B882B88F6
:10955800980748BF2B882B88D90748BF2B8800233A
:1095680013707C4A2B803B70137094F8533013B9F6
:1095780094F855301BB3784D2B889BB2FBB13878E3
:10958800032840F0B0802B88DA0702D500232B800F
:109598003B702B889BB293B12B88990548BF2B88C9
:1095A8002B889A0748BF2B882B88694ADB0748BF56
:1095B8002B8800231370674A2B803B701370674B0E
:1095C8001A7802F0FF09002A00F073824FF00008B1
:1095D80083F8008094F8523094F85300DFF880A1A3
:1095E800002B00F0CD80002800F08E815949584AA0
:1095F8000B78002B40F08A801678B6EB080618BF67
:1096080001261378012B00F2E382002E40F0E68257
:1096180035467CE110228262002B7FF460AF01E7BF
:1096280040F2E73362E74F4B1B7813B14E48FAF725
:1096380071FE4D48FAF728FE0146404802F0EFFC5B
:109648004A48FAF721FE0146494802F0E8FC94F836
:1096580052306BB139484FF6FF71F9F761F802F0F3
:1096680074FD3648002102F0A4FD7D20F9F772F957
:1096780094F853306BB13E484FF6FF71F9F7A2F8F2
:1096880002F063FD3A48002102F093FD7D20F9F7CE
:1096980061F92F4A01233B70002313702D4A137080
:1096A8002D4A1380294A138035E73248FBF7B8FB67
:1096B800314B187AFFF700FC03233B700023EFE7D8
:1096C800012B7FF43CAF2B889A077FF538AF204BEE
:1096D8001978B1FA81F1002049092880FFF708FCC0
:1096E8001C4B18702BE701287FF453AF2B889B077E
:1096F8007FF54FAF00232B80164B1978B1FA81F113
:109708004909FFF7F5FB124B187042E7012B064693
:109718003FF477AF9AF9A130009312789AF9A03004
:10972800097816483546F7F7E2FF464637E000BFA6
:1097380000040048181F002000030020C81E002055
:109748009FC800080C000020580600205006002082
:1097580057060020560600204E0600203103002040
:109768000C1E00202B0300203C0300201C040020BA
:10977800E41E0020521D0020081F0020501D00205C
:10978800002800F0C180A74B1B78012B8CBF012556
:1097980000250CBF01260026002B00F0B880FFF73B
:1097A80047FB94F8542094F85530002A00F0B38011
:1097B800002B00F0B5809AF9A1309A4A9A49009393
:1097C80012789AF9A03009789848F7F7C5FF2DB9AB
:1097D800974B1D77DD831D62964B1D70DFF858820D
:1097E80098F80010012900F2C680B5B19AF8A8309F
:1097F8003E2B00F29F809AF8A700904A002840F07C
:10980800A68092F816C09C4500F08F80D17D937594
:10981800994240F288802E46002598F80030002BA7
:1098280040F0CC8106B13B70854EB4F84E203378B9
:109838000133DBB29342337005DB8048FAF76AFDE7
:10984800002333703B707D48FAF734FD06467D48A7
:10985800FAF730FD06B908B100233B707A4B0022B5
:109868001A7098F80020002A00F0A2811DB9012280
:109878001A7002233B707548FAF702FC7448FAF72D
:10988800FFFB98F80030022B02D0724B00221A70AE
:10989800714A13880BB9B4F84A30013B9BB2138064
:1098A80013B96E48F7F76DFC6C48F7F71EFC98F88B
:1098B8000030022B0CD06948F7F7C7FB98F8003046
:1098C80033B9FFF793F9664A01231370654A137099
:1098D800654D2846F9F73CFC6B786448012B01BFBD
:1098E80000226A70614A5371FBF7B0F8FBF7C6F8BB
:1098F8000128054667D0022800F0CC805C4B052281
:109908001A7004B0BDE8F087474B3DE70546514B58
:1099180001221A7045E71BB1444B01221A7256E71F
:10992800424B0022FAE7907575E75248027842F0F8
:1099380001020270504849BB3F2B4E4B01704FF05B
:10994800010228BF032188F80020197016E092F858
:10995800F60098420AD092F8F71082F8F630994249
:109968003FF659AF002382F8F63054E741480278B1
:1099780042F00202DDE7002D3FF44FAF3F4BB4F851
:109988004C201A8002233B704D4646E703783C4939
:1099980001330A78DBB203706AB994F85020934215
:1099A800ECD3344B1B78032B07D1022388F8003003
:1099B80001230B70E2E70522F1E7531EDBB2934265
:1099C8000370F2D2DAE72948FAF7EEFFB4F8483024
:1099D8002C4A2D4803EB830303EB83039B0013807E
:1099E800F9F768FC154BB4F8482083F8D85041F2D1
:1099F8008831B1FBF2F10022A3F8DA10A3F8BA110A
:109A0800A3F8DC2083F8B851A3F8BC211F4B102120
:109A18009961082199621E4B88F800209D703A7060
:109A28006CE700BF5706002056060020081F0020DC
:109A380060060020080F00202B0300203C030020B4
:109A4800290300201C0400204C060020C81E00200A
:109A5800E41E0020001F00201A1F00200C1E0020FA
:109A6800590600201C1F0020241D00200003002090
:109A780033030020280300202C0300202E0300209D
:109A88002A030020440000200A1E00200004004889
:109A980052060020534B93F8D930052B08D8524A68
:109AA800D25C524B83F81921514B01221A7025E7D9
:109AB800FEE75049504A0B781BB1013BDBB20B70F3
:109AC80013B11378002B34D0484D4C4895F8281022
:109AD8000024147000F058F9494B1B78022B46D12A
:109AE800484F494897F80090F7F708FB80464648E2
:109AF800F7F716FB454923464A46CDE900803F481B
:109B080000F05AFC3D48FBF715FB3A7840494148BC
:109B18002346FDF78BFA3A783D493F482346FEF73E
:109B2800EDFD95F8263095F8332038493B48FBF78A
:109B3800A1F9324800F050FD3648FEF721FA3648C0
:109B4800FFF704FB2A4B1B78002B3FF4DAAE3448AE
:109B5800FAF796FA3348FAF793FA334B08229A61E0
:109B680010229A61FAF7DEF801233370C9E62F4B09
:109B78001B78C3B16FF07E03009301231A46234973
:109B88001E48019400F018FC1C4800F014F9012349
:109B98001A461F491F48FDF749FA01231C491E4868
:109BA8001A46FEF7ABFD1D4B95F826205A70C0E704
:109BB8003B7813F0FD0F3FF45EAE66E61C4B1B8846
:109BC800002B7FF44BAE1B4A88F80030137044E634
:109BD800002E3FF49BAE4FF000089BE5B0460026F0
:109BE80098E500BF3C030020F0CB0008A40000204B
:109BF800300300203303002032030020DC1C002047
:109C08002B0300204C0600200C1E00202C1D0020D9
:109C1800001D002060060020080F0020521D0020B3
:109C2800C81E0020E41E0020000400482A0300206B
:109C38002E0300202903002008B5FFF7FBFAFCE7F4
:109C48001E4B1F4A10B51A601E4B1F4A1A601F4B45
:109C58001F4A204C1A605A619A62DA631A651E4AD2
:109C68005A669A671D4AC3F88C20204600F048F8C7
:109C78001B4B23601B4B002240F2FF11C3F8E82462
:109C8800C3F8EC14184BC3F81C26C3F8502A7D22DD
:109C980083F8542A154A40F2FF311068C3F8201699
:109CA800516803F65C2403C490682060D068128A67
:109CB800C3F8680AA3F86C2A10BD00BFC81E0020AC
:109CC800ACC80008E41E0020D4C800080C1E002000
:109CD80014C80008DC1C0020FCC7000808C80008DD
:109CE8005CC9000860060020080F002010C60008A4
:109CF8007047002070470020704700207047000020
:109D080010B5044B0446012140F8043BF7F74AF923
:109D1800204610BD2CE4000838B5242204460D4620
:109D2800FF23002103618182104402F0F1FBE5600A
:109D380038BD38B50D46017CA942044615D0012925
:109D480018D0022912D011B903685B68984700231C
:109D5800012D6374257413D0022D0ED02DB92368FC
:109D68005B68012120469847607438BD0368DB684A
:109D78000021EBE703689B68FAE72368DB68F0E7F4
:109D8800236829469B68EDE70430F7F719B9037C87
:109D9800012B10B50ED100F1160301F10C0251F898
:109DA800044B43F8044B9142F9D10A881A8040F2D7
:109DB8000113438210BD037C012B0BD148F28113A0
:109DC800C3824FF401420023C0E90632038440F203
:109DD800011343827047F0B5054689B008880C46E0
:109DE80016461F46F7F751FA9DF806308DF805001C
:109DF80023F00703C0F30220034360888DF8063080
:109E0800F7F743FA9DF8063000F01F0203F0070346
:109E180043EAC2038DF806309DF80730C0F34510B9
:109E280023F03F030343A0888DF80730F7F72DFA96
:109E38009DF8073000F0030203F03F0343EA821362
:109E48008DF80730C0F387038DF808309DF8093086
:109E5800C0F3802023F001030343E0888DF8093024
:109E6800F7F713FA9DF8093000F07F0203F00103B9
:109E780043EA42038DF809309DF80A30C0F3C31055
:109E880023F00F03034320898DF80A30F7F7FDF913
:109E98009DF80A3000F00F0203F00F0343EA0213A3
:109EA8008DF80A309DF80B30C0F3061023F07F03BD
:109EB800034360898DF80B30F7F7E7F99DF80B300D
:109EC80000F0010203F07F0343EAC2138DF80B3060
:109ED800C0F347038DF80C309DF80D30C0F34120D6
:109EE80023F003030343A0898DF80D30F7F7CDF96C
:109EF8009DF80D3000F03F0203F0030343EA8203AC
:109F08008DF80D309DF80E30C0F3841023F01F0338
:109F18000343E0898DF80E30F7F7B7F99DF80E3056
:109F280000F0070203F01F03C0F3C70043EA42131F
:109F38008DF80F00208A8DF80E30F7F7A6F99DF8F6
:109F480011308DF8100023F00703C0F302200343FB
:109F5800608A8DF81130F7F798F99DF8113000F004
:109F68001F0203F0070343EAC2038DF811309DF87E
:109F78001230C0F3451023F03F030343A08A8DF845
:109F88001230F7F782F99DF8123000F0030203F05F
:109F98003F0343EA82138DF81230C0F387038DF82C
:109FA80013309DF81430C0F3802023F001030343DD
:109FB800E08A8DF81430F7F768F99DF8143000F04E
:109FC8007F0203F0010343EA42038DF814309DF841
:109FD8001530C0F3C31023F00F030343208B8DF813
:109FE8001530F7F752F99DF8153000F00F0203F01D
:109FF8000F0343EA02138DF815309DF81630C0F3AD
:10A00800061023F07F030343608B8DF81630F7F7B3
:10A018003CF99DF8163000F0010203F07F0343EA93
:10A02800C2138DF81630C0F347038DF817309DF82A
:10A038001830C0F3412123F003030B43A08B8DF8A4
:10A048001830F7F722F99DF8183000F03F0203F0B6
:10A05800030343EA82038DF818309DF81930C0F3E2
:10A06800841023F01F030343E08B8DF81930F7F7B2
:10A078000CF99DF81930218C00F0070203F01F033A
:10A0880043EA42138DF81930628C40F2A953994281
:10A0980088BF0121C0F3C70098BF00219A428DF8FC
:10A0A8001A0088BF41F002010EB141F004010FB15E
:10A0B80041F008010F238DF8043000238DF81C307F
:10A0C8002B688DF81B101B68192201A92846984790
:10A0D80009B0F0BD30B5054689B008880C46F7F7D9
:10A0E800E1F89DF808308DF8070023F00703C0F366
:10A0F8000220034360888DF80830F7F7D3F89DF8FD
:10A10800083000F01F0203F0070343EAC2038DF88A
:10A1180008309DF80930C0F3451023F03F0303438E
:10A12800A0888DF80930F7F7BDF89DF8093000F0E0
:10A13800030203F03F0343EA82138DF80930C0F3AA
:10A1480087038DF80A309DF80B30C0F3802023F088
:10A1580001030343E0888DF80B30F7F7A3F89DF867
:10A168000B3000F07F0203F0010343EA42038DF84D
:10A178000B309DF80C30C0F3C31023F00F030343DA
:10A1880020898DF80C30F7F78DF89DF80C3000F029
:10A198000F0203F00F0343EA02138DF80C309DF809
:10A1A8000D30C0F3061023F07F03034360898DF858
:10A1B8000D30F7F777F89DF80D3000F0010203F045
:10A1C8007F0343EAC2138DF80D30C0F347038DF8BF
:10A1D8000E309DF80F30C0F3412023F003030343F2
:10A1E800A0898DF80F30F7F75DF89DF80F3000F073
:10A1F8003F0203F0030343EA82038DF80F309DF812
:10A208001030C0F3841023F01F030343E0898DF856
:10A218001030F7F747F89DF8103000F0070203F008
:10A228001F03C0F3C70043EA42138DF81100208AC8
:10A238008DF81030F7F736F89DF813308DF81200C6
:10A2480023F00703C0F302200343608A8DF813301C
:10A25800F7F728F89DF8133000F01F0203F0070302
:10A2680043EAC2038DF813309DF81430C0F345104B
:10A2780023F03F030343A08A8DF81430F7F712F850
:10A288009DF8143000F0030203F03F0343EA821301
:10A298009DF816208DF81430C0F387038DF815301B
:10A2A80022F00102C0F380231343E08A8DF81630B0
:10A2B800F6F7F8FF9DF8163000F07F0203F001036F
:10A2C80043EA42038DF816309DF81730C0F3C310E7
:10A2D80023F00F030343208B8DF81730F6F7E2FFC6
:10A2E8009DF8173000F00F0203F00F0343EA021342
:10A2F8008DF817309DF81830C0F3061023F07F034F
:10A308000343608B8DF81830F6F7CCFF9DF81830B2
:10A3180000F0010203F07F0343EAC2139DF81A20FC
:10A328008DF81830C0F347038DF8193022F0030276
:10A33800C0F341231343A08B8DF81A30F6F7B2FF10
:10A348009DF81A3000F03F0203F0030343EA82034A
:10A358008DF81A309DF81B30C0F3841023F01F03CA
:10A368000343E08B8DF81B30F6F79CFF019B03F04D
:10A378007F42104B134301939DF81B3000F00702F6
:10A3880003F01F03C0F3C70043EA42138DF81C0013
:10A398000DF10601172200208DF81B30F6F7EEFFAD
:10A3A8002B688DF81D001B681A2201A928469847BA
:10A3B80009B030BDC81816002DE9F04700F1240790
:10A3C8009DF920A09DF8249090461E4604463B46E1
:10A3D80001F1240251F8040B43F8040B9142F9D11E
:10A3E800251D39462846F6F70FFEE1684B7966B118
:10A3F800042B77D8DFE803F07C76345C03004FF059
:10A408000423C4E909330026B046E3681D796B1EAE
:10A418000B2B07D850460435F6F70DFFEDB204EBC9
:10A4280045056884E3681D7B6B1E0B2B07D84846DF
:10A438000435F6F71BFFEDB204EB45056884637C31
:10A44800002B55D0237C012B46D013F0FD0F4FD1A4
:10A458003346424639462046BDE8F047FFF7BBBCC5
:10A4680001F1130304F1220001F11F054FF0780CEC
:10A4780013F9012FC2EB8222AB4292FBFCF202F5E8
:10A48800806220F8022FF3D104F13A02233140F21E
:10A49800FF7513F8010F48B102280CBF28464FF486
:10A4A8008060994222F8020FF3D1AEE70120F8E765
:10A4B80004F1220304F146024FF4806123F8021FDD
:10A4C8009342FBD102212846F6F7BCFD103004EB7D
:10A4D80040000023838098E739462046BDE8F047CE
:10A4E800FFF7F8BD042B90D813F0FD0F8DD0E9E7E6
:10A4F800BDE8F08730B54B7B032B85B005460C468D
:10A5080042D191F90000F6F713FF8DF8030094F992
:10A518000100F6F70DFFA3788DF80530E3788DF884
:10A5280004008DF80630207B23798DF80730F6F784
:10A53800F7FE8DF8080094F90600F6F7CBFE8DF8C3
:10A54800090094F90700F6F7F3FE237A8DF80B302B
:10A55800637A8DF80C3040F6C8438DF80A00ADF8E0
:10A5680000300DF1020114230B2200208DF8023077
:10A57800F6F704FF2B688DF80D001B680E2269465C
:10A588002846984705B030BD022B03D1FF238DF82C
:10A598000330BCE791F90000F6F7CAFE8DF8030016
:10A5A800FF20B8E7837C10B5044633B1F8F7A0FD67
:10A5B800E37C1BB10023A082E37410BDA28A801A39
:10A5C80080B2B0F57A6FF8D9A37404F11601204669
:10A5D800BDE81040FFF78EBF427C22B1037C012BFF
:10A5E80001D1FFF7DFBF704730B59BB020220021B3
:10A5F8000BA801F08DFF1822002102A801F088FFA6
:10A608001C4A136823F4C06343F40073136013688F
:10A6180003F4C0630193019B01224FF40413CDE9B5
:10A62800082300230A9310210623CDE915134FF4BC
:10A6380000330224032517934FF0005C4FF000739A
:10A6480008A8CDE91345CDE9183C00F045FB08B151
:10A6580072B6FEE7CDE90400CDE906004F23214696
:10A6680002A8CDE9023500F0D1FD08B172B6FEE7C7
:10A678001BB030BD00040058154B07B51A6842F4EA
:10A6880080721A601A6842F400721A601A6822F41A
:10A6980080621A6000F0A0F8FFF7A6FF4FF0B04301
:10A6A800DA6C42F00102DA64DA6C02F0010201921B
:10A6B800019ADA6C42F00202DA64DB6C03F00203FE
:10A6C8000093009B03B05DF804EBFFF7B5BA00BF39
:10A6D800004000587047FEE7FEE7FEE7FEE7FEE7AA
:10A6E800704770477047F8F7F1BC70470D488546CA
:10A6F800FFF7FBFF0C480D490D4A002302E0D45830
:10A70800C4500433C4188C42F9D30A4A0A4C0023B3
:10A7180001E013600432A242FBD301F02FFFFFF7E0
:10A72800ABFFFEE700000120000000202800002009
:10A7380018E5000828000020782D0020FEE7704763
:10A748004FF0B04310B59A6B4FF0FF329A63D96B54
:10A75800DA630024996B9C63D96BDC63196C1A6407
:10A76800196C1C64596C5A64596C5C64996A9A62D5
:10A77800996A9C62D96ADA62D96ADC62196B1A63CF
:10A788001A6B1C63FFF7DBFF204610BD38B5104C71
:10A79800237805460BB9012038BD00F08DFA2278E0
:10A7A8004FF47A73B3FBF2F3B0FBF3F000F074F8F4
:10A7B80004460028EFD10F2DEDD8024629464FF068
:10A7C800FF3000F037F8034B20461D60E4E700BF78
:10A7D800200000202400002010B5032000F018F805
:10A7E80000F06AFA064B18600F20FFF7CFFF044607
:10A7F80018B9FFF76FFF204610BD0124FBE700BF23
:10A808001C000020014B1868704700BF3C2D002039
:10A818000749CA6822F4E0620302120403F4E06301
:10A82800120C134343F0BF6343F40033CB6070470B
:10A8380000ED00E0164B30B5DC68C4F30224C4F127
:10A848000703251D042B28BF0423062D4FF0FF35D1
:10A858008CBF033C002405FA03F321EA0303A54057
:10A8680022EA0502A340002843EA0203ACBF00F134
:10A878006040084A4FEA0313B8BF00F00F00DBB28C
:10A88800AABF00F56140135480F8003330BD00BF03
:10A8980000ED00E014ED00E00138B0F1807F0BD24C
:10A8A8004FF0E023054A5861F02182F82310002078
:10A8B800072298611A6170470120704700ED00E097
:10A8C8000A4A536943F4802330B55361EFF3108487
:10A8D80072B60023CD58C5500433B3F5807FF9D143
:10A8E8001369DB03FCD484F3108830BD00400058A2
:10A8F800064B5A69002ABFBF054A9A6002F188329E
:10A908009A60BABF5869C00F0020704700400058CD
:10A9180023016745044B5A6942F000425A6158695D
:10A92800C043C00F704700BF0040005870B50546CF
:10A93800FFF768FF124E04463369D90313D433690D
:10A94800DA0744BF012232614CF2FA32134011D1C6
:10A958000B4E306910F480200BD0FFF753FF001B1B
:10A96800A842F6D304E0FFF74DFF001BA842E3D34B
:10A97800032070BD024A1361024A01205360F8E7C0
:10A9880000400058402D00202DE9F041184D984610
:10A998002B78012B06460C46174626D001232B7030
:10A9A8004FF47A7000236B60FFF7C0FFA0B9012E47
:10A9B80016D1104A536943F0010353612760BFF36E
:10A9C8006F8FC4F804804FF47A70FFF7AFFF094A1D
:10A9D800536923EA0603536100232B70BDE8F08115
:10A9E80039462046FFF76CFFEDE70220F6E700BF87
:10A9F800402D002000400058054A536923F47E7317
:10AA080043EAC00040F4803040F0020050617047D3
:10AA1800004000582DE9F041234F3B78012B0546B3
:10AA280088463FD001233B704FF47A7000237B6047
:10AA3800FFF77CFF044688B92B68042B13D11B4A07
:10AA4800536943F4803343F0040353614FF47A703D
:10AA5800FFF76CFF0446154B1A681B6800233B7010
:10AA68002046BDE8F0814FF0FF33C8F800306E682B
:10AA7800D5E901321344B3420AD93046FFF7BCFF87
:10AA88004FF47A70FFF752FF50B1C8F800600446DF
:10AA9800064A536923F47E7323F002035361DAE70D
:10AAA8000136E5E70224DBE7402D0020004000588E
:10AAB800024A136843F48073136070470004005817
:10AAC800024B186800F4C060704700BF00040058CB
:10AAD8004FF0B0431868C0F3404070474FF0B043A0
:10AAE8001868C0F3400070474FF0B042536823F431
:10AAF8007F4343EA0023536070474FF0B043186820
:10AB0800C0F34060704700007FB54FF0B0432C4A57
:10AB1800D3F80831C0F3031003F00F0352F82040B4
:10AB2800284A52F82330B4FBF3F4FFF7C9FF264B49
:10AB3800054693E80700B5F5007F04AB03E9070075
:10AB480010D0224B9C4218D303F5B70303F67F536A
:10AB58009C4229D903F5741303F510639C4225D848
:10AB680002230BE01A4B9C4207D91A4B9C421BD973
:10AB780003F5370303F5D853F0E7002304AA02EBE3
:10AB8800830353F80C4C144D2B6823F0070323431D
:10AB98002B60FFF737FE06462B6803F007039C423D
:10ABA80006D1002004B070BD0123E7E70024EAE7DE
:10ABB800FFF728FE801B0228EED90320F2E700BF2A
:10ABC8009CE400083CE4000824C60008C0CF6A00E2
:10ABD800BFEA21013F933402004000584FF0B043D0
:10ABE80010B59A68D96812F00C0205D00C2A4AD11F
:10ABF80001F00303012B50D14FF0B0412B480B68F3
:10AC080013F0080306D00B6813F0080337D1D1F806
:10AC1800941007E00C68240756BFD1F894300968EF
:10AC2800C3F3032350F82330002A0CBF1846002032
:10AC38004FF0B0418A6802F00C020C2A1ED1CA6893
:10AC480002F00302022A2ED0032A06D10B68184A02
:10AC580013F4801F174B18BF13464FF0B042D0684B
:10AC6800D168D268C0F306205843C1F302130133F8
:10AC7800B0FBF3F0530F0133B0FBF3F010BD0B68DA
:10AC8800C3F30313CEE7042A0AD0082A05D11B68A8
:10AC980013F4801304D10748CAE700231846C7E70E
:10ACA80003480023C4E7024BD7E700BF9CE4000831
:10ACB8000024F4000048E80108B5FFF78FFF4FF0C3
:10ACC800B043044A9B68C3F3031352F82330B0FB24
:10ACD800F3F008BD3CE400082DE9F04104460028E3
:10ACE80053D04FF0B0439D68DE6803689B0605F0BB
:10ACF8000C0506F0030668D5026A1DB10C2D46D175
:10AD0800012E44D1002A40D04FF0B043A16A1A68FE
:10AD1800170756BFD3F894301B681B0903F0F003DC
:10AD280099421FD90846FFF7EFFE00282DD14FF0B2
:10AD3800B042136843F0080313601368A16A23F054
:10AD4800F0030B431360606AFFF7CEFEFFF7B4FF12
:10AD5800AB4B1860AB4B1868FFF718FD002834D0D0
:10AD6800BDE8F0814FF0B042136843F00803136068
:10AD7800136823F0F0030B431360606AFFF7B4FE17
:10AD88000846FFF7C1FE0028E0D00120E8E74FF0B1
:10AD9800B043002A54D01A6842F001021A60FFF743
:10ADA80031FD0746FFF79AFE002842D04FF0B04227
:10ADB800136843F0080313601368A16A23F0F003D3
:10ADC8000B431360606AFFF78FFE2368D80748D4E7
:10ADD8002368990700F18C8023681E0740F1FA80E8
:10ADE800A3694FF0B046002B00F0E180D6F894300C
:10ADF800E16903F01002914200F0C48003F00302FD
:10AE0800022AC2D0D80740F1B380D6F8943023F094
:10AE18000103C6F89430FFF7F5FC0746D6F89430DE
:10AE2800990740F1A580FFF7EDFCC31B112BF5D95D
:10AE380004E0FFF7E7FCC01B0228B3D903208FE723
:10AE48001A6822F001021A60FFF7DCFC0746FFF7D8
:10AE580045FE0028B9D0FFF7D5FCC01B0228F6D95B
:10AE6800ECE7082D03D00C2D05D1032E03D1636820
:10AE7800002BADD189E74FF0B043A1681A6822F4DE
:10AE880080120A431A606268B2F5803F10D11A68CE
:10AE980042F480321A60FFF7B5FC0746FFF718FE48
:10AEA800002895D1FFF7AEFCC01B6428F6D9C5E78A
:10AEB800B2F5041F04D11A6842F400121A60E6E7DA
:10AEC800196821F480311960196821F4001119609A
:10AED800002AE0D1FFF796FC0746FFF7F9FD0028A6
:10AEE8003FF476AFFFF78EFCC01B6428F5D9A5E7C1
:10AEF800042D236903D00C2D0ED1022E0CD1002B6A
:10AF08003FF443AF4FF0B0426169536823F0FE430A
:10AF180043EA016353605FE74FF0B046BBB1336863
:10AF280043F480733360FFF76DFC074633685A05B6
:10AF380007D57368626923F0FE4343EA02637360CE
:10AF48004AE7FFF75FFCC31B022BEFD976E73368AC
:10AF580023F480733360FFF755FC074633685B05BD
:10AF68007FF53AAFFFF74EFCC31B022BF6D965E716
:10AF78004FF0B042E169D2F8943023F010030B434C
:10AF8800C2F894304FF0B047D7F8943043F001033B
:10AF9800C7F89430FFF736FC0646D7F894309A077E
:10AFA80018D4FFF72FFC831B112BF6D946E7D6F8E8
:10AFB800943023F00103C6F89430FFF723FC0746CA
:10AFC800D6F894309B0705D5FFF71CFCC31B112B43
:10AFD800F6D933E72368580754D50B4F3B68D90592
:10AFE80014D4FFF765FDFFF70DFC06463B68DA054C
:10AFF8000CD4FFF707FC831B022BF7D91EE700BF11
:10B008001C0000202400002000040058E3684FF0D2
:10B01800B046002B58D023F08003052B02BFD6F88A
:10B02800903043F00403C6F890304FF0B046FFF775
:10B03800E9FBD6F8903043F001030746C6F8903094
:10B0480041F28838D6F890309B0705D4FFF7DAFB31
:10B05800C31B4345F6D9F1E6E36823F00403812BCB
:10B068001BD1FFF7CFFBD6F8903043F08003C6F82A
:10B07800903007464FF0B04641F28838D6F8903005
:10B08800180504D5E06A00284AD1002068E6FFF7D1
:10B09800B9FBC01B4045F1D9D0E6FFF7B3FBD6F8A2
:10B0A800903023F08003C6F8903007464FF0B04642
:10B0B80041F28838D6F890301905E3D5FFF7A2FB9E
:10B0C800C01B4045F6D9B9E6FFF79CFBD6F890308F
:10B0D80023F080030746C6F8903041F28838D6F846
:10B0E80090301A0516D4FFF78DFBD6F8903023F070
:10B0F8000103C6F8903007464FF0B04841F2883651
:10B10800D8F890309B07BDD5FFF77CFBC31BB34233
:10B11800F6D993E6FFF776FBC01B4045DFD98DE6ED
:10B128000C2D4ED04FF0B04302281A6822F08072DE
:10B138001A6033D1FFF766FB0546FFF7DEFC38BB24
:10B14800D4E90C314FF0B0420B43D0682D4901408F
:10B158000B43E16B0B43216C0B43616C0B43A16BFD
:10B1680043EA0123D360136843F080731360D36804
:10B1780043F08053D360FFF745FB0446FFF7BDFC5F
:10B18800002882D1FFF73EFB001B0A28F6D955E6B6
:10B19800FFF738FB401B0A28CFD94FE6FFF732FBF1
:10B1A8000446FFF7AAFC30B94FF0B042164BD168FD
:10B1B8000B40D360D4E5FFF725FB001B0A28F0D924
:10B1C8003CE601283FF4CCAD4FF0B043226BDB687E
:10B1D80003F0030191427FF4D8AD616B03F0700274
:10B1E8008A427FF4D2ADA16B03F4FE42B2EB012F89
:10B1F8007FF4CBAD626C03F0604393423FF445AFFC
:10B20800C3E500BF8C80C111FCFFFEEE2DE9F041C3
:10B218000D46044610B90120BDE8F081684E336838
:10B2280003F007038B4216D323689A0727D54FF0FC
:10B23800B047A268BB6823F0F0031343BB60FFF775
:10B24800E1FA0646BB68DB0319D4FFF7DBFA831B78
:10B25800022BF7D911E0336823F007030B4333605F
:10B26800FFF7D0FA0746336803F00703AB42DBD099
:10B27800FFF7C8FAC01B0228F5D90320CCE72368DA
:10B28800580617D54FF0B0476269D7F8083123F050
:10B298000F0343EA1213C7F80831FFF7B3FA06465B
:10B2A800D7F80831D90305D4FFF7ACFA831B022B72
:10B2B800F6D9E2E723685A0713D54FF0B047E2689A
:10B2C800BB6823F4E0631343BB60FFF79BFA0646B1
:10B2D800BB689B0305D4FFF795FA831B022BF7D9AC
:10B2E800CBE72368180714D54FF0B0472269BB682D
:10B2F80023F4605343EAC203BB60FFF783FA0646B0
:10B30800BB68590305D4FFF77DFA831B022BF7D9D5
:10B31800B3E72368DA070FD4294C236803F007033F
:10B32800AB4239D8FFF7C8FC264B1860264BBDE85E
:10B33800F0411868FFF72ABA6268022A1DD1FFF7A0
:10B34800C7FB00283FF467AF4FF0B04641F288389A
:10B35800B36823F003031343B360FFF753FA0746B8
:10B36800B368626803F00C03B3EB820FD4D0FFF725
:10B3780049FAC01B4045F3D97FE7032A02D1FFF7FA
:10B38800BCFBDEE712B9FFF7A9FBDAE74FF0B043E1
:10B398001B685B05D8D43EE7236823F007032B43DB
:10B3A8002360FFF72FFA0646236803F00703AB4232
:10B3B800B8D0FFF727FA801B0228F5D95DE700BF50
:10B3C800004000581C0000202400002030B504680C
:10B3D80091FAA1F3B3FA83F303255B0005FA03F3AB
:10B3E80024EA030391FAA1F1B1FA81F149008A40F4
:10B3F8001A43026030BD0000B0F1904F0BD14FF0FE
:10B40800B043DA6A42F00102DA62DA6A22F0010233
:10B41800DA6201207047144B984209D14FF0B043CB
:10B42800DA6A42F00202DA62DA6A22F00202EFE72E
:10B438000E4B984209D14FF0B043DA6A42F0040249
:10B44800DA62DA6A22F00402E2E7094B984209D18B
:10B458004FF0B043DA6A42F08002DA62DA6A22F028
:10B468008002D5E700207047000400480008004823
:10B47800001C00482DE9F84F0E460F6897FAA7F50B
:10B488004FF0010BB5FA85F54FF0030A4FF00F089E
:10B4980037FA05F302D10120BDE8F88F0BFA05F45D
:10B4A8003C4053D0D6F8049021464A46FFF78EFF19
:10B4B80009F1FF33012B19D8B368816894FAA4F213
:10B4C800B2FA82F252000AFA02F221EA020294FA6D
:10B4D800A4F1B1FA81F149008B40134383604268BB
:10B4E800F36822EA04026343134343603369C16883
:10B4F80094FAA4F2B2FA82F252000AFA02F221EAAB
:10B50800020294FAA4F1B1FA81F149008B40134385
:10B51800B9F1020FC36015D1FF2C716918D8026AFE
:10B5280094FAA4F3B3FA83F39B0008FA03F322EA2C
:10B53800030294FAA4F3B3FA83F39B0001FA03F32A
:10B54800134303624A462146FFF740FF01359FE750
:10B55800426A230A93FAA3FCBCFA8CFC4FEA8C0CCF
:10B5680008FA0CFC22EA0C0293FAA3F3B3FA83F369
:10B578009B00994011434162E4E74FF0B0431868DB
:10B58800C0F3005070474FF0B0431868C0F38020F4
:10B5980070474FF0B043D3F89000C0F340007047B5
:10B5A8004FF0B0431868C0F3C00070474FF0B04385
:10B5B8001868C0F3406070474FF0B043044A9B6876
:10B5C800C3F3031352F82330B0FBF3F0704700BF06
:10B5D8003CE400084FF0B043034A9B68C3F30223DE
:10B5E80052F82330D84070477CE400084FF0B0424E
:10B5F80038B5916801F00C01082950D017D889B3E3
:10B60800042900F08C80FFF7CBFF4649024600284A
:10B6180076D1FFF7C5FF4FF0B043012816BFD3F826
:10B6280094201B68C2F3032251F822002AE00C2957
:10B63800E9D1D36803F00303022B5FD0032B37D083
:10B64800FFF7AEFF374C014600284AD1FFF7A8FFA5
:10B65800012816BFD2F894101368C1F3032154F8D7
:10B6680021302CE0FFF79CFF2E4D044658B9FFF718
:10B6780097FF012816BFD2F894401368C4F3032437
:10B6880055F8240038BDFFF78BFF01280ABF116861
:10B69800D2F89430C1F3031155F82100F2E7FFF70F
:10B6A8006CFF214B01462148012908BF1846E9E7EC
:10B6B800FFF763FF1D4A1C4B012818BF13464FF0C4
:10B6C800B042D068D168D268C0F306205843C1F3AD
:10B6D80002130133B0FBF3F0530F0133B0FBF3F067
:10B6E800D0E7FFF75DFF01280BBF1368D2F894304D
:10B6F800C3F30313002354F82330E0E70A4BDEE7D3
:10B70800FFF74EFF4FF0B04301280BBF1B68D3F87B
:10B718009430C3F30313002351F82300B2E702481F
:10B72800B0E700BF9CE400080024F4000048E801EA
:10B738004FF0B04307B51A6842F001021A601A6860
:10B748009207FCD51A6822F0F00242F060021A60F3
:10B758005A6822F47F425A605A6822F0FE4242F048
:10B7680080425A604FF4E0229A601A680192019967
:10B77800104A0A400192019A1A60FFF717FF002841
:10B78800FBD14FF0B0430C4ADA6040F23F32986187
:10B798000192019A1A62D3F8942042F40002C3F885
:10B7A800942001204FF44032C3F8082103B05DF81B
:10B7B80004FB00BFFFF4CEFE0010042210B54FF0CA
:10B7C800B0440328D4F888302AD11F4A03F0030371
:10B7D80043F44033934209D0B3F1031F0DD0013A2B
:10B7E800934211D1BDE81040FFF700BFFFF7CBFE31
:10B7F8000128164818BF002010BDFFF7CAFE431ED7
:10B8080058425841C003F7E7FFF7F0FEFFF7D4FEB0
:10B81800A3680F4AC3F3C22352F82330D840EBE79A
:10B82800034043EA00400B4B9842DFD0B0F10C1FB5
:10B83800E3D0043B9842D5D0FFF7D8FEFFF7BCFE13
:10B84800BDE81040FFF7C6BE020003000024F40064
:10B858007CE4000808000C0003685B0670B502462B
:10B868002DD4D1E900363343CE68056848690C6A9F
:10B8780033430E6933438E6903433343CE6925F45A
:10B888007F45334325F0BF0523432B43136053689B
:10B898008D6823F4706323F0040345EA10401843CD
:10B8A800B5F5006F50603EBF536843F48053536052
:10B8B800B4F5005F01D18B8C1361012000E00020FA
:10B8C800D36923F40063D36170BD00001A4A03688A
:10B8D800904210B502D0B0F1804F09D14C6823F0E6
:10B8E8007003904243EA040309D0B0F1804F06D0B8
:10B8F800124A904203D002F58062904203D1CA688E
:10B9080023F44073134303608B68C3620B8883621C
:10B91800094B984207D003F5C053984203D003F56A
:10B928008063984201D10B690363436943F00103C3
:10B938004361012010BD00BF002C014000440140BC
:10B94800B1F5805F30B500F0F08009D8102975D0C6
:10B95800B1F5807F00F0AE80012935D0002030BDE0
:10B96800B1F5803F00F00E81B1F5801FF6D1036A72
:10B97800146823F480130362036A416D21F0807117
:10B9880021F4E04141EA0424116923F4001343EA55
:10B998000153516823F4801343EA015391498842C3
:10B9A80007D001F5C051884203D001F58061884273
:10B9B80006D14168956921F4802141EA85214160D9
:10B9C800D2684465C26536E0036A156823F001034E
:10B9D8000362036A4168846924F4803424F07304A0
:10B9E8002C43156923F002032B43556823F0010308
:10B9F8002B437C4DA84207D005F5C055A84203D07B
:10BA080005F58065A84212D1556923F0080343EA79
:10BA18008503956823F0040343EA8503956921F4B7
:10BA280080712943D56921F4007141EA4501D26842
:10BA38004160846142630362012090E7036A1568EC
:10BA480023F010030362036A4168846924F0807458
:10BA580024F4E64444EA0524156923F0200343EA64
:10BA68000513556823F0100343EA05135D4DA842FA
:10BA780007D005F5C055A84203D005F58065A84252
:10BA880013D1556923F0800343EA8513956823F0A1
:10BA9800400343EA8513956921F4806141EA8501F1
:10BAA800D56921F4006141EAC501D2684160846129
:10BAB8008263C0E7036A156823F480730362036A2C
:10BAC8004168C46924F4803424F073042C43156954
:10BAD80023F4007343EA0523556823F4807343EA8B
:10BAE8000523404DA84207D005F5C055A84203D00C
:10BAF80005F58065A84213D1556923F4006343EA2C
:10BB08008523956823F4806343EA8523956921F4A6
:10BB1800805141EA0511D56921F4005141EA4511E6
:10BB2800D2684160C461C26385E7036A156823F47B
:10BB380080530362036A4468C16921F0807121F46B
:10BB4800E64141EA0521156923F4005343EA053328
:10BB5800556823F4805343EA0533224DA84207D0A1
:10BB680005F5C055A84203D005F58065A84204D163
:10BB7800956924F4804444EA8514D2684460C1611C
:10BB8800026458E7036A146823F480330362036A83
:10BB9800416D21F4803121F070010C43116923F4C7
:10BBA800003343EA0143516823F4803343EA0143F5
:10BBB8000C49884207D001F5C051884203D001F5ED
:10BBC8008061884206D14168956921F4803141EA53
:10BBD800052141604465816DD268090C090411434F
:10BBE800816528E7002C01400F4B98420BD14FF09C
:10BBF800B0431A6C42F480421A641A6C22F48042F0
:10BC08001A6401207047094B98420AD14FF0B0439B
:10BC18009A6B42F400329A639A6B22F400329A6368
:10BC2800EFE70020704700BF0038014000440040A3
:10BC380038B50368DB0704460D464DD42A69AB685E
:10BC4800016813436A691343EA691343234A0A40A4
:10BC5800134303604368EA6823F440531343436083
:10BC68008368AA6923F44073134383601C4B98428A
:10BC780020D10320FFF7A2FD2B68F0B16A68E2B17A
:10BC88000B2B15D8174951F82330E969B0FBF3F0AD
:10BC9800B1F5004F4FEA520319D103EB4003B3FB50
:10BCA800F2F34FF6F0721A40C3F342031343E36012
:10BCB800012003E00C4B984207D00020E26A2B8851
:10BCC80022F00F021343E36238BD0C20D2E703448D
:10BCD800B3FBF2F39BB2EAE70020F5E7F369FFEF65
:10BCE80000380140DCE400080044004030B530244E
:10BCF80042F20F75A84212D80C703021B0F57A7F45
:10BD080014D211703022632816D81A7030230928EB
:10BD180017D8039A1370049B3030187030BDA0F503
:10BD28001C5001341038E4B280B2E3E70131A0F5C9
:10BD38007A70C9B280B2E1E701326438D2B280B217
:10BD4800E1E701330A38DBB280B2E0E713B50B1D37
:10BD58000193CB1C00934A1C8B1C0C46FFF7C6FFB3
:10BD68000023637102B010BD03099F2800F00F0083
:10BD780094BF3033373309280B7094BF30303730D5
:10BD8800002348708B70704708B50249FFF7ECFF35
:10BD9800084608BD582D002013B503688DF8071014
:10BDA8009C680DF107010123A04702B010BD07B53B
:10BDB80003688DF807101B6901220DF107019847E8
:10BDC80003B05DF804FB2DE9F0411D460368044605
:10BDD8005B690F4616469847236820461B689847B4
:10BDE800221D39462046FFF7D7FF2DB123682A4682
:10BDF8001B69314620469847236820465B68984768
:10BE0800236820469B69BDE8F0410C2118472DE9BD
:10BE1800F0411E46036804465B6915460F4698477D
:10BE2800236820461B689847221D39462046FFF79D
:10BE3800B3FF20460021FFF7BAFF23682046DB68DE
:10BE4800324629469847236820465B68BDE8F0419A
:10BE580018472DE9F0411F46036804465B690D4603
:10BE680016469847236820461B689847221D204697
:10BE78000D21FFF791FF290A2046FFF798FFE9B245
:10BE88002046FFF794FF236831463A4620461B694F
:10BE98009847236820465B689847236820469B6933
:10BEA800BDE8F0410C21184707B501238DF807209C
:10BEB8000DF10702FFF7CDFF03B05DF804FB2DE994
:10BEC800F0411F46036804465B690D4616469847CD
:10BED800236820461B689847221D20461D21FFF72E
:10BEE8005BFF290A2046FFF762FFE9B22046FFF709
:10BEF8005EFF20460021FFF75AFF23682046DB68D3
:10BF08003A4631469847236820465B68BDE8F041C9
:10BF1800184707B501230DF10702FFF7D0FF9DF879
:10BF2800070003B05DF804FB2DE9F0411E460368E5
:10BF380004465B690F4615469847236820461B68E8
:10BF48009847221D20460E21FFF726FF3946204636
:10BF5800FFF72DFF23682946324620461B6998477C
:10BF6800236820465B689847236820469B69BDE89C
:10BF7800F0410C2118472DE9F0411E46036804469C
:10BF88005B690F4615469847236820461B68984703
:10BF9800221D20461E21FFF7FFFE39462046FFF7E7
:10BFA80006FF20460021FFF702FF23682046DB68D2
:10BFB800324629469847236820465B68BDE8F04129
:10BFC800184710B5002304461A46C021FFF7FBFEA8
:10BFD800207910BD37B504460D468DF807100123AA
:10BFE80080210DF10702FFF7EEFE2368012D9B6902
:10BFF8000CBF322140F2DC51204603B0BDE830408E
:10C00800184737B501230C468DF807100DF10702C4
:10C018008A210546FFF7D7FEAC7103B030BD07B5DE
:10C02800042309BA01910DEB03028621FFF7CBFE29
:10C0380003B05DF804FB07B502238DF804108DF8F2
:10C0480005208F2101AAFFF7BEFE03B05DF804FBAF
:10C0580037B58DF8063000238DF8073004230446E1
:10C0680015468DF804108DF805208B210DEB030281
:10C07800FFF7A9FE40F689012046FFF74AFF062D83
:10C0880016BF40F0040200F0FB02D2B240F689016C
:10C0980020468DF80420FFF707FF03B030BD73B5C5
:10C0A80015468DF8033000229DF818309DF81C6065
:10C0B8008DF8002004468DF801108DF804308C218D
:10C0C80006236A468DF802508DF80560FFF77BFE5F
:10C0D80040F236712046FFF71CFF5EB100F0FB020C
:10C0E80040F2367120468DF80020FFF7DDFE6571BD
:10C0F80002B070BD40F00402D2B2F1E707B55BBAF6
:10C10800ADF80430BDF810305BBAADF8063049BA66
:10C11800082352BAADF80010ADF8022019466A4655
:10C12800FFF751FE03B05DF804FB07B5022301AA2F
:10C138001221FFF76CFE9DF804309DF8050000EB16
:10C14800032080B203B05DF804FB07B5022349BAA7
:10C15800ADF8041001AA1946FFF735FE03B05DF8E3
:10C1680004FB07B502238DF804108DF805208E21F5
:10C1780001AAFFF728FE03B05DF804FB13B56FF0C2
:10C188007F43994228BF19460B0C04468DF80430AA
:10C198000B0A8DF805308DF8061001AA03238321B8
:10C1A800FFF711FE236864219B692046984702B077
:10C1B80010BD13B56FF07F43994228BF19460B0C89
:10C1C80004468DF804300B0A8DF805308DF80610FA
:10C1D80001AA03238221FFF7F6FD236864219B69E6
:10C1E8002046984702B010BD37B503230D461446C4
:10C1F800142101AAFFF70BFE9DF804305B085B428F
:10C208002B809DF90530002BB8BF03339B1023709A
:10C2180003B030BD37B502230D461446132101AAD9
:10C22800FFF7F5FD9DF804302B709DF8053023705D
:10C2380003B030BD10B543680D4A23F07F4323F0A7
:10C24800FF039342044611D1002240F60211FFF782
:10C258002BFE40F644112046FFF75BFE40F0020239
:10C26800D2B240F644112046FFF71EFE10BD00BFB3
:10C278000001010070B505460E46FFF756FF31462E
:10C2880004462846FFF761FFA30702D52846FFF7B3
:10C29800D1FF204670BD07B5002914BF40232023D5
:10C2A8008DF807300DF1070201239321FFF78BFD6D
:10C2B80003B05DF804FB10B5002304461A46C121FB
:10C2C800FFF781FD236820469B69BDE810404621A1
:10C2D800184708B5FFF775FE80B208BD07B50023FB
:10C2E800ADF8043001AA02230721FFF76CFD03B063
:10C2F8005DF804FB07B5130C8DF8053052BA04231A
:10C308008DF80410ADF8062097210DEB0302FFF716
:10C318005AFD03B05DF804FB08B50A4640F6AC01C7
:10C32800FFF7C2FD08BD10B540F6D8010446FFF777
:10C33800F0FD40F01E02D2B240F6D8012046FFF7C9
:10C34800B3FD10BD08B50A4640F6E701FFF7ACFD9E
:10C3580008BD000007B5054B019304230DEB03024C
:10C368009521FFF730FD03B05DF804FB04070001D9
:10C3780007B502238DF804108DF80520982101AA2D
:10C38800FFF721FD03B05DF804FB0000000000008A
:10C3980013B504461C48B0FBF1F1080C8DF80000F9
:10C3A800080A8DF8010004988DF803208DF80430F0
:10C3B8008DF80210F4F730F811A3D3E90023F4F74D
:10C3C800CFF9F4F7B5FA030C8DF8053043BA6A468D
:10C3D800ADF80630204608238B21FFF7F4FC40F621
:10C3E80089012046FFF795FD40F00402D2B240F6DD
:10C3F800890120468DF80020FFF756FD02B010BDD8
:10C40800000000008084EE3F0000093D1FB58DF854
:10C4180007309DF818308DF808309DF81C308DF8DD
:10C4280009309DF820308DF80A309DF824308DF8B9
:10C438000B3049BA9DF82830ADF804108DF8062065
:10C448008DF80C3001AA09238C21FFF7BCFC05B03C
:10C458005DF804FB07B5002349BAADF80010ADF844
:10C46800023001936A4608234FF4D861FFF7F1FCC4
:10C4780003B05DF804FB13B503230C4601AA14218D
:10C48800FFF7C5FC9DF806305B085B42238002B0CD
:10C4980010BD0000C0F3C7537F3B162B10B50146F3
:10C4A80014DC002B07DA013300F0004101D141F020
:10C4B8007E51084610BD084A1A411042F9D04FF47F
:10C4C80080011941014421EA0201F2E7802BF0D1F1
:10C4D800F4F754FA0146ECE7FFFF7F00884210B5F5
:10C4E80001EB020402D98442234607D8431EA14225
:10C4F80008D011F8012B03F8012FF8E70244014690
:10C508008A4200D110BD13F8014D02F8014DF7E73A
:10C5180002440346934200D1704703F8011BF9E730
:10C5280010B50246147813460132002CFAD1013BAB
:10C5380011F8012B03F8012F002AF9D110BDC9B257
:10C548000346184613F8012B12B18A42F9D17047F5
:10C55800002918BF0020704710B56AB10139841846
:10C5680010F8012B11F8013F9A4203D1A04201D0E3
:10C57800002AF5D1D01A10BD1046FCE770B50D4D54
:10C588000D4C641BA4100026A64209D10B4D0C4C7F
:10C5980000F02EF8641BA4100026A64205D170BD39
:10C5A80055F8043B98470136EEE755F8043B9847A1
:10C5B8000136F2E70CE500080CE500080CE5000878
:10C5C80014E50008034611F8012B03F8012B002A93
:10C5D800F9D170470A44914200F1FF3300D1704706
:10C5E80010B511F8014B03F8014F9142F9D110BD74
:10C5F800F8B500BFF8BC08BC9E467047F8B500BF48
:08C60800F8BC08BC9E46704717
:10C6100000206C0002206A006D0074000205010217
:10C620000201000000000000010000000200000004
:10C630006D696E2C00206D572C0020572C00322E77
:10C640003447003931354D003836384D00343333F6
:10C650004D003730636D003836364D003F003530C1
:10C66000487A003331487A003139487A00464C52D2
:10C67000430046534B003139487A377800011F1385
:10C680006F01130000D57FAAFE2B815429FC56832D
:10C69000D702A87D52872DF8AC79D3067BAE04D1A2
:10C6A0008550FA2FA471DB0E5A8F25F08D58F22792
:10C6B00073A60CD9F623895C08DD77A2DF0AA07582
:10C6C00021F45E8B9D48E23763B61CC9B461CB1E72
:10C6D0004A9F35E0CF1AB06531E44E9BE633994C62
:10C6E00018CD67B239EC4693C712B86D10C56FBA52
:10C6F000EE3B91446BBE14C19540EA3F42973DE842
:10C70000BC69C316EF3A904511C46EBBC613B96C31
:10C7100038ED4792BD68C21743963CE99441EB3E21
:10C720006ABF15C04B9E34E1B560CA1F62B71DC811
:10C730009C49E33619CC66B3E732984D30E54F9A01
:10C74000CE1BB16472A70DD88C59F3265B8E24F1F1
:10C75000A570DA0F20F55F8ADE0BA17409DC76A3E1
:10C76000F722885DD603A97C28FD5782FF2A8055D1
:10C7700001D47EAB8451FB2E7AAF05D0AD78D207C1
:10C7800053862CF96162636465666768696A6B6CDD
:10C790006D6E6F707172737475767778797A3031E7
:10C7A00032333435363738395F232D2E00000100FF
:10C7B0000100020002000200030004000500060060
:10C7C00008000A000C0010001400190020002800C6
:10C7D00032003F00500064007D009E00C800FA0057
:10C7E0003C019001F40176022003E803E204DC0539
:10C7F000D007000000000000000000003B1A000805
:10C800000000000000000000471A000800000000BF
:10C8100000000000231A00086D6C72732E30005364
:10C8200065747570537461727453747834527800FF
:10C83000536574757053746172744D61726B657277
:10C840000021656E64210044495920453737204551
:10C850003232204475616C42616E64006D4C5253FB
:10C8600001020304006D4C525304030201000A004C
:10C8700040504152414D2F706172616D2E70636B5B
:10C88000006661696C20610020005378206E6F742F
:10C89000206F6B00537832206E6F74206F6B002E08
:10C8A000000000000000000000000000E522000879
:10C8B000FD2200089D2B0008C92B0008E72B00086B
:10C8C0000D270008E91B0008893E00080000000051
:10C8D00000000000011F0008ED1E0008AB2C00083E
:10C8E000D52C0008F32C0008AD270008E91B000830
:10C8F000713E00080000000000000000551B000809
:10C900009B300008712F00085B1B0008B72E000841
:10C910005D1C0008152F0008C1220008E12E000848
:10C920006B1C00080000000000000000551B000800
:10C93000571B0008591B00085B1B00085F1B000801
:10C94000611B0008651B0008691B00086B1B0008C1
:10C950006F1B00080000000000000000AB4F000843
:10C96000495000082D5000080D500008000000003C
:10C9700000000000551B0008891C0008591B000816
:10C980005B1B0008B58700082D8800081971000896
:10C99000917100086B1B00086F1B0008414E474C4B
:10C9A0004500484F52495A4F4E004E415620414C87
:10C9B00054484F4C440048454144494E4720484F55
:10C9C0004C44004845414446524545004845414491
:10C9D00041444A0043414D53544142004E41562088
:10C9E000525448004E415620504F53484F4C44003B
:10C9F0004D414E55414C00424545504552004C4535
:10CA00004453204F4646004C4947485453004F5327
:10CA100044204F46460054454C454D45545259001C
:10CA20004155544F2054554E4500424C41434B42D2
:10CA30004F58004641494C53414645004E4156200F
:10CA4000575000414952204D4F444500484F4D45F5
:10CA500020524553455400474353204E415600460B
:10CA6000505620414E474C45204D49580053555291
:10CA70004641434500464C415045524F4E005455A7
:10CA8000524E20415353495354004E4156204C417D
:10CA9000554E434800534552564F204155544F542C
:10CAA00052494D0043414D45524120434F4E54524F
:10CAB0004F4C20310043414D45524120434F4E548D
:10CAC000524F4C20320043414D45524120434F4E7E
:10CAD00054524F4C2033004F534420414C5420318A
:10CAE000004F534420414C542032004F53442041C6
:10CAF0004C542033004E415620434F55525345204D
:10CB0000484F4C44004D43204252414B494E470050
:10CB100055534552310055534552320055534552F5
:10CB200033005553455234004C4F4954455220432D
:10CB300048414E4745004D5350205243204F5645E3
:10CB400052524944450050524541524D00545552AD
:10CB5000544C45004E4156204352554953450041DF
:10CB600055544F204C4556454C205452494D005782
:10CB70005020504C414E4E455200534F4152494E69
:10CB800047004D495353494F4E204348414E474576
:10CB900000424545504552204D555445004D554C99
:10CBA00054492046554E4354494F4E004D4958452F
:10CBB000522050524F46494C452032004D4958456D
:10CBC00052205452414E534954494F4E00414E4712
:10CBD0004C4520484F4C4400800CD007B704C71B7D
:10CBE000800CB7040410020A0B06972304100B06EE
:10CBF0000001020503040000000000000000000026
:10CC000000000000000000007CDF00082B00000096
:10CC10006AE200080100000054DF00080A0000007A
:10CC200069E20008010000000000000000000000B0
:10CC3000000000000000000048DF000803000000C2
:10CC400068E2000801000000000000000000000091
:10CC50000000000000000000800080FF00000100D4
:10CC60000A000A000E0019001400640016009E005D
:10CC70006162636465666768696A6B6C6D6E6F702C
:10CC80007172737475767778797A303132333435DE
:10CC9000363738395F232D2E0000000000070E09BB
:10CCA0001C1B1215383F363124232A2D70777E79CC
:10CCB0006C6B6265484F464154535A5DE0E7EEE9BC
:10CCC000FCFBF2F5D8DFD6D1C4C3CACD90979E99AC
:10CCD0008C8B8285A8AFA6A1B4B3BABDC7C0C9CE9C
:10CCE000DBDCD5D2FFF8F1F6E3E4EDEAB7B0B9BE8C
:10CCF000ABACA5A28F88818693949D9A2720292E7C
:10CD00003B3C35321F18111603040D0A5750595E6B
:10CD10004B4C45426F68616673747D7A898E87805B
:10CD200095929B9CB1B6BFB8ADAAA3A4F9FEF7F04B
:10CD3000E5E2EBECC1C6CFC8DDDAD3D4696E67603B
:10CD400075727B7C51565F584D4A4344191E17102B
:10CD500005020B0C21262F283D3A33344E4940471B
:10CD600052555C5B7671787F6A6D64633E3930370B
:10CD700022252C2B0601080F1A1D1413AEA9A0A7FB
:10CD8000B2B5BCBB9691989F8A8D8483DED9D0D7EB
:10CD9000C2C5CCCBE6E1E8EFFAFDF4F300000000F9
:10CDA0003209000000000000010000007C2B0000A0
:10CDB0000000000002000000890C000000000000DC
:10CDC00004000000ED0E030C0D0000000500000043
:10CDD000D91C0100000000000600000068030000EC
:10CDE00000000000070000007720000000000000A5
:10CDF0000800000075240000000000000B00000087
:10CE00005906010400000000130000008918030403
:10CE10000500000014000000D61403020300000007
:10CE2000150000009F020300010000001600000032
:10CE3000DC1900000000000017000000A817030420
:10CE40000500000018000000183400000000000079
:10CE50001900000017650000000000001A00000023
:10CE6000AA180000000000001B000000901D000038
:10CE7000000000001C000000431000000000000043
:10CE80001D00000073100000000000001E000000E4
:10CE9000271C0000000000001F000000F63000000A
:10CEA0000000000020000000B91C0000000000008D
:10CEB00021000000681C00000000000022000000AB
:10CEC000ED1600000000000023000000F416000032
:10CED0000000000024000000DE250000000000002B
:10CEE00025000000D4070304050000002600000010
:10CEF000090703040500000027000000FE260320A8
:10CF00002100000028000000E605030203000000E5
:10CF1000290000001C040302030000002A00000096
:10CF20001C120000000000002B000000840303001E
:10CF3000010000002C000000DD09030203000000D6
:10CF40002D000000E8030300010000002E00000097
:10CF50000B020000000000002F00000099080300F1
:10CF600001000000300000002915010C0000000045
:10CF70003100000027140000000000003200000013
:10CF80004E2503121300000033000000C405030205
:10CF90000300000035000000030500000000000051
:10CFA000360000000F1B03181900000037000000B6
:10CFB00003190000000000003D000000A748000029
:10CFC000000000003E000000B71A00000000000052
:10CFD0003F00000077B500000000000040000000A6
:10CFE000BFE100000000000041000000762A0000C0
:10CFF000000000004200000094060302030000004D
:10D00000430000001504000000000000450000007F
:10D01000F31E010A00000000460000007C260310F9
:10D020001100000049000000262603202100000016
:10D030004A00000014140000000000004B00000033
:10D040009E23031E1F0000004C0000009821031EB9
:10D050001F0000004D0000008F0A030809000000B7
:10D06000500000000E040302030000005100000005
:10D070006A16000000000000520000003133032453
:10D0800025000000530000001625000000000000ED
:10D09000540000008F3503323300000055000000BB
:10D0A0008C330000000000005600000005350332FC
:10D0B000330000005700000096330000000000001D
:10D0C00059000000E71C0000000000005A000000AA
:10D0D000B7380000000000005B0000003F2A00009D
:10D0E000000000005C00000036210000000000008D
:10D0F0005D0000002F5100000000000064000000EF
:10D10000AF2200000000000065000000667500000E
:10D1100000000000660000009E7500000000000096
:10D1200067000000D0390000000000006800000027
:10D130003874000000000000690000005D3F00003E
:10D14000000000006A0000008A2C000000000000BF
:10D150006B0000006C410000000000006C0000004B
:10D16000205C0000000000006D000000B909000014
:10D17000000000006E00000054FE030102000000E9
:10D180006F00000022120310110000007000000068
:10D19000AE0C000000000000710000007C270000C1
:10D1A0000000000072000000ED2C000000000000F4
:10D1B0007300000004400000000000007400000044
:10D1C0004C180000000000007500000080060304F9
:10D1D0000500000076000000380E0000000000008E
:10D1E00077000000740C030A0B00000078000000B8
:10D1F000866100000000000079000000ED020300DD
:10D20000010000007A000000CB02030001000000D2
:10D210007B000000FA710300010000007C000000A8
:10D2200057390000000000007D000000CB06000020
:10D23000000000007E000000DC51034F50000000A1
:10D240007F000000192300000000000080000000A3
:10D25000E223000000000000810000002E18000002
:10D2600000000000820000001D0D00000000000012
:10D2700083000000DFFF00000000000084000000C9
:10D280005527000000000000850000000612000085
:10D290000000000086000000E52B000000000000F8
:10D2A00087000000CB08000000000000880000009C
:10D2B000011600000000000089000000C3100000FB
:10D2C000000000008A0000006D78000000000000EF
:10D2D0008B000000A82B03292A0000008C0000000E
:10D2E000B5290000000000008D0000002F20000084
:10D2F000000000008E00000048F300000000000065
:10D300008F0000008310000000000000900000006B
:10D310007F5D0000000000009200000067640000D4
:10D3200000000000930000009A360000000000009A
:10D3300094000000B24E00000000000095000000C4
:10D34000C83C00000000000096000000862A000093
:10D350000000000097000000DB0803060700000043
:10D3600098000000D00800000000000099000000B4
:10D37000BC0C0000000000009A000000540F0306DF
:10D38000070000009B000000160D030405000000CC
:10D390009C00000013060300010000009D00000037
:10D3A000150F030C0D0000009E000000860F030CFB
:10D3B0000D000000A00000004E0C03080900000052
:10D3C000A10000004403030001000000A2000000CF
:10D3D000BD09000000000000A30000007F1C000049
:10D3E00000000000A40000009A2C000000000000D3
:10D3F000A50000001503000000000000A6000000CA
:10D400001509000000000000A700000090160000B1
:10D4100000000000A8000000010C00000000000057
:10D42000A9000000EA12000000000000AA000000AD
:10D430004922000000000000AB000000B5420000DF
:10D4400000000000AC0000001662000000000000B8
:10D45000AD0000005308000000000000AE00000016
:10D46000A730000000000000AF0000008A13030E88
:10D470000F000000B0000000EA03030001000000FC
:10D48000B1000000F014000000000000B200000035
:10D490002F18000000000000B3000000BD1D011A9D
:10D4A00000000000B4000000342F012A000000003A
:10D4B000B5000000AE04000000000000B60000004F
:10D4C000E528000000000000B7000000550203003E
:10D4D00001000000B80000009FCE0304050000001A
:10D4E000B9000000BA07030405000000BA000000FC
:10D4F000481D030001000000BF0000005C1B00008D
:10D5000000000000C0000000243600000000000001
:10D51000C1000000471A000000000000C200000027
:10D520006221000000000000C30000007825000018
:10D5300000000000C8000000862A0328290000001F
:10D54000C9000000CD0E030C0D000000D600000045
:10D550004508030607000000D7000000650300002F
:10D5600000000000D80000003203030001000000AA
:10D57000D9000000CA06000000000000DA00000028
:10D580001107030001000000DB000000A202000000
:10D5900000000000DC00000022200000000000006D
:10D5A000DD000000472A000000000000DE0000004F
:10D5B0000F03000000000000DF000000772F032AA7
:10D5C0002B000000E0000000662D032A2B00000065
:10D5D000E1000000D049000000000000E20000006F
:10D5E000CF08000000000000E6000000A32A0000B1
:10D5F00000000000E70000006928000000000000B3
:10D60000E80000009741000000000000E900000071
:10D6100023B6000000000000EA0000009628000089
:10D6200000000000EB000000B32A00000000000032
:10D63000F10000005A20000000000000F20000008D
:10D64000683C000000000000F3000000553D01347C
:10D6500000000000F40000005F0600000000000071
:10D66000F50000008202000000000000F60000004B
:10D67000B826000000000000F70000005113000071
:10D6800000000000F800000008FE03030400000092
:10D69000F9000000CC24000000000000FA000000A7
:10D6A000311E000000000000FB000000AA12000074
:10D6B00000000000FC0000002C1200000000000030
:10D6C000FD0000005336000000000000FE000000D6
:10D6D0002E0900000000000000010000472A030896
:10D6E00009000000010100008309000000000000A3
:10D6F00002010000BBE8030001000000030100007C
:10D700005CED00000000000004010000920E00002B
:10D710000000000005010000B33D00000000000013
:10D72000060100000C1700000000000007010000C7
:10D7300085FF00000000000008010000312000000B
:10D7400000000000090100001A14000000000000A1
:10D750000A010000C1FF0302030000000B010000EA
:10D7600023FF0302030000000C0100000E0403026B
:10D77000030000000D0100006DD700000000000054
:10D780000E0100003B140000000000000F0100002B
:10D790001635000000000000130100007E2000008C
:10D7A0000000000014010000123200000000000020
:10D7B000150100003E1E00000000000018010000DE
:10D7C000462100000000000019010000300D00009B
:10D7D000000000001A0100007B230320210000004C
:10D7E0001B0100004A910000000000001C01000025
:10D7F0006320031E1F0000001D0100008931032665
:10D80000270000001E010000D2390332330000005F
:10D810001F01000001170314150000002001000083
:10D82000141703141500000022010000FB2E000055
:10D8300000000000230100000A3900000000000081
:10D8400027010000EA0C0000000000002A0100008F
:10D85000ED250000000000002B0100001362000015
:10D86000000000002C010000D9160000000000009C
:10D870002D010000F33A0000000000003601000016
:10D880001C11000000000000370100005F74000060
:10D890000000000040010000F31403020300000038
:10D8A0004101000058020300010000004201000095
:10D8B000F395000000000000430100004E930300B8
:10D8C00001000000440100008492000000000000FC
:10D8D0004A01000017A70000000000004B010000F3
:10D8E0005BE90000000000004C010000ECEF0000CC
:10D8F000000000004D010000E76D00000000000086
:10D900004E010000480A0000000000004F01000026
:10D91000E11800000000000050010000F554000074
:10D920000000000053010000C705000000000000D7
:10D930005401000063460000000000005E0100008A
:10D94000E8FC00000000000062010000D20E030CA1
:10D950000D00000063010000060C00000000000044
:10D96000680100000B1900000000000069010000C0
:10D970005D21000000000000710100009718000008
:10D9800000000000720100001A8C0000000000007E
:10D99000730100000A1A0000000000007501000079
:10D9A000752A00000000000077010000FB8C0000D9
:10D9B0000000000078010000C7080000000000001F
:10D9C0007C010000E814000000000000810100005C
:10D9D0009385030203000000820100008410030409
:10D9E0000500000083010000044803040500000056
:10D9F00084010000082503202100000086010000AA
:10DA00009CEE0000000000008B01000000D400002C
:10DA1000000000008C01000032A0000000000000A7
:10DA20008D010000B66C00000000000090010000B5
:10DA30006EFE03040500000091010000B706030418
:10DA4000050000009A010000A03500000000000061
:10DA50009B0100006A030000000000009C01000020
:10DA600021060304050000009D0100004D0703048A
:10DA7000050000009E0100006D1000000000000085
:10DA80009F010000A110000000000000A4010000A0
:10DA90001449030607000000B3010000862E0000B1
:10DAA00000000000B4010000C109000000000000F7
:10DAB000B50100001E01000000000000B8010000D8
:10DAC0004223000000000000B9010000A91100007D
:10DAD00000000000FE010000F56A000000000000E8
:10DAE000FF0100001C47000000000000421F000072
:10DAF000DA10000000000000431F0000E7290000CA
:10DB000000000000441F0000AC62000000000000A4
:10DB1000451F0000FB26000000000000461F00001B
:10DB2000610E000000000000471F000040200000C0
:10DB300000000000481F0000EA2100000000000073
:10DB4000491F000090100000000000004A1F000064
:10DB50009B290000000000004B1F0000146600001D
:10DB6000000000004C1F0000361000000000000004
:10DB70004D1F0000DE2E0000000000004E1F0000C0
:10DB8000C80E0000000000004F1F00001718000022
:10DB900000000000501F000095120000000000006F
:10DBA0002823000071890000000000002D230000E0
:10DBB000752200000000000011270000D1140000B1
:10DBC0000000000012270000BA2900000000000039
:10DBD000132700000401000000000000A727000038
:10DBE000C355000000000000F82A0000863403043A
:10DBF00005000000F92A00000F8800000000000066
:10DC0000FA2A0000EAB4030405000000FB2A000021
:10DC10004005000000000000FC2A00000BE803089B
:10DC200009000000FD2A00005DE600000000000081
:10DC3000022B00002E31000000000000032B00002A
:10DC40006A2C0000000000000C2B0000CD1000002A
:10DC500000000000162B0000902C000000000000C7
:10DC6000172B0000852C000000000000182B00007E
:10DC7000552C000000000000192B0000C3250310E4
:10DC8000110000001A2B00004F05000000000000EA
:10DC90001B2B000080080304050000001C2B000063
:10DCA000B1220000000000001D2B0000821C0000BB
:10DCB000000000001E2B00002F26000000000000C6
:10DCC0001F2B00008E09000000000000202B000028
:10DCD000842C000000000000212B0000D02C00004C
:10DCE00000000000222B0000C92C000000000000F2
:10DCF000232B0000C12C000000000000242B00009A
:10DD0000BD2C00000000000064320000722C0300F3
:10DD10000100000065320000FE3B031E1F000000F2
:10DD2000663200008C3503040500000067320000F5
:10DD3000F92E030001000000683200004D36031C7C
:10DD40001D00000069320000312B030001000000BB
:10DD5000733200005EF9030001000000763200001B
:10DD60008B33000000000000773200000712031020
:10DD700011000000783200001405000000000000CF
:10DD80006842000067B3000000000000FE4200008F
:10DD90001A21000000000000FF42000048100000AF
:10DDA000000000000143000013110000000000000B
:10DDB000024300005911000000000000034300006E
:10DDC0001B0A000000000000044300000E5B00007E
:10DDD0000000000005430000BB54000000000000EC
:10DDE000064300006A1800000000000010A40000B4
:10DDF000E30100000000000011A40000EF2E00006D
:10DE00000000000051C30000F620000000000000E8
:10DE100052C30000B5F600000000000053C300002C
:10DE20003E1300000000000054C30000F00A030885
:10DE30000900000055C30000980603040500000017
:10DE400020CB00000D6400000000000021CB00008A
:10DE5000EF0100000000000022CB000018010000CC
:10DE60000000000023CB0000A61A00000000000004
:10DE700024CB0000270100000000000025CB00009B
:10DE8000910100000000000060EA00000416031485
:10DE9000150000006AEA0000D02100000000000028
:10DEA0006BEA0000B7070000000000006CEA000009
:10DEB00063240320210000006DEA00008118031490
:10DEC000150000006EEA000086080304050000004B
:10DED00074EA0000CA0400000000000088EA0000A4
:10DEE0009CF500000000000089EA0000BFFF000070
:10DEF000000000008DEA00000E170302030000007E
:10DF00008EEA0000AB1C0308090000008FEA000045
:10DF1000370700000000000092EA0000DC0E00005D
:10DF20000000000093EA0000F51800000000000067
:10DF300094EA0000652C00000000000095EA000053
:10DF40002D060000000000008FC2151B51B81E1BDB
:10DF500014AE171B6666F435CCCCFC35333305366E
:10DF600099990D360000163666661E36CCCC2636DC
:10DF700033332F3699993736000040366666663857
:10DF8000000070389999793833338338CCCC8C3889
:10DF9000666696380000A0389999A9383333B338AB
:10DFA000CCCCBC386666C6380000D0389999D938D0
:10DFB0003333E338CCCCEC386666F63800000039F1
:10DFC0009999093933331339CCCC1C396666263913
:10DFD000000030399999393933334339CCCC4C3935
:10DFE0006666563900006039999969393333733957
:10DFF000CCCC7C396666863900009039999999397C
:10E000003333A339CCCCAC396666B6390000C0399D
:10E010009999C9393333D339CCCCDC396666E639C2
:10E020000000F0399999F9390000891112239B32C7
:10E030002446AD573665BF74488CC19D5AAFD3BED8
:10E040006CCAE5DB7EE9F7F88110080193331A22E8
:10E05000A5562C47B7753E64C99C408DDBBF52AEB8
:10E06000EDDA64CBFFF976E802218B3010029913C8
:10E070002667AF763444BD554AADC3BC588ED19F98
:10E080006EEBE7FA7CC8F5D983310A2091121803A8
:10E09000A7772E66B5543C45CBBD42ACD99E508F78
:10E0A000EFFB66EAFDD874C904428D5316619F7078
:10E0B0002004A9153227BB364CCEC5DF5EEDD7FC58
:10E0C0006888E1997AABF3BA85520C4397711E6068
:10E0D000A1142805B3373A26CDDE44CFDFFD56EC38
:10E0E000E9986089FBBB72AA06638F7214409D5148
:10E0F0002225AB343006B9174EEFC7FE5CCCD5DD18
:10E100006AA9E3B8788AF19B87730E6295501C4127
:10E11000A3352A24B1163807CFFF46EEDDDC54CDF7
:10E12000EBB962A8F99A708B088481951AA793B607
:10E130002CC2A5D33EE1B7F04008C919522BDB3AF7
:10E14000644EED5F766DFF7C899400859BB712A6C7
:10E15000ADD224C3BFF136E0C1184809D33B5A2AD7
:10E16000E55E6C4FF77D7E6C0AA583B418869197A7
:10E170002EE3A7F23CC0B5D14229CB38500AD91BB7
:10E18000666FEF7E744CFD5D8BB502A49996108787
:10E19000AFF326E2BDD034C1C3394A28D11A580B97
:10E1A000E77F6E6EF55C7C4D0CC685D71EE597F457
:10E1B0002880A1913AA3B3B2444ACD5B5669DF7877
:10E1C000600CE91D722FFB3E8DD604C79FF516E447
:10E1D000A9902081BBB332A2C55A4C4BD7795E6857
:10E1E000E11C680DF33F7A2E0EE787F61CC495D527
:10E1F0002AA1A3B03882B193466BCF7A5448DD5937
:10E20000622DEB3C700EF91F8FF706E69DD414C506
:10E21000ABB122A0B9923083C77B4E6AD5585C4916
:10E22000E33D6A2CF11E780FA08601000B19000057
:10E2300050C300001000041000005B01010000004A
:10E24000B01D000096FF00000506010C015B0000F8
:10E250009033000091FF00000606010C015B0000F6
:10E260002058000090FF00000000130049CB000878
:10E27000000000009CC9000802000000A2C90008BC
:10E2800003000000AAC9000804000000B6C9000885
:10E2900005000000C3C9000806000000CCC9000842
:10E2A000FF000000D4C90008FF000000DCC900081E
:10E2B00007000000E4C9000808000000F0C90008D9
:10E2C00009000000F7C90008FF000000FEC90008AF
:10E2D000FF00000007CA0008FF0000000ECA000887
:10E2E000FF00000016CA0008FF00000020CA000856
:10E2F0000A0000002ACA0008FF00000033CA000814
:10E30000010000003CCA00080B00000043CA0008DE
:10E310000C0000004CCA0008FF00000057CA0008AB
:10E32000FF0000005FCA0008FF0000006DCA00087F
:10E33000FF00000075CA00080D0000007ECA00083A
:10E340000E0000008ACA00080F00000095CA0008ED
:10E35000FF000000A4CA0008FF000000B5CA0008C2
:10E36000FF000000C6CA0008FF000000D7CA00086E
:10E37000FF000000E1CA0008FF000000EBCA00082F
:10E38000FF000000F5CA00081000000005CB0008DF
:10E39000FF00000010CB0008FF00000016CB0008B3
:10E3A000FF0000001CCB0008FF00000022CB00088B
:10E3B000FF00000028CB0008FF00000036CB00085B
:10E3C000FF00000046CB0008FF0000004DCB000816
:10E3D0001100000054CB0008120000005FCB0008C1
:10E3E000FF0000006FCB0008FF0000007ACB0008A0
:10E3F0001300000082CB0008FF00000091CB000852
:10E40000FF0000009DCB0008FF000000ACCB00081F
:10E41000FF000000BCCB0008FF000000CDCB0008CF
:10E42000140000000000000000000000F99C00083B
:10E43000FB9C0008FF9C0008039D000801000000F1
:10E4400003000000050000000100000001000000C2
:10E45000060000000A00000020000000020000008A
:10E460000400000008000000100000004000000050
:10E470008000000000010000000200000000000019
:10E48000000000000000000000000000010000008B
:10E49000020000000300000004000000A08601004C
:10E4A000400D0300801A060000350C0040420F00AA
:10E4B00080841E0000093D0000127A000024F40050
:10E4C00000366E010048E801006CDC02000000002C
:10E4D000000000000000000000000000010000003B
:10E4E0000200000004000000060000000800000018
:10E4F0000A0000000C0000001000000020000000D6
:0CE500004000000080000000000100004E
:08E50C005D010008499C0008B4
:04E5140039010008C1
:10E5180090BADCFE785634120A0000002CC90008B4
:10E52800FCC80008FFFF000074C9000800093D008E
:08E538000100000010000000CA
:040000050800A6F554
:00000001FF
